:020000040040BA
:1040000080530020EDD94000F54E4000B94F4000EC
:10401000ADDA4000ADDA4000ADDA4000000000004B
:10402000000000000000000000000000A1DD4000D2
:10403000ADDA40000000000001DE400065DE400017
:10404000ADDA4000ADDA4000ADDA4000ADDA400054
:10405000ADDA4000ADDA4000ADDA4000000000000B
:10406000ADDA4000F5FF400000000000B9B54000A7
:10407000CDB54000FDD14000ADDA4000ADDA4000E2
:10408000ADDA4000ADDA40000DD24000418C400076
:1040900009004100ADDA4000ADDA4000495140006E
:1040A000ADDA4000ADDA4000ADDA4000ADDA4000F4
:1040B000ADDA4000A94A4000ADDA4000000000003F
:1040C00000000000000000000000000000000000F0
:1040D00000000000000000000000000000000000E0
:1040E00000000000000000000000000000000000D0
:1040F000000000000000000000000000ADDA4000F9
:10410000CDC64000ADDA4000000000000000000015
:10411000000000000000000000000000000000009F
:10412000000000000000000000000000000000008F
:10413000000000000000000000000000000000007F
:10414000000000000000000000000000000000006F
:10440000DC17010010B5054C237833B9044B13B108
:104410000448AFF300800123237010BDE80C002096
:1044200000000000F84A41000C4B43B10C480D4914
:1044300010B5AFF300800C48036823B910BD0A48DB
:10444000036833B97047094B002BF7D0BDE8104023
:104450001847064B002BF5D0184700BF000000009E
:10446000F84A4100EC0C0020F84A4100000000002E
:104470000120704770470120704700207047704747
:1044800001207047014B1878704700BF0C0D0020C9
:104490007047000058B908B5054B1B78012B00D0B8
:1044A00008BD044B1B68002BFAD09847F8E770470B
:1044B000100D0020040D002008B50C4B9847C37860
:1044C0000B4A1370012B0CD101220A4B1A700022E7
:1044D000094B1A80094B9847094B1B681BB1984739
:1044E00001E0084B9847012008BD00BF01B2400021
:1044F0000C0D0020100D00200E0D0020D5FF4000F7
:10450000040D0020E1FF400008B5054B1B78012B8E
:1045100000D008BD0022034B1A70034B9847F8E700
:104520000C0D0020100D0020E1FF400010B582B0FE
:10453000074B00930B46024600218420054CA04700
:1045400018B9054A13680133136002B010BD00BFEB
:104550009544400005CE4000080D0020014B186036
:10456000704700BF040D00202DE9F0474FF40046CE
:10457000BF4B5E600B20BF4CA0470C20A047BE4B3A
:104580004FF0400CC3F810C0C3F8A0C0C3F834C04B
:104590004FF0807EC3F810E0C3F8A0E0C3F834E029
:1045A000B64A01271761C2F8A0705763022414614C
:1045B000C2F8A04054631C61C3F8A0405C631F664E
:1045C000C3F890705F655F62C3F88070196F3943FC
:1045D0001967596F21F0010159675F604FF480310D
:1045E0001966C3F8901059655962C3F88010186FA6
:1045F00008431867586F20F48030586759601C6171
:10460000C3F8A0405C6304205861C3F8A00058665A
:10461000C3F8900058655862C3F88000196F21F004
:1046200004011967596F21F00401596718211966AF
:10463000C3F8901059655962C3F880101D6F25F0BA
:1046400018051D675D6F25F018055D675960082521
:104650001D66C3F890505D655D62C3F88050196FA8
:1046600021F008011967596F21F0080159675D6051
:1046700010211966C3F8901059655962C3F880106B
:10468000D3F8708028F01008C3F87080D3F87480D5
:1046900028F01008C3F8748059604FF48028C3F8DC
:1046A0001480C3F8A0804FF02009C3F81490C3F819
:1046B000A090C3F810C0C3F8A0C0C3F834C0C3F8BA
:1046C00010E0C3F8A0E0C3F834E01761C2F8A070AE
:1046D00057631461C2F8A04054634FF4007CC3F8E0
:1046E00060C0C3F890C0C3F854C0C3F824C0C3F876
:1046F00080C01C6F44EA0C041C675C6F24F40074D7
:104700005C67C3F804C04FF480641C66C3F8904033
:104710005C655C62C3F880401F6F27431F675F6F53
:1047200027F480675F675C604FF4006EC3F810E0A9
:10473000C3F8A0E0C3F834E04FF400275F61C3F88A
:10474000A0701F66C3F890705F655F62C3F88070E9
:104750001F6F27F400271F675F6F27F400275F672D
:104760004FF480175F61C3F8A0701F66C3F89070A4
:104770005F655F62C3F880701F6F27F480171F6743
:104780005F6F27F480175F674FF480575F61C3F84E
:10479000A0705F66C3F890705F655F62C3F8807059
:1047A0001F6F27F480571F675F6F27F480575F677D
:1047B0004FF400575F61C3F8A0704FF480775761E2
:1047C000C2F8A0704FF48048C3F86080C3F89080AE
:1047D000C3F85080C3F82480C3F88080D3F870A059
:1047E0002AF4804AC3F870A0D3F874A02AF4804A4F
:1047F000C3F874A0C3F81080C3F8A080C3F8308059
:104800005E61C3F8A0604FF400365E61C3F8A0603B
:104810001066C2F8900050655062C2F88000166FB2
:1048200026F004061667566F26F004065667506099
:104830001566C2F8905055655562C2F88050106FE9
:1048400020F008001067506F20F008005067556096
:104850000B4DD5F8140140F03000C5F8140151613A
:10486000C2F8A0105166C2F890105165516209E07B
:1048700050140E4035D74000000E0E4000100E4080
:1048800000020E40C2F88010116F21F01001116774
:10489000516F21F010015167C2F81090C2F8A0903A
:1048A000C2F83490C2F810C0C2F8A0C0C2F830C03C
:1048B0004FF400015961C3F8A0105966C3F8901075
:1048C00059655962C3F88010196F21F40001196706
:1048D000596F21F400015967C2F860E0C2F890E016
:1048E000C2F854E0C2F824E0C2F880E0116F21F46D
:1048F00000611167516F21F400615167C2F804E053
:104900001466C2F8904054655462C2F88040116F3A
:1049100021F480611167516F21F480615167546007
:104920001F66C3F890701F655F62C3F880701A6FCE
:1049300022F480721A675A6F22F480725A671F61DC
:10494000C3F8A0701F63BDE8F08700BF08B5034B34
:1049500053F8203003B1984708BD00BF6C10002009
:1049600010B582B0036B0193002400E00134172CD2
:1049700009D8064B53F82420019B1A42F6D0204652
:10498000034B9847F2E702B010BD00BFE83D41007D
:104990004D49400000230360064A4260064A826097
:1049A0004FF48022C2600222027442748374C37482
:1049B000037570470000DC05808D5B00036C1943B4
:1049C0000164704710B58B7C23B34FF000434A68F5
:1049D0008C686400B2FBF4F2013A120292B2134303
:1049E0000A7C120602F0706213434A7C120702F03E
:1049F00040521343CA6813434360CB7C63B14FF00A
:104A000080730A7D52B90022134303640968054B81
:104A1000984710BD0023DAE70023F2E74FF4801235
:104A2000F2E700BFBD49400008B5036B13F0807F7B
:104A300001D0192008BD01230360064B98470023CD
:104A400004E00021044A42F823100133172BF8D95F
:104A5000002008BDC54940006C100020B1F1FF3FA7
:104A600004D0044B53F82130436270474FF0FF33BA
:104A700043627047E83D410010B5084C44F82120DE
:104A8000074A4FF00054C2F880411B01DBB282F8A4
:104A90001D331460034B984710BD00BF6C100020FD
:104AA00000E100E05D4A400008B50248024B98472B
:104AB00008BD00BF008003406149400042F26663C8
:104AC00003FB00F008E000BF00BF00BF00BF00BF55
:104AD00000BF00BF00BF01380028F4D170470000BC
:104AE0000C4B1A68126802601B685A6842609A6828
:104AF0008260DB68C360084B1B68DA6802611A6970
:104B000042615A6982619A69C261DA6902621B6A0A
:104B10004362704724130020D81000200D4B1A6800
:104B2000526A02601B689A6A42600B4A12681169F5
:104B300081600A490968C1605169016191694161F7
:104B4000D26982611A68C2615A6802629B684362D4
:104B5000704700BFD810002024130020DC10002074
:104B6000FEE70000284B5B6A13F0010F05D0EFF35E
:104B70000583042B01D004207047234B5B6A13F09C
:104B8000020F05D0EFF30583052B01D005207047F8
:104B90001D4B5B6A13F0080F05D0EFF30583062B5E
:104BA00001D006207047184B5B6A13F0800F05D0C8
:104BB000EFF305830B2B01D00B207047124B5B6A80
:104BC00013F4807F05D0EFF305830C2B01D00C206C
:104BD00070470D4B5B6A13F4806F05D0EFF30583CC
:104BE0000E2B01D00E207047074B5B6A13F4006F49
:104BF00005D0EFF305830F2B03D00F207047002063
:104C000070470020704700BF00ED00E000230FE078
:104C1000114AD2F80412A3F120000122824011426D
:104C200005D0EFF3058203F11000904213D1013358
:104C3000312B0FD81F2BEBD8074AD2F800120122D4
:104C40009A401142F3D0EFF3058203F11000904235
:104C5000EDD070470020704700E100E010B5EFF3A1
:104C600008831C4613F0070F00D01C1F174B5B680E
:104C700013F0010F01D0B7EE000A154B5B6813F477
:104C8000006F15D0134A22F001026FF0060E0023C8
:104C900003F1807344F8043C44F8082C0E4B44F8AC
:104CA0000C3C203C84F3088884F30988704710BDCD
:104CB0000A4B9847034628B1094A22F001026FF0D7
:104CC0000E0EE5E7074B98470346F5E730EF00E0A7
:104CD00000ED00E07D4D4000614B4000654B400021
:104CE0005D4C40000D4C4000064A936823F07F4322
:104CF00023F4706343F0254343F4E0639360024B75
:104D00001360704700140E40080000A5024B1860A5
:104D1000024B1960704700BFD41000202013002000
:104D2000014B1870704700BF110D0020C0F3080040
:104D3000014B1880704700BFD010002008B5024614
:104D400050B9084B08491960084959600021996019
:104D50001046074B984708BD024B064919600649A3
:104D60005960F5E7FC0100209802002008020020AD
:104D70001DAB4000E0000020F800002008B56420D2
:104D80000A4B984762B661B60120094B9847094B18
:104D90009847094B98470A20044EB047074C022514
:104DA00065630A20B0472563F5E700BFBD4A4000B0
:104DB0003D4D40000DB24000EDFF4000000E0E40A2
:104DC000F8B505463D4B4FF0FF32C3F88020C3F8DD
:104DD0008420C3F88021C3F8842103F540635A6816
:104DE00042F020625A605A6A22F400425A62344BFE
:104DF0009A6D5A6C22F040625A645A6C42F000621A
:104E00005A64304C4FF4804363634FF40063636330
:104E10004FF48073636302202B4EB0474FF08073D2
:104E200063630420B047294F01237B630420B0470C
:104E300002237B6340236363254A136823F0010345
:104E40001360244B5A6F42F480725A675A6F42F4CF
:104E500000725A67204AD2F8143143F44063C2F812
:104E60001431002383F311881C4B1D60EB6A13F08F
:104E7000040F1FD06A681A4B1A60194B1A6802F1A6
:104E8000200318490B60526912F0100F01D048330B
:104E90000B60AB6813F4007F03D0124A136804332D
:104EA0001360114B1B7813B90322104B1A80104B5F
:104EB0009847F8BD2A680A4B1A60DEE700E100E077
:104EC00000000140000E0E40BD4A400000100E40A0
:104ED00010E000E00040044000020E40D810002026
:104EE00024130020DC100020110D0020D010002021
:104EF0005D4C40006FF0060E7047704738B50446B1
:104F0000402200212048214B98472378433B112B16
:104F100013D8DFE803F03612121212121212121214
:104F20001212121212091627174B52221A70184A1F
:104F300012785A70174A12885A801348164B9847AD
:104F400038BD114B53221A7062785A702822DA70D9
:104F500063781BB91148124B9847EEE70F48114B85
:104F60009847EAE7084C542323700F4D1021286816
:104F70000E4B9847C2B262702968A01C0C4B984730
:104F8000DBE70C4B9847D8E7E01200209D16410064
:104F9000110D0020D010002029AB4000E4120020A9
:104FA000E14A40001D4B4000201300201D1A410023
:104FB000A1144100E94C400072B671B6EFF30383CF
:104FC000EFF30982EFF30881DFF814D02DE9FE4FEB
:104FD0006846FFF7F5FEBDE8FE4F8D4670470000BE
:104FE000E012002010B51720234CA0471820A0473E
:104FF000224B4FF480321A66C3F890205A655A62E9
:10500000C3F88020196F11431967596F21F480315B
:1050100059675A6001225A66C3F890205A655A624D
:10502000C3F88020196F11431967596F21F00101EE
:1050300059675A60A3F5206340F21262DA644FF4B4
:1050400000621A600E4B0F4A5A6041225A620521D3
:1050500019600D4A5A644FF4F572DA6500229A65B8
:1050600019640A4B1A700A4B4FF400021A6070223E
:1050700083F8172310BD00BF35D74000000E0E4047
:10508000000001400406090001C4000A2C1300209E
:1050900000E100E010B54FF40002124BC3F880208D
:1050A000BFF34F8FBFF36F8F0F4B4FF480321A66F1
:1050B000C3F890205A655A62C3F88020196F21F412
:1050C00080311967596F21F4803159671A601A616C
:1050D000C3F8A0205A631720044CA0471820A0470B
:1050E00010BD00BF00E100E0000E0E4089D7400077
:1050F000642800D964200F4AD36D03FB00F30E49E6
:10510000A1FB03135B09936548B10A4B5A6C22F06B
:1051100040625A645A6C42F080625A647047134687
:10512000526C22F040625A645A6C42F000625A6437
:10513000704700BF000001401F85EB51014B1888EC
:10514000704700BF301300200F4B1B6A13F0010F94
:1051500006D000220D490A700D490A600D490A6007
:1051600013F0400F0ED00122084B1A70064B9A69BB
:10517000094BB3FBF2F3064A1360C3EB03139A0027
:10518000044B1A60704700BF000001402C13002040
:1051900028130020301300201F1A0500014B18703F
:1051A000704700BF00010020064B1B7823B94FF465
:1051B0000062054B1A6370474FF40062024B5A635A
:1051C000704700BF00010020000E0E40064B1B7808
:1051D00023B94FF40062054B5A6370474FF40062E5
:1051E000024B1A63704700BF00010020000E0E4002
:1051F0002DE9F04186B00F4616469846B8B9344BB3
:10520000984704460025049598238DF8043001231F
:105210008DF805308DF8065002238DF8083005AB67
:1052200003938DF8075020462A4B98470EE02A4BEF
:1052300098470446E6E72046284B9847002044E07C
:105240009DF8153008F805300135EDB2B54238D279
:105250008DF814708DF8155000238DF80630322229
:1052600001A920461E4B9847A379DBB2022B0BD035
:1052700020461C4B9847322201A92046184B9847DC
:10528000A379DBB2022BD6D101238DF8063032226E
:1052900001A92046124B9847A379DBB2022BCFD04D
:1052A0002046104B9847322201A920460C4B9847C4
:1052B000A379DBB2022BC3D02046084B98470020CD
:1052C00003E02046054B9847012006B0BDE8F08179
:1052D000C5FF400015704000CDFF40002970400020
:1052E00041704000F17140002DE9F04186B00C465C
:1052F00017469846D8B9264B984705460026049687
:1053000098238DF8043001238DF8053002238DF8A1
:10531000063003238DF8083005AB03938DF8074062
:105320008DF8156028461B4B9847344605E01A4B0C
:1053300098470546E2E70134E4B2BC4221D28DF839
:10534000144018F804308DF81630322201A928468E
:10535000124B98470646AB79DBB2022BEBD02846BE
:105360000F4B9847322201A928460C4B9847064616
:10537000AB79DBB2022BDED028460A4B98470026D9
:1053800002E02846074B9847304606B0BDE8F0815A
:10539000C5FF400015704000CDFF40004170400047
:1053A000F171400029704000F8B506460D461746D9
:1053B000344BAA221A7011225A700222F021324C68
:1053C000A047012801D00020F8BD2C0AEDB22D4BDA
:1053D0001C705D709C70DD701C715D7100229A7193
:1053E0009022DA7167B182221A72264B0922C221F9
:1053F0003046254FB847012806D001280BD0F8BD0C
:105400000222204B1A72F0E71E4B0922C2213046BD
:105410001E4EB047F1E71B4B1B789C4201D0002089
:10542000F8BD184B9B789C4201D00020F8BD154B6D
:105430001B799C4201D00020F8BD124B5B789D4245
:1054400001D00020F8BD0F4BDB789D4201D0002039
:10545000F8BD0C4B5B799D420BD10A4B9B7953B93C
:10546000084BDB79902B08D1064B1B7A022B06D117
:10547000F8BD0020F8BD0020F8BD0020F8BD0020D8
:10548000BDE700BF34130020E9524000F151400055
:1054900010B50022054B1A7029B91121034B0122C6
:1054A000034CA04710BD1021F8E700BF34130020C3
:1054B000E952400070B504460022104B1A700D46A8
:1054C00039B129210D4B012220460D4EB04715B9A7
:1054D00070BD2821F6E7094DAA232B7011236B70AC
:1054E0002B460222F0212046B047FF232B702B468B
:1054F0000122C0212046B047EAE700BF3413002054
:10550000E952400010B539B90022044B1A7001224B
:105510003621034CA04710BD0322F6E734130020C8
:10552000E952400038B505460C4BAA221A701222E7
:105530005A700222F0210A4CA047012801D0002015
:1055400038BD064B0322BF212846064CA047012840
:1055500001D0002038BD014B987838BD34130020AD
:10556000E9524000F151400038B50D46094B0E227A
:105570008421094CA047012801D0002038BD054BEB
:10558000186859689A6828606960AA609B89AB812D
:105590000E2038BD34130020F151400010B50B46E9
:1055A0002C227021014CA04710BD00BFE9524000E1
:1055B0002DE9F04182B000238DF80730013905292B
:1055C0002BD8DFE801F00705030C0E10154D02E0A3
:1055D000154D00E0154D8046012000240FE0144DCC
:1055E000F9E7144DF7E7144DF5E70DF1070302460F
:1055F0004046124EB0473C44E4B20134E4B20128C4
:105600000CD123462F5D4FB1621CA95C012FECD950
:1056100002332B44781EC0B2E9E7002002B0BDE897
:10562000F08100BFBC3E410054404100EC404100CD
:10563000483E4100743F4100E43F4100E9524000D0
:1056400008B50621014B984708BD00BFB155400081
:1056500010B5274900238B72CB720B7340F2DC52DA
:105660008A806422CA800B8021F8083F0620214BE3
:1056700098470B20204B984780B90C201E4B984729
:1056800088B900221A4B5A801C4B984701211C4BA9
:10569000984701280CD0164B987A10BD19490B2059
:1056A000144B9847E9E718490C20124B9847E8E754
:1056B00001220F4B9A72114B98470521134B9847C3
:1056C000034650B10A4AD372002BE4D00B4B9847E3
:1056D0000F4B9847064B5880DDE7084CA047002148
:1056E000074B9847A0470321084B98470346E9E733
:1056F0009413002089794000BD794000CDFF40001F
:10570000F9574000981300209A130020295A4000AE
:10571000B9594000014B987A704700BF941300209C
:1057200008B5224B9B7A8BB9214A13781F49088808
:10573000204921F813000133DBB213700F2B02D97B
:1057400000221B4B1A7000231A4615E01A4B98478B
:105750001A4B9847154B1B89984203D80022134BCC
:105760001A80E1E7C01A114B1880DDE7114931F8C2
:1057700013100A440133DBB20F2BF7D912090B4B7C
:105780001B7B4BB109498B88C9885B1A9A420CD89C
:105790000022064B1A7308BD04498B88C9880B4444
:1057A0009A4202D30122014B1A7308BD94130020C0
:1057B000120D002074130020CDFF40004959400015
:1057C000014B187B704700BF94130020014B1888D1
:1057D000704700BF9413002008B5014B984708BDDF
:1057E000F95A400008B5024B9847024B984708BD4C
:1057F000CDFF4000015B400030B587B005460C4648
:1058000000238DF8073072228DF808208DF80B30B8
:1058100001228DF809208DF80C200DF10702049269
:1058200002228DF80A200593434B9847322202A9A1
:105830002846424B9847002C43D1012402238DF87F
:105840000A3080238DF80B3001238DF807309C42FD
:1058500044D08F238DF80B3003238DF80A30012CB0
:1058600043D09DF8073003F0F00343F005038DF8B3
:10587000073002238DF80A30012C3DD0AA238DF881
:105880000B3001238DF807309C423CD007238DF864
:105890000730F9238DF80B30012C3BD005238DF810
:1058A000073080238DF80B30012C3AD02846244B4A
:1058B0009847012C3CD00022224B1A70204607B09A
:1058C00030BDA8238DF80B3001238DF8073032222C
:1058D00002A92846194B98470446AFE7322202A98D
:1058E0002846164B98470446B3E7322202A92846B9
:1058F000124B98470446B4E7322202A928460F4BC0
:1059000098470446BAE7322202A928460B4B98472B
:105910000446BBE7322202A92846084B98470446B2
:10592000BCE7322202A92846044B98470446BDE74B
:105930000122044B1A70C1E715704000417040000D
:1059400029704000130D002030B587B004460023B5
:10595000059301AB049372238DF8083001238DF871
:1059600009309C238DF80B3002238DF80C30032373
:105970008DF80A300C4B9847322202A920460B4B77
:105980009847054620460A4B9847012D04D0002031
:10599000084B187007B030BD9DF804009DF8053025
:1059A00000EB032080B2F5E7157040004170400025
:1059B00029704000130D002030B587B00446002345
:1059C000059301AB049372238DF8083001238DF801
:1059D0000930C0238DF80B3002238DF80C300323DF
:1059E0008DF80A300C4B9847322202A920460B4B07
:1059F0009847054620460A4B9847012D04D00020C1
:105A0000084B187007B030BD9DF804009DF80530B4
:105A100000EB032080B2F5E71570400041704000B4
:105A200029704000130D0020F0B587B00646002312
:105A300005930DF10703049372238DF808300123B9
:105A40008DF80930D9228DF80B208DF80C30022307
:105A50008DF80A304901C9B241F010018DF80710E4
:105A6000214B9847322202A93046204B98470546E1
:105A7000D7238DF80B3021238DF8073001280BD068
:105A800030461B4B9847DC238DF80B3003238DF8F1
:105A90000A300024274608E0322202A93046134B80
:105AA00098470546ECE70134A4B2012D18D1BFB9DF
:105AB000092C15D819200F4B984730460A4B9847A8
:105AC000322202A93046094B984705463046084B1A
:105AD00098479DF8073013F0010FE4D00127E2E763
:105AE000384607B0F0BD00BF15704000417040005F
:105AF0002970400075EC400000487047A413002056
:105B0000A84BDB78032B00F24081A64B1B793F2B7F
:105B100000F23D81A34B5B79072B00F23A81A14B48
:105B20009B79082B00F237819E4B1B7A013BDBB23D
:105B3000022B00F232819B4B5B7A032B00F22F8108
:105B4000984B9B7A072B01D90020704710B586B07F
:105B500004460023059372238DF8083001238DF845
:105B600009300DF1070204928DF80C308E4B9847E6
:105B700080238DF80B3003238DF80A30322202A9DE
:105B800020468A4B9847012817D1864B1B78D3B102
:105B90009DF8073043F010038DF8073002238DF88D
:105BA0000A30322202A92046804B9847012811D0A2
:105BB00020467F4B9847002003E020467C4B9847C7
:105BC000002006B010BD9DF8073023F010038DF8BB
:105BD0000730E3E782238DF80B30724B5B788DF84A
:105BE0000730322202A92046704B9847012817D16E
:105BF0008D238DF80B3040238DF80730694B9B784F
:105C000013B148238DF80730322202A92046674B92
:105C10009847012809D02046654B98470020D0E7D7
:105C20002046634B98470020CBE78E238DF80B303E
:105C30005C4AD3789B01DBB2127902F03F02134336
:105C40008DF80730322202A92046584B9847012888
:105C500004D02046564B98470020B2E78F238DF89A
:105C60000B30504A53795B01DBB2927902F00F029C
:105C700013438DF80730322202A920464B4B984738
:105C8000012804D020464A4B9847002099E7A923D1
:105C90008DF80B30434BDB798DF80730322202A9A7
:105CA0002046424B984701280CD1AA238DF80B308F
:105CB0003C4B1B7A022B18D0032B1AD0012B06D099
:105CC00000207EE720463A4B9847002079E78DF880
:105CD0000730322202A92046344B984701280CD0C5
:105CE0002046334B984700206BE702238DF807309E
:105CF000EFE703238DF80730EBE7B3238DF80B3084
:105D0000284B5B7A03F003038DF80730322202A997
:105D10002046264B9847012804D02046244B98471C
:105D200000204EE7D9238DF80B3003238DF80A307D
:105D3000322202A920461D4B9847012804D0204654
:105D40001B4B984700203CE79DF8073003F0F80311
:105D500043F01003134A927A02F0070213438DF8BE
:105D6000073002238DF80A30322202A920460F4B59
:105D70009847012804D020460D4B9847002020E783
:105D800020460B4B984701201BE70020704700205E
:105D900070470020704700207047002070470020A7
:105DA000704700BFA41300201570400041704000F0
:105DB0002970400000FB01F0C0F3C71070470000DD
:105DC000F0B587B004460E46234B98470023049352
:105DD0008A238DF8043001238DF805308DF80830C2
:105DE0000DF11703039334278DF8077002238DF804
:105DF000063033788DF81730322201A92046174D2E
:105E0000A8478DF8077033788DF81730322201A932
:105E10002046A8478DF8077033788DF81730322266
:105E200001A92046A84735238DF8073073788DF8EF
:105E30001730322201A92046A84736238DF80730B3
:105E4000B3788DF81730322201A92046A8472046A2
:105E5000034B984707B0F0BD1570400041704000FB
:105E600029704000F0B587B00446002505958A23C7
:105E70008DF8083001268DF809608DF80C600DF161
:105E800007030493254B984755238DF807308DF869
:105E90000B5002238DF80A30322202A92046204DF1
:105EA000A84703238DF807308DF80B60322202A932
:105EB0002046A8478DF8076004238DF80B30322266
:105EC00002A92046A84707238DF8073030238DF814
:105ED0000B30322202A92046A8470F278DF8077001
:105EE00031238DF80B30322202A92046A8478DF8C5
:105EF000077032268DF80B60324602A92046A8476B
:105F00008DF8077033238DF80B30324602A92046F6
:105F1000A8472046034B984707B0F0BD15704000D6
:105F20004170400029704000F0B583B007460C4630
:105F3000802900D980240C4B1C700C4E21463078EF
:105F40000B4DA8478DF8040021467078A8478DF8BE
:105F500005002146B078A8478DF8060001A938460B
:105F6000044B984703B0F0BD01010020140D002040
:105F7000B55D4000C15D400010B5054B0C888A78C6
:105F80001C809A70034B1978034B984710BD00BFD3
:105F9000140D002001010020295F400010B586B0DB
:105FA00004468DF8081000230593E7238DF80B3085
:105FB0000DF10703049301238DF80C308DF809309F
:105FC00003238DF80A30322202A90A4B9847012890
:105FD00001D006B010BD9DF8073043F001038DF8E5
:105FE000073002238DF80A30322202A92046014BE5
:105FF0009847EEE74170400010B586B004468DF832
:106000000810002305930DF10703049301238DF875
:106010000C308DF8093006238DF80B3003238DF8F2
:106020000A30322202A9224B98479DF8073063F0CC
:106030007F038DF8073002238DF80A30012818D02D
:1060400000238DF807300C238DF80B30012816D073
:106050000D238DF80B30012817D00E238DF80B304F
:10606000012818D00F238DF80B30012819D006B065
:1060700010BD322202A920460D4B9847E0E732229C
:1060800002A920460A4B9847E2E7322202A920469D
:10609000074B9847E1E7322202A92046044B984774
:1060A000E0E7322202A92046014B9847DFE700BF14
:1060B0004170400010B586B004468DF808100023EA
:1060C0000593E7238DF80B300DF1070304930123AB
:1060D0008DF80C308DF8093003238DF80A30322208
:1060E00002A90A4B9847012801D006B010BD9DF8BF
:1060F000073023F001038DF8073002238DF80A30B2
:10610000322202A92046014B9847EEE74170400039
:1061100070B504462022214B1A630A20204B984771
:106120002046204B9847102120461F4EB047054679
:1061300012212046B0470646012D0ED0012E12D066
:10614000012D16D0012E1AD02046184B9847012D4C
:106150001BD0012E1DD0284670BD10212046144BA7
:1061600098470546EAE712212046114B9847064614
:10617000E6E7102120460F4B98470546E2E712213B
:1061800020460C4B98470646DEE701220A4B1A7060
:10619000DFE70122094B1A70DDE700BF00100E4057
:1061A00075EC4000157040009D5F40002970400074
:1061B000F95F4000B5604000170D0020180D002069
:1061C00010B1034B18787047024B1878704700BF26
:1061D000180D0020170D002030B587B004460D467D
:1061E00000220592A8238DF8083001238DF809308C
:1061F0008DF80B200DF1070204928DF80C3002236C
:106200008DF80A30124B9847012D0ED0022D15D073
:1062100000238DF80730322202A920460D4B984703
:1062200020460D4B984707B030BD03238DF807304B
:10623000322202A92046074B9847F1E702238DF846
:106240000730322202A92046024B9847E8E700BFF8
:1062500015704000417040002970400030B587B093
:1062600072238DF8003001238DF8013000238DF862
:1062700002308DF8033008228DF8042004AA02921F
:1062800003938DF81000C0F307238DF81130C0F38D
:1062900007438DF81230000E8DF813008DF814109E
:1062A000C1F307238DF81530C1F307438DF816307D
:1062B000090E8DF81710084CA047084B9847A047C7
:1062C00032226946064B98470546A047054B98473A
:1062D000284607B030BD00BFC5FF40001570400024
:1062E000417040002970400030B587B00D467223E0
:1062F0008DF8043001238DF8053000238DF8063029
:106300008DF8073004228DF8082005AA0392049323
:106310008DF81400C0F307238DF81530C0F3074340
:106320008DF81630000E8DF81700184CA047184B4A
:106330009847A047322201A9164B984704460128E6
:1063400008D0124B9847144B9847012C0DD020468B
:1063500007B030BD01238DF806300C4B9847322230
:1063600001A90C4B98470446EBE79DF814309DF8C3
:10637000152003EB02239DF8162003EB02439DF842
:10638000172003EB02632B60E1E700BFC5FF40006D
:106390001570400041704000297040002DE9F04E1A
:1063A00082B08246894693461BB11E4600250127CE
:1063B0002FE00127012F40D0012F49D0012F4DD0D0
:1063C000012F51D04FF4000301932F4B98470446FF
:1063D000012F4FD1019B13F4000F4BD00A99204697
:1063E0002A4B984700284DD101A92948294B9847A5
:1063F0000746EDE7EA18B25C4FEAC30E02FA0EF266
:1064000011440133DBB2A342F4D3012F0DD0254454
:10641000EDB228464D45CDD2A9EB0504042C28BF8A
:106420000424E4B200231946EDE700F1201000F542
:106430008070194B98470746E9E74FEA0A4101F493
:10644000FE0101F500011248134B98470746B3E7D8
:1064500049461248104B98470746AFE7594610483F
:106460000D4B98470746ABE7F2210E480A4B984779
:106470000746A7E71FB9052002B0BDE8F08E9DF8DA
:106480000700F9E70620F7E77976400091764000AB
:1064900010012000E96240005D6240001801200008
:1064A00014012000FC00200010B584B00A4B93E8D2
:1064B000030002908DF80C103223009302AB0022EF
:1064C00005210120054CA047034610B90121044ACB
:1064D0001170184604B010BD844141009D63400016
:1064E000190D002070B5074D4FF480466E630A20E9
:1064F000054CA0472E6340F21310A047034B98476A
:1065000070BD00BF000E0E4075EC4000A964400055
:1065100030B583B00D463223009300230246042198
:106520003120074CA047044610B1204603B030BDCF
:1065300029460448044B98470128F6D00524F4E77F
:106540009D63400020012000E962400010B584B046
:106550008DF80C100B0A8DF80D300B0C8DF80E30E9
:10656000090E8DF80F103223009303AB024604216D
:106570002120024CA04704B010BD00BF9D63400025
:1065800008B5044B1B780BB1002008BD024B98479F
:1065900008BD00BF190D0020A96440002DE9F0439B
:1065A00083B059B1012904D00124204603B0BDE8CD
:1065B000F08340F65D0740F6050503E040F2DD7725
:1065C00040F2857580464FF000094C4601E0002CF2
:1065D000EBD1BD42E9D225F00306002CF7D101A989
:1065E0003046164B984704460028F0D1019B8DF8A1
:1065F0000030C3F307228DF80120C3F307428DF862
:1066000002201B0E8DF80330E9B2F3B2C91AC9B2E9
:10661000C1F10403BE1B9E4228BF1E46042E28BFA4
:106620000426F6B23246694408EB0900044B984749
:1066300035444E445FFA86F9C9E700BF1165400052
:10664000A114410028B1012801D000207047094859
:1066500000E0094800B583B001A9084B984728B964
:10666000019B13F4006F02D0012000E0002003B072
:106670005DF804FB4000350040003100116540002A
:1066800010B52DED028B82B0044601A93548364B7A
:1066900098470346F8B14BB3002B32D0002B3BD0C8
:1066A000DFED328A002B49D09FED308A73B9DDEDE2
:1066B000017AB8EE677AC8EE077A9FED2D7A67EE19
:1066C000877AFCEEE77A17EE902A6281184602B0CC
:1066D000BDEC028B10BD02A951F8043D23801B0CB8
:1066E00063802448204B98470346D4E702A951F819
:1066F000043DA3801B0CE3801F481B4B98470346B7
:10670000CAE702A951F8043D03F01F0323721B4896
:10671000154B98470346C1E702A951F8043DC3F35E
:10672000094308EE903AF8EE688A9FED158A68EE04
:10673000888A14480C4B98470346B3E702A951F8DE
:10674000043DDBB208EE103AB8EE488A28EE888A9B
:10675000DFED077A28EE278A0B48034B984703465C
:10676000A4E700BF300822001165400000000000CF
:106770000000C84238082200540822000800200007
:1067800000401C46040822001408220000B583B013
:1067900001A941F23070094B9847034618B11846D9
:1067A00003B05DF804FB019921F00601019141F26B
:1067B0003070034B98470346F1E700BF1165400076
:1067C0004D65400030B583B015460C4AA2FB01234D
:1067D0001B090F330093002302461120084CA047E9
:1067E000044610B1204603B030BD29460548064B8B
:1067F00098470128F6D00524F4E700BF1F85EB5128
:106800009D63400020012000E962400010B582B085
:1068100096230093134602462020024CA04702B064
:1068200010BD00BF9D634000072801D901207047BB
:1068300010B584B08DF80C0030238DF80D3041F286
:106840008833009303AB002202211420014CA0479F
:1068500004B010BD9D63400010F0800F11D110B541
:1068600084B08DF80C0010238DF80D3041F2883380
:10687000009303AB002202211420034CA04704B074
:1068800010BD0120704700BF9D634000F0B583B08C
:10689000032832D8DFE800F00209050747F6F07652
:1068A00004E0184E02E0184E00E0184E00240127C4
:1068B0003D4604E09CB10F2C11D00134E4B20F2C02
:1068C00013D801AA0121A019114B9847B8B9002D7E
:1068D000F0D09DF80430FF2BECD00025EAE79DF8BE
:1068E0000430002BE9D10027E7E717B11DB10020E4
:1068F00006E0002004E0012002E0002000E000208B
:1069000003B0F0BDF0FF0100F0FF0300F07F0200D4
:10691000C567400070B582B006460020114B98470D
:1069200020B14FF4BE65002423460BE001200D4B3F
:10693000984718B90323184602B070BD0A4DF2E714
:106940000134E4B20E2CF6D8002BF9D101AA0121B2
:106950002819064B984703460028F1D19DF80420DA
:106960003255EDE78D684000F0050200C567400034
:1069700030B587B01D201C4B98471C4C236C23F46A
:106980000013236468461A4B984769462046194B02
:106990009847636823F47F436360636843F47F43ED
:1069A0006360042323610823236101232361626858
:1069B00022F08F026260104A032120460F4DA84743
:1069C000002120460E4B9847636813F0800F01D1D9
:1069D000082222600B4B4FF000521A60702283F89D
:1069E0001D2307B030BD00BF35D7400000800340F5
:1069F00095494000294A4000296A4000794A4000F0
:106A0000BD49400000E100E00222014B1A607047DE
:106A100000800340024B1880024B1980704700BF72
:106A2000020100200401002010B5064C206D80B248
:106A3000054B9847A06DE16D89B280B2034B984732
:106A400010BD00BF008003401D7B4000156A400060
:106A5000014B1888704700BF02010020014B1888C5
:106A6000704700BF040100200D4B1B8840F689626F
:106A7000934205D90B4A12883E2A01D80320704759
:106A8000084A128840F689618A4203D93E2B01D810
:106A900004207047934201D80220704701207047BC
:106AA000020100200401002008B50120034B984793
:106AB000034B186000B1012008BD00BFEDE24000AB
:106AC000B013002008B54FF0FF31024B1868024B9D
:106AD000984708BDB0130020A9E4400010B500237A
:106AE0001A46194602480068024CA04710BD00BF74
:106AF000B0130020B5E14000154B98421BD003F5C0
:106B0000A033984219D003F58043984217D0A3F5DB
:106B10004043984215D003F58043984213D0A3F523
:106B2000A033984211D003F56033984201D032204F
:106B300070471620704708207047092070470E20C4
:106B4000704713207047142070471520704700BF0E
:106B500000C000404900B0FBF1F00338002302E020
:106B600040080133DBB2FF28FAD8020202F47F4268
:106B700052FA80F01B0403F4E0231844704700002D
:106B80002DE9F843D0F80090037ADBB2012B00F036
:106B9000E68009F5C0650B7913B91846BDE8F8839E
:106BA00017460E460446012303720023C371E160B9
:106BB0006E4B98478046B378022B08D07378012B30
:106BC00018D033781B0403F4FE036B6050E0737835
:106BD000012B09D033781B0403F4FE0303F5807303
:106BE0006B60F378EB6043E033785B081B0403F5DC
:106BF0008073F5E733785B081B04E6E70323A37192
:106C000000232372237A002B00F0AB802B6A13F44D
:106C1000807F53D113F4007F78D113F0400F7AD1E5
:106C200013F0800F7CD113F0040F4BD1394640464E
:106C30004F4B98470028E9D00723A3710023237204
:106C40004C4BC9F800363DE00423A37100232372A6
:106C5000D8E70523A37100232372D3E70623A3718A
:106C600000232372CEE739464046414B9847E8B9A6
:106C70003379E2799B1A002BC4DD2B6A13F4807FF1
:106C8000BCD113F4007FDFD113F0400FE1D113F03A
:106C9000800FE3D113F0040FE5D0B168E379DBB2E4
:106CA0005A1CD2B2E271CB5C6B63DCE70723A371A1
:106CB000002323722F4BC9F80036A3E70323A371E7
:106CC00000232372237A002B4DD00223C9F800360B
:106CD0002B6A13F0010F28D113F4807F2BD113F40A
:106CE000007F2DD113F0400F2FD113F0800F31D141
:106CF000394640461E4B98470028E9D00723A37128
:106D0000002323721B4AC9F8002646E70423A37117
:106D100000232372D6E70523A37100232372D1E752
:106D20000623A37100232372CCE7002323720223DE
:106D3000A371012331E70323A371002323722CE7FE
:106D40000423A3710023237227E70523A3710023E3
:106D5000237222E70623A371002323721DE7002379
:106D60001BE7002319E7002317E700BF79764000EF
:106D700091764000028000052DE9F84FD0F800B070
:106D8000037ADBB2012B00F0CE800BF5C0670B79E4
:106D900013B91846BDE8F88F90460E460546012304
:106DA00003720023C371E960614B98478146B37851
:106DB000032B14D07378012B24D033781B0403F4F5
:106DC000FE0303F580537B6096F804A0BAF1010F2F
:106DD0001ED00123CBF800364FF0000A64E0737830
:106DE000012B09D033781B0403F4FE0303F5885309
:106DF0007B60F378FB60E7E733785B081B0403F5FF
:106E00008853F5E733785B081B0403F58053DAE712
:106E10000323CBF8003647E00323AB7100232B722A
:106E20002B7A002B00F081803B6A13F0010F60D1B8
:106E300013F4807F63D113F4007F65D113F0400F0A
:106E400067D113F0800F69D141464846394B9847C6
:106E50000028E9D00723AB7100232B72364ACBF808
:106E6000002696E70423AB7100232B72D8E7052395
:106E7000AB7100232B72D3E70623AB7100232B7277
:106E8000CEE70723AB7100232B722B4BCBF80036D8
:106E9000C6E714F0020F07D0B168EB79DBB25A1CD9
:106EA000D2B2EA713A6BCA54EB79DBB232799342CF
:106EB000B6D23C6A14F4807FAED114F4007FD1D1F5
:106EC00014F0400FD3D114F0800FD5D1414648467D
:106ED000184B98470028D4D1BAF1000FD9D1337993
:106EE000EA799B1A012BD4D102233B604FF0010AAF
:106EF000CFE700232B720223AB71012349E7032361
:106F0000AB7100232B7244E70423AB7100232B7277
:106F10003FE70523AB7100232B723AE70623AB71E1
:106F200000232B7235E7002333E7002331E700BF4E
:106F30007976400091764000028000052DE9F0410D
:106F400006468846046820461B4B9847312801D9DD
:106F5000BDE8F0810546194B98470323236024239D
:106F6000C4F8003641461648164B9847C4F8100638
:106F7000002333720123B3716BB2002B07DB5A0974
:106F800005F01F00012181400F4840F82210002B1E
:106F90000BDB03F1604303F56143202283F80023F8
:106FA00001200A4B98473061D2E705F00F05084BE6
:106FB00020225A55F4E700BFF96A400035D7400057
:106FC0000000DC05556B400000E100E0EDE2400010
:106FD00014ED00E008B500680B4B9847312811D834
:106FE00043B2002B0CDB5B0900F01F0101228A4039
:106FF0002033064941F82320BFF34F8FBFF36F8F33
:10700000034B984708BD00BFF96A400000E100E06B
:1070100089D7400008B54FF0FF310069014B984710
:10702000C0B208BDA9E4400010B500231A461946B5
:107030000069024CA047C0B210BD00BFB5E14000DE
:1070400008B5837963B18B78032B0BD8DFE803F0A5
:1070500002050205044B984708BD044B984708BD3C
:10706000002008BD002008BD816B4000796D400004
:1070700080797047F8B50646036803F5C064256A51
:10708000C76815F0040F0BD0E26A12F0040F07D0A6
:10709000BA78002A4DD0022A4BD0BA78032A5ED0A3
:1070A00015F0020F08D0E26A12F0020F04D0BA788D
:1070B000012A73D0032A71D015F4807F0DD0E36AC2
:1070C00013F4807F09D040F20733A36200233372A8
:1070D0000323B371FB6803B1984715F4007F0DD00B
:1070E000E36A13F4007F09D040F20733A362002360
:1070F00033720423B371FB6803B1984715F0010F95
:1071000016D0E36A13F0010F12D0BB780BB1022B3B
:1071100009D140F20533A362002333720223B37115
:10712000FB6803B19847BB78012B54D0032B52D096
:10713000F8BDF279D2B239798A4208D2B868F279C8
:10714000D2B2511CC9B2F171825C6263A5E702221E
:10715000C3F80026012262620422A2629DE77A78C7
:10716000012A11D03A78120402F4FE0202F580528C
:1071700062603A79012A0DD00122C3F80026042268
:10718000A262022262628BE73A785208120402F588
:107190008052EDE70322C3F80026F0E7B868F279E1
:1071A000D2B2511CC9B2F171216B8154F179C9B2CB
:1071B0003A79013A91420AD0F379DBB23A799342B3
:1071C0007FF47AAF012363620223A36274E7022291
:1071D000C3F80026F0E740F20333A36200233372C2
:1071E0000223B371FB68002BA2D09847A0E70000F0
:1071F00070B4056805F5C0660379202B0BD9A3F19F
:107200002001CBB21A4C01219940216021652161F6
:107210002163002211E0174CF5E701339BB2B3F56F
:107220002F7FFAD36163002301E001339BB2B3F5F2
:107230002F7FFAD321630132D2B2092A01D8002369
:10724000EDE76161616032698023C5F80036002393
:1072500001E001339BB2B3F52F7FFAD332612423CF
:10726000C5F80036002303720123837170BC704798
:1072700000100E40000E0E4030B591B000238DF886
:1072800035308DF836308DF837308DF839308DF84F
:107290003A30ADF83E300F238DF834300223ADF88C
:1072A0003C3001248DF838400DAA0B4907A80B4D3E
:1072B000A8470DAA0A4901A8A8471023079A1360F6
:1072C000019A1360074B1C70074B1C7045F6FF7248
:1072D000064B1A8011B030BD00C002401DD24000E4
:1072E000000003401C0D0020941500205E160020B5
:1072F00042B110B420B119B1034B586099605A8063
:107300005DF8044B704700BF1C0D0020154B1B7827
:107310003BB3144B5B8823B3124A52680AB311493A
:107320008968F1B1F0B583B0009201930E4D6A46C1
:10733000694628460D4FB8474FF480362E62094BF8
:107340009B6800930A4C6A4669462046B847266205
:1073500001212846074DA84701212046A84703B030
:10736000F0BD70471C0D002000C1024059D1400003
:107370000001034071D140000223034A136202F569
:1073800080421362704700BF00C1024010B58CB04C
:107390000A4B9847069A136823F010031360009A6B
:1073A000136823F0100313600D20054CA047122032
:1073B000A0470022034B1A700CB010BD7973400037
:1073C00089D740001C0D0020064B1B783BB1054BB4
:1073D0005888054BD3F80431C01A80B2704700209A
:1073E000704700BF1C0D002000C00240094AD36D49
:1073F00023F4FF4323F07F03C0F30E000343D36560
:1074000002F58042D36D23F4FF4323F07F0318433A
:10741000D065704700C00240014B1880704700BF24
:107420005E160020014B1870704700BF94150020B5
:10743000004870476016002000487047B4130020D1
:10744000704770472DE9F8434F4B984705464F4B1F
:10745000984704467FE0A0EB070E1FFA8EFE0EF160
:10746000F00E1FFA8EFE85E03121002308E02F2167
:10747000FBE747480078C0B2012831D001339BB206
:10748000994259D9DA1992B2EF2A01D9F03A92B257
:107490003F4800780028ECD13E48B0F9000035F9AB
:1074A000126006FB00F6F6134FEA8308DFF8ECC023
:1074B0000CF8236008F10109C6F307260CF80960EF
:1074C00034F9122000FB02F2D21308F102000CF88A
:1074D000002008F10308C2F307220CF80820CDE7CA
:1074E00035F9120034F91220024402EBD272521024
:1074F00012F5004F05DBB2F5004F03DB47F6FF72D4
:1075000000E0254A2348B0F9000012B202FB00F265
:10751000D21398005FFA82FC204E06F823C000F1D7
:107520000108C2F3072206F8082000F1020806F855
:1075300008C003303254A1E7194BA3F800E07744A8
:10754000BFB2184B1F80EF2F01D9F03F1F80890079
:107550001248154B98474FF0FF310120134B9847C5
:10756000134B98470F4B1F88B842FFF474AFC01BF2
:107570001FFA80FEBEF1300F3FF676AFBEF12F0F3F
:107580007FF675AF302170E73174400039744000E8
:10759000941500205E1600200080FFFF9815002043
:1075A0005C160020280D00202D45400081F1400090
:1075B000C9734000F8B5084C4FF4804666630A2052
:1075C000064DA847402767630A20A84727630A207B
:1075D000A8472663F8BD00BF000E0E4075EC4000C2
:1075E000F8B578B9114D4FF480736B630220104CDD
:1075F000A0474FF080736B630420A04701220D4B1E
:107600005A63F8BD094E4FF480737363094F022526
:107610003D632846064CA04701233B630420A04756
:107620004FF0807333632846A047F8BD000E0E402C
:1076300075EC400000100E4010B5084C4FF480432C
:1076400063630020064B98470220064B98470222AE
:10765000054B5A634023636310BD00BF000E0E400C
:10766000E175400075EC400000100E400322014B14
:107670001A60704730140E40044B986801E0034BC9
:107680009868024B9B689842F9D1704730140E40BD
:1076900010B584B001900C46064B98470390039BAD
:1076A000019A9B1AA34202D2002004B010BD01200F
:1076B000FBE700BF7976400030B585B01E4B1B68F4
:1076C000002B31D01D4B98474FF0FF311A4B1868F3
:1076D0001B4B9847EFF31083B3FA83F35B090393D3
:1076E00072B6BFF35F8F0022164B1A70039D802382
:1076F0000093154B152214211448154CA04704463D
:107700002DB101220F4B1A70BFF35F8F62B60023B9
:107710001A461946084800680E4DA8470E4B984770
:1077200044B1002005B030BD01200C4B9847024BFE
:107730001860C7E70120F5E72C0D0020C56A40005E
:10774000A9E440002F03002040180020000A0E404A
:1077500011000020B5E14000DD6A4000EDE240008C
:1077600010B5074B9847002213210648064B98474F
:107770000446064B9847B4FA84F0400910BD00BF98
:10778000C56A4000000A0E4095D44000DD6A400002
:1077900038B5114B9847EFF3108404B972B6002343
:1077A00008E09A0002F580020C4951F8231011609C
:1077B00001339BB27F2BF4D9002212210848094BD8
:1077C0009847C5B204B962B6074B98470DB100207F
:1077D00038BD012038BD00BFC56A400040180020F8
:1077E000000A0E4095D44000DD6A400010B4002429
:1077F0000EE0400080F00700C0B20133DBB2072B7F
:1078000005D810F0800FF4D14000C0B2F5E7013484
:10781000944204D211F8013B58400023EFE75DF891
:10782000044B704770B50646002501E02C44A5B214
:10783000B5F5007F15D20E4BE918EA5CFF2A14D08B
:107840006B1C0B481B5C0333DCB2B242EED1621EF0
:10785000FF20084B98472B19074A9B5C9842E5D1BB
:1078600001E04FF6FF75284670BD4FF6FF75FAE749
:1078700040180020ED7740003F18002008B5094B64
:107880001B781BB1022B01D0074808BD074B984756
:10789000012804D10122034B1A70034808BD0020BF
:1078A00008BD00BF300D002040180020B976400010
:1078B00008B5094B1B781BB1022B01D0074808BD46
:1078C000074B9847012804D10122034B1A70034843
:1078D00008BD002008BD00BF300D0020401800206A
:1078E000B9764000A8B108B50346B1F5007F12D2C1
:1078F0008818B0F5007F01D9002008BD0846194658
:10790000064B1844064B98470222064B1A7001207A
:1079100008BD00207047002008BD00BF40180020AF
:10792000A1144100300D002008B5064B1B78022B36
:1079300001D0002008BD044B98470128FAD1034B21
:10794000984708BD300D00206177400091774000D6
:1079500090B110B504460268094B9A4201D000204C
:1079600010BD9A220146FF20064B984794F89A30A2
:10797000984203D0002010BD00207047012010BDA8
:107980005FE1AD5AED77400010B50C46084B9847C3
:10799000B0F5007F01D3002010BD811C054B5A1C9F
:1079A000125C19442046044B9847012010BD00BFCB
:1079B0002578400040180020A114410008B5044B70
:1079C0009847B0F5007F01D2012008BD002008BD16
:1079D0002578400008B5054B9847B0F5007F02D2E6
:1079E000034BC05C08BD002008BD00BF25784000E7
:1079F00041180020FF292FD02DE9F843D61CF6B2FC
:107A00008419B4F5007F03D94FF6FF70BDE8F88301
:107A100017460C4605460221114A1170DFF84C80CA
:107A200000EB080900F80840421C02F808700844FE
:107A30003A46194640440B4B98477C190234721E53
:107A40004946FF20084B984708F80400E81980B21F
:107A5000033080B2BDE8F8834FF6FF70704700BF77
:107A6000300D0020A1144100ED77400040180020A7
:107A700010B5A8B0224B98470446224B984708B946
:107A800028B010BD9B22214601A81F4B98474FF4F8
:107A90000072FF211D481E4B984702AB10220121A6
:107AA00000201C4CA0474FF6FF73984203D026AB32
:107AB00003220221A0474FF6FF73984205D00DF133
:107AC0009B0301220321134CA0474FF6FF739842FA
:107AD00004D027AB012204210E4CA0474FF6FF73C0
:107AE000984205D00DF19D0301220521094CA047C4
:107AF0004FF6FF739842C3D0074B9847C0E700BFCB
:107B00007D78400051794000A114410040180020C8
:107B10009D164100F579400029794000044B1880FA
:107B2000044A1378591C1170034A22F81300704755
:107B3000441C0020310D0020441A002008B5194BC8
:107B40001B8807EE903AF8EE677A9FED177A67EE9A
:107B5000877A164BC3ED007AF7EE006A76EEE76A95
:107B600087EEA67ADFED126A67EE267A114BC3ED37
:107B7000007A86EEA77A17EE100A0F4B9847DFEDD2
:107B80000F7A07EE100A27EE277ADFED0D7A77EEEF
:107B9000C77ADFED0C6A86EEA77A0B4B83ED007A8D
:107BA00008BD00BF441C002001088039401A002095
:107BB00000401C464C1C0020350041003313954307
:107BC00000F05745C47D7B49481C0020BFF35F8F00
:107BD000024B1868BFF35F8F704700BF481C00203E
:107BE00068B90F4A1368B3F1FF3F0AD00320B3F11D
:107BF000333F0ED013B9536803B902207047094AC6
:107C0000F0E75168B1F1FF3F01D00320EFE700201A
:107C1000EDE75168B1F1333FECD10120EAE700BF55
:107C200000C0470000E0470018B101280FD0022033
:107C300070470B4841F6F87383B130B4C518C45887
:107C40008C4206D0083B002BF8D1012004E0054807
:107C5000F0E76B681360002030BC7047012070476C
:107C600000C0470000E0470070B505460020124CF8
:107C7000A04706460120A0471DB1012D12D00220C9
:107C800070BD022803D0022E07D0022070BD012E45
:107C900001D0012070BD002070BD012801D000205E
:107CA00070BD70BD022E05D0022801D0022070BD2B
:107CB000012070BD002070BDE17B4000F8B5044696
:107CC0000F461646450A094B984704F4FE7000F526
:107CD00080031F605E602A4601210548054B9847D6
:107CE0000446054B98472046F8BD00BFC56A4000D2
:107CF000000A0E4095D44000DD6A4000012909D0F9
:107D000002290CD1002108B538B906480A46064BAD
:107D1000984708BD4FF03331F5E70448F6E70120F6
:107D2000704700BF00C04700BD7C400000E0470036
:107D300038B518B101280DD0022038BD0A4C0823EF
:107D4000B3F5005F0ED2E018E558B5F1FF3F03D060
:107D50000833F5E7054CF2E7054B984708B10220D8
:107D600038BD38BD012038BD00C0470000E04700E5
:107D7000BD7C400010B568B140F2F234074B984723
:107D8000224607210648074B98470446064B98476A
:107D9000204610BD40F2E234F0E700BFC56A400063
:107DA000000A0E4095D44000DD6A400070B50546DB
:107DB0000E460B4C4FF0FF3120680A4B98470120CC
:107DC000094B984732462946084B984705460023F9
:107DD0001A4619462068064CA047284670BD00BFC9
:107DE000501C0020A9E44000697C4000297C400030
:107DF000B5E14000F8B505460E464FF0FF31144B93
:107E00001868144B98470020134B98470746324692
:107E10002946124B98470446012808D000231A46E9
:107E200019460B4800680E4DA8472046F8BDB7FA22
:107E300087F46409214638460A4B984708B1022462
:107E4000ECE7324629462046044B98470446E5E7CE
:107E5000501C0020A9E44000697C4000317D4000B6
:107E6000B5E14000ED7E400030B583B000230193C2
:107E7000044660B9164D17490023B3F5006F24D2AC
:107E800051F82320B2F1FF3F04D10133F5E7124D41
:107E90001249F1E72046124B9847044610B120469C
:107EA00003B030BD01A928460E4B984740B901994F
:107EB000013128460C4B98470028F0D00124EEE70A
:107EC00001212846084B9847F6E70024E7E700BF62
:107ED0000120FFFF00C047000220FFFF00E0470035
:107EE000757D4000AD7D4000F57D400070B582B0ED
:107EF00005460E460846284B9847012806D0012122
:107F00003046264B98470446002841D1002400E023
:107F10000134234B1B689C4215D201AA214B53F814
:107F200024102846204B9847022830D00028EFD153
:107F3000019A1C4B53F8241030461C4B98470028DC
:107F4000E6D0012424E02846194B98470446F8B9A6
:107F500002213046114B98470446C8B985B9154DE2
:107F600002A9002341F8083D2846134B984748B919
:107F7000009901312846114B984748B1012407E088
:107F80000F4DEDE7012128460C4B9847F5E70124FA
:107F9000204602B070BD00BFE17B4000FD7C400088
:107FA0002001002008010020297C4000317D400094
:107FB000757D40000120FFFFAD7D4000F57D400054
:107FC0000220FFFF10B500200E4B9847044608B171
:107FD000204610BD01200B4B984704460028F7D1DE
:107FE0000221094B984704460028F1D10121074896
:107FF000074B984708B10124EAE701210548044BE3
:108000009847E5E7757D4000FD7C40000120FFFFBB
:10801000F57D40000220FFFF38B501202D4B984729
:108020002D4B1860002852D000202C4DA847044644
:108030000120A847012C20D034B1022C35D0284B88
:1080400098470346184638BD012806D0022810D1AB
:108050000020244B98470346F4E70020214B984723
:1080600003460028EED1022101201F4B984703460A
:10807000E8E71B4B98470346E4E738B1022810D1E4
:1080800000210120194B98470346DBE70120154BDF
:10809000984703460028D5D10221134B9847034641
:1080A000D0E70F4B98470346CCE728B1022808D108
:1080B0000B4B98470346C5E701200A4B98470346F8
:1080C000C0E701210020094B98470346BAE7012386
:1080D000B8E700BFEDE24000501C0020E17B40000B
:1080E000C57F4000697E4000FD7C4000ED7E400081
:1080F00008B50020094B984708B1012008BD20228F
:10810000074B5A630A20074B9847074B9847074B82
:108110009847012801D0002008BD08BDC16140007A
:1081200000100E4075EC4000CDFF40001161400092
:1081300030B587B0174B984704468A238DF808302E
:108140000025059501238DF809308DF80C300DF1CF
:1081500007030493104B98478DF80B5003238DF8B9
:108160000A30322202A920460C4B984720460C4B7D
:108170009847022806D0002520460A4B98472846F3
:1081800007B030BD9DF80730092B01D00025F3E77B
:108190000125F1E7CDFF400015704000417040001F
:1081A000717040002970400030B587B01A4B984775
:1081B000044600220592A8238DF8083001238DF88B
:1081C00009308DF80B2001AA049202228DF80C20B0
:1081D0008DF80A30114B9847322202A92046104BE5
:1081E000984720460F4B9847022806D00025204686
:1081F0000D4B9847284607B030BD9DF8043033B981
:108200009DF8053013F0F80F03D00025EFE70025A7
:10821000EDE70125EBE700BFC5FF4000157040000A
:1082200041704000717040002970400008B5034B58
:10823000984708B1002008BD012008BD81654000B5
:1082400030B587B0184B9847044600230593722336
:108250008DF8083001238DF8093092228DF80B201B
:108260000DF1070204928DF80C3003238DF80A30CB
:108270000E4B9847322202A920460D4B98472046C4
:108280000C4B9847022806D0002520460A4B9847F9
:10829000284607B030BD9DF80730442B01D000259B
:1082A000F3E70125F1E700BFCDFF40001570400066
:1082B00041704000717040002970400070B586B078
:1082C000002832D11C4B9847044600250595982379
:1082D0008DF8083001268DF809608DF80A500223C8
:1082E0008DF80C3001AB04938DF80B502046134BE6
:1082F000984736238DF804308DF80550322202A9B4
:1083000020460F4DA8478DF80A60322202A9204668
:10831000A84720460B4B984702280AD00025204644
:10832000094B9847284606B070BD084B984704464D
:10833000CBE73546F3E700BFC5FF400015704000AE
:10834000417040007170400029704000CDFF400036
:1083500038B50020064CA04705460120A047012D56
:1083600001D0002038BD0128FCD0002038BD00BF5E
:10837000BD8240002DE9F0473D4BD3F858801920CD
:108380003C4B98474FF496703B4B9847002409E0CC
:108390003A4B98473A4B23F814000320364B984742
:1083A0000134E4B21F2CF3D9364B9847824600269D
:1083B0003746354634463FE0314931F813100A4418
:1083C0000133DBB21F2BF7D94FEA5219B9F10A0F6B
:1083D00017D92A4B9847631CDBB2294A22F81400AC
:1083E0001F2B1DD81C46A9F1FA0398421AD309F194
:1083F000FA02904225D80135EDB2202D13D901267D
:1084000011E0B8F1000F05D0194BC3F858800020D7
:10841000BDE8F0870020174B98470020BDE8F087A3
:108420000024E0E700250320134B98474FF47A61BE
:108430005046154B984707462FB926B900231A46D0
:10844000C0E70025EFE7B8F1000F07D0084BC3F8ED
:10845000588057B936B10120BDE8F0870020054BA0
:108460009847F6E70020BDE8F0870020BDE8F087D8
:1084700000000140F150400075EC40003D514000CB
:10848000541C0020797640009176400000487047E7
:108490008C414100072070472DE9F84305460E4600
:1084A00017460A469C211E4B98470446451B40B17F
:1084B000731B052B05D94378552B07D010237B70F0
:1084C00001E000237B702046BDE8F88390F802802D
:1084D000C37888EA0303FF2B02D011237B70F2E7F5
:1084E00090F80490437909EB03291FFA89F9B9F14F
:1084F0003A0F06D84D440635AE4205D200237B70B4
:10850000E1E712237B70DEE74A46811D381D054BEB
:108510009847A7F8029087F8008001237B70D2E784
:10852000A1134100A114410010B553889C1D8C4239
:1085300019D83A2B01D9002010BD11469C23037095
:1085400055234370137883701378DB43C37093789B
:10855000037153881B0A4371528804310630034B60
:108560009847012010BD002010BD00BFA11441009C
:1085700070B582B004460378253B332B00F2198294
:10858000DFE813F045001702170217021702340044
:108590001702170217021702170217021702170213
:1085A0001702170217021702170217021702170203
:1085B0001702170217021702170217023E011702CD
:1085C0001702FA0017021702170217021702BA0160
:1085D00013015C0017021702170217021702170295
:1085E000170265017900CB00A600E3009C4C2A230A
:1085F00023709C4DA84760809B4B98470646A84730
:1086000002463146201D994B984702B070BD0120AB
:10861000974B984780B2924B588010B945221A70F8
:10862000F3E794490120944B984718B125228C4BCD
:108630001A70EAE745228A4B1A70E6E74388032B53
:1086400005D0874B00225A8045221A70DDE7037956
:108650008DF8043043798DF8053083798DF8063034
:10866000864B984701A9864B98477D4B00225A803C
:1086700024221A70C9E74388012B05D0784B0022C9
:108680005A8045221A70C0E703790F2B05D9744B25
:1086900000225A8045221A70B7E77A4B9847704AF1
:1086A0005523137020235380237900EB4310066871
:1086B00045688468C16856609560D4601161066938
:1086C00045698469C16956619561D46111629CE70D
:1086D0004388212B05D0624B00225A8045221A7014
:1086E00093E701790F2905D95D4B00225A80452275
:1086F0001A708AE7202249010530634B9847012808
:1087000005D0574B00225A8045221A707DE7544B02
:1087100000225A8024221A7077E743882BB1504BED
:1087200000225A8045221A706FE7584B984701285B
:1087300005D04B4B00225A8045221A7065E7484B02
:1087400000225A8024221A705FE743882BB1444BE1
:1087500000225A8045221A7057E74D4B984728B996
:108760003F4B00225A8024221A704EE73C4B0022D5
:108770005A8045221A7048E74388012B05D0384BB0
:1087800000225A8045221A703FE70079414B9847F2
:1087900028B9334B00225A8024221A7035E7304B17
:1087A00000225A8045221A702FE74388082B05D0F3
:1087B0002B4B00225A8045221A7026E70379427912
:1087C00003EB0223827903EB0243C079217A627AB8
:1087D00001EB0221A27A01EB0241E47A01AA01EB4A
:1087E000046103EB00602C4B984700287FF40DAF29
:1087F0001B4B019A5A604B221A7004225A8004E7DC
:108800004388063B9BB21F2B05D9154B00225A808B
:1088100045221A70F9E64379807903EB0023E07969
:1088200003EB0043207A04F10902217903EB006095
:108830001A4B984728B90A4B00225A8024221A70F2
:10884000E3E6074B00225A8045221A70DDE6438892
:1088500033B3034B00225A8045221A70D5E600BF7D
:10886000941C0020958440008D844000A114410098
:10887000D5794000981C002089794000CDFF400048
:10888000795F4000B1784000E578400029794000E8
:108890008165400029684000C56740000D684000C0
:1088A0000020474B1871474B984720B1444A137931
:1088B00043F0010313710120424B984720B1404A15
:1088C000137943F00203137102203E4B984720B105
:1088D0003B4A137943F0040313710320394B984743
:1088E00020B1374A137943F008031371344B012246
:1088F0005A8054221A7088E64388012B05D0304BE9
:1089000000225A8045221A707FE60379463B102BDD
:1089100049D8DFE803F03F4809484848124848363C
:108920002D48481B48482400274B9847244B187172
:108930004A221A7001225A8067E6244B9847204B3E
:1089400018714A221A7001225A805EE6204B98471D
:108950001B4B18714A221A7001225A8055E61D4B92
:108960009847174B18714A221A7001225A804CE618
:10897000194B9847124B18714A221A7001225A80DB
:1089800043E6164B98470E4B18714A221A70012283
:108990005A803AE6124B9847094B18714A221A70CE
:1089A00001225A8031E6064B45221A7000225A8075
:1089B0002BE6034B00225A8045221A7025E600BFA1
:1089C000941C00208D684000F180400031814000FF
:1089D000A98140002D824000418240005183400027
:1089E0007583400000487047941C0020F0B583B0A8
:1089F000EFF31083B3FA83F35B09019372B6BFF30D
:108A00005F8F0022364B1A70019E364B1B68364A28
:108A100015682B447F2B2AD8324B1C6822463349D9
:108A200033482844334B98472C442F4B1C6000227A
:108A30002C4B1A602EB10122294B1A70BFF35F8FA5
:108A400062B62D4A284B196829482C4B9847014695
:108A5000D0B1274BC31A284842881A44951D447840
:108A6000012C15D044BB802B1CD900242AE01D4AC0
:108A7000136814682C441B1B03F18004204A1378EC
:108A800043F001031370C9E70024174B1C6019E081
:108A90001748154F3E68761B32464119194B9847C7
:108AA0003E600FE0104D2C68E41A22461048154B2A
:108AB00098472C60002405E00133802B05D9002461
:108AC000094B1C60204603B0F0BD0948064D2C68D8
:108AD000E41A2246C1180B4B98472C600024F1E79A
:108AE0002F030020DC1F0020EC1F0020342000207A
:108AF000DC1E0020A1144100F01F002099844000DA
:108B0000E81F0020D515410010B50DE0144B195D8C
:108B10001448154B98470134E4B2144B1B689C422F
:108B2000F4D30022114B1A600120114B9847114BCE
:108B300098470128F8D11048104B9847104B984798
:108B40000246802106480F4B98470128ECD10C4B78
:108B5000984743880633054A13600024DDE700BFC9
:108B60005C1F0020008201401FD94000E41F00204C
:108B700075EC4000ED894000F01F00207185400039
:108B8000E58940002985400030B583B08024224625
:108B900000211C481C4DA847224600211B48A8471D
:108BA00000231B4A13601B4A13601B4A13701B4AA5
:108BB00010215166C2F8901051655162C2F88010C0
:108BC000116F21F010011167516F21F010015167F1
:108BD000134A4FF400211160202182F81313012160
:108BE000104A9160104A0192009322460F491048A2
:108BF000104CA047012802D00F48104B984703B0F3
:108C000030BD00BF342000209D1641005C1F0020B5
:108C1000DC1F0020E41F0020E81F0020000E0E4093
:108C200000E100E000820140E01F0020944141008B
:108C3000098B4000A1E940009C414100F50D410035
:108C4000104B1B6913F0010F12D00E4B5B6913F030
:108C5000010F0DD00C4B1B687F2B0AD90B4A1378E0
:108C600043F001031370074B9A69094B83F87F2087
:108C70007047054A1368591C1160024A9169044AF9
:108C8000D154704700820140DC1F0020E81F002003
:108C900034200020064A936823F07F4323F4706356
:108CA00043F0254343F4E0639360024B1360704745
:108CB00000140E40080000A570B506460D46094B8D
:108CC00098470446002040B929462046064B98475D
:108CD00028B93046054B9847F5E7012070BD0020C4
:108CE00070BD00BF797640009176400029AB40000E
:108CF00010B54FF47A722B4B1A8004E04022002109
:108D000029482A4B9847274B188880B2284B984708
:108D1000254C2323237014236370264B9847C0F3FC
:108D20000F23A370E070244B9847C0F30F232371E7
:108D30006071224B9847C0F30F23A371E071204B61
:108D40009847C0F30F23237260721E4B9847C4F8F4
:108D50000A001D4B1B7807EE103AB8EE477A9FEDDC
:108D60001B6A27EE067ADFED1A6A37EE667A17EE8F
:108D7000103AC4F80E30174B1B7807EE903AF8EE15
:108D8000677A67EE867A77EEE67A17EE903AC4F85D
:108D90001230114B98470028B0D0322120460F4B9B
:108DA0009847ABE728210020D82000209D164100DD
:108DB00075EC40003D514000CD574000516A4000E5
:108DC0005D6A4000CD7B4000F8010020B4C8363F0A
:108DD0006FDB4A42F9010020EFFF4000B98C4000F0
:108DE000F0B583B0402200219A489B4B98470BE294
:108DF0009A4B98479A4B984711E2984B9847994B52
:108E0000BB221A601A225A60954B98470AE2914990
:108E10000B462A2203F8012B934A1068C1F801007F
:108E200091889279104699809A71FEE101208F4BCA
:108E3000984728B9874B45221A7002225A70F7E1E9
:108E40008449252301F8013B0120894B9847EFE134
:108E50000820864B984728B97E4B45221A7002227B
:108E60005A70E8E17B49262301F8013B0820804B3A
:108E70009847E0E109207D4B984728B9754B45227A
:108E80001A7002225A70D9E172497E2301F8013B1F
:108E90000920774B9847D1E1C4F30723032B09D866
:108EA000DFE803F0020B0406724807E0724805E0B1
:108EB000724803E04FF0FF3000E07148B0F1FF3F2F
:108EC00010D001A96F4B984730B9624B5A221A70E3
:108ED000019AC3F80120B5E15E4B45221A700222C7
:108EE0005A70AFE15B4B45221A7001225A70A9E11A
:108EF000C4F30723032B09D8DFE803F0020B0406B1
:108F00005C4807E05C4805E05C4803E04FF0FF3058
:108F100000E05B48B0F1FF3F0ED05B4B19685B4B44
:108F2000984718B924224B4B1A708EE1494B4522C1
:108F30001A7003225A7088E1464B45221A700122AA
:108F40005A7082E12422434B1A7081E1414B452241
:108F50001A704F4A12785A707DE14E4B1B780F2BD6
:108F600005D93C4B45221A7001225A7076E14A4BD2
:108F70009847384A5523137020235370454B1B786C
:108F800000EB4310D0F800E047688668C168C2F87B
:108F900002E0C2F80670C2F80A60C2F80E10D0F8FB
:108FA00010E047698669C169C2F812E0C2F816701C
:108FB000C2F81A60C2F81E1050E1264B4B221A70FC
:108FC00004225A706A44354B1968354B1868354B82
:108FD000984720B91F4B019AC3F8022041E10022B3
:108FE000314B1A603DE11B4B54221A70002058701F
:108FF0002E4B984720B1174A537843F00103537022
:1090000001202A4B984720B1124A537843F00203BB
:1090100053700220254B984720B10E4A537843F0F5
:10902000040353700320214B9847002800F01C8153
:10903000084A537843F00803537015E11C4B187825
:10904000072837D9802841D0024B45221A700122C7
:109050005A700CE1302100209D16410049FF40006C
:10906000958C400090140E4034424100D579400068
:10907000897940000110FFFF0310FFFF0410FFFF7C
:109080000210FFFFAD7D400024210020F57D40004F
:109090002A21002020210020B17840002C2100202E
:1090A0001C210020C5674000322100208D6840004F
:1090B000B42000207C4B984718B924227B4B1A70AF
:1090C000D5E07A4A452111705070D0E0784B18787D
:1090D00010F0800FB8D1774B984718B92422734B02
:1090E0001A70C4E0714B452119705870BFE0724A84
:1090F000724B1968724B1868724B984718B9242242
:109100006A4B1A70B6E0694B452119705870B1E08E
:1091100066484E2300F8013B6B4B9847002800F04F
:10912000AC806A4B4FF020321A605A609A60C3F8E4
:109130000B20A2E014F47F4F5C4E31464FF05E03EB
:1091400001F8023B14BF01200020614B984770706A
:10915000002840F095804522327091E04A22534B1E
:109160001A70C4F30723463B102B2DD8DFE803F019
:10917000272C092C2C2C0E2C2C221D2C2C132C2CA7
:109180001800544B9847494B58707CE0524B984715
:10919000464B587077E0514B9847444B587072E0FB
:1091A0004F4B9847414B58706DE04E4B98473F4BA3
:1091B000587068E04C4B98473C4B587063E04B4B01
:1091C00098473A4B58705EE0384B45221A7001229E
:1091D0005A7058E0464B98472422344B1A7054E09A
:1091E0009A000232434951F823003049505001336C
:1091F000DBB20B2BF4D9404B984700284ED14022CC
:1092000000212A483D4B98474FF0FF3101203C4B4D
:10921000984704460028F7D043283FF4E9AD422C94
:109220003FF4EBAD2A2C3FF4F2AD252C3FF4FEAD1C
:10923000262C3FF40DAE7E2C3FF41CAEE5B25A2D29
:109240003FF42AAE7A2D3FF453AE242C3FF47AAE8D
:10925000452C3FF47BAE552C3FF47FAE4B2C3FF4B6
:10926000ACAE542C3FF4BFAE442C3FF4E7AE412CDF
:109270003FF43DAF4E2C3FF44BAF5E2D3FF45AAF61
:109280004A2D3FF46BAF3D2CA4D0732CB3D1074BC8
:1092900073221A7030225A700023AAE73221034841
:1092A000184B9847ABE700BF2968400030210020E9
:1092B0001821002059684000B82000202C210020EF
:1092C0001C2100200D68400015694000312100205C
:1092D00069554000F180400031814000A981400083
:1092E0002D82400041824000518340007583400040
:1092F000F9A2400014230020EFFF40009D1641001A
:1093000081F14000B98C400010B5002303220146D2
:1093100002480068024CA04710BD00BF340D002079
:10932000A9F2400010B584B0002304AA42F8043D1D
:1093300009490C680092032201462046074CA047C9
:10934000039B3BB14FF08052054B1A60BFF34F8F28
:10935000BFF36F8F04B010BD340D002055F34000F3
:1093600004ED00E010B582B00F4B01930123009390
:10937000002380220D490E480E4CA047012802D040
:109380000D480E4B98470023019301220092802242
:109390000B490C48074CA047012802D00A48074B4C
:1093A000984702B010BD00BF340D0020BC41410001
:1093B000E18D4000A1E94000CC414100F50D4100A4
:1093C000FC414100F18C40000842410070B584B07E
:1093D000044603782A2B00F091802378252B00F097
:1093E00091802378262B00F0918023787E2B00F04B
:1093F000918023785A2B00F0918023787A2B00F00B
:1094000094802378532B00F0A3802378472B00F01F
:10941000AC802378672B00F0B9802378462B00F0CE
:10942000C0802378522B00F0C3802378502B00F0AB
:10943000D38023785E2B00F0F7802378492B00F04F
:1094400004812378432B00F013812378422B00F012
:1094500013812378552B00F013812378572B00F0CC
:1094600016812378562B00F0258123784C2B00F0B1
:109470002E8123784D2B00F03E8123784B2B00F07A
:1094800083812378542B00F09B812378442B00F0B8
:109490009B812378412B00F0AE812378592B00F07B
:1094A000CC8123784E2B00F0E18123784A2B00F009
:1094B000E1812378402B00F0E38123786F2B00F0CB
:1094C000F8812378642B00F006822378702B00F05B
:1094D000248223785B2B00F0398223783D2B00F027
:1094E0003B822378732B00F03B8225782C2D00F0F3
:1094F0003B822E2D00F0418204B070BD2A20934B98
:1095000098476AE72520914B98476AE726208F4BBA
:1095100098476AE77E208D4B98476AE7607800029B
:1095200040F05A00894B984767E7A378E27803EB4D
:109530000223227903EB0243627903EB0263844A3C
:1095400013606078000240F07A00804B984758E73B
:10955000637833B901207F4B984724207B4B984791
:1095600053E700207B4B9847F7E76378A07800EB40
:10957000032080B210F4004F05D1774B9847242088
:10958000724B984745E747F6FF70F6E76378A07897
:1095900000EB032000B2714B984724206B4B984797
:1095A0003BE760786E4B98472420684B984738E734
:1095B0006278A37803EB02239BB2092B05D9694A91
:1095C00013802420614B98472FE70122664B1A70C5
:1095D00045205E4B984728E763785BB1012B16D096
:1095E0000022624B1A7001225F4B1A704520574BC4
:1095F00098471EE702205E4B984730B904225A4B29
:109600001A704520514B984713E72420FAE70120B0
:10961000574B984720B90422534B1A70452000E05D
:1096200024204A4B984704E763782BB1012B07D0DD
:109630004520464B984700E75E20444B9847FCE6A0
:109640004FF4AF70414B9847F7E66278A37803EB8D
:109650000223484A13800520454B984720B904222D
:10966000414B1A70452000E02420384B9847E8E62B
:109670004320364B9847E8E64220344B9847E8E6CB
:1096800062783D4B1A705520304B9847E5E661787B
:109690000F2908D820224901A01C384B98472420C4
:1096A0002A4B9847DDE601222F4B1A704520274BA5
:1096B0009847D6E608202E4B984720B904222A4B1B
:1096C0001A70452000E02420204B9847CDE62C4B13
:1096D00062781A70A2785A70E2789A700720244B48
:1096E000984720B90422204B1A70452000E024201E
:1096F000164B9847BDE6234B98476378003318BF55
:1097000001230370A3784370E378003318BF01236B
:1097100083702379C37063790371A3794371E3790B
:109720008371237AC371637A0372A37A4372E37AF3
:10973000837209200E4B984720B904220A4B1A70F5
:10974000452000E02420014B984796E625934000F1
:109750002421002025744000ED734000197440005E
:10976000F1504000282100202A210020DB21002088
:10977000D9A94000F621002020210020E5784000F2
:10978000D8210020D95740006378A27803EB022348
:10979000E27803EB0243227903EB0263804A136011
:1097A0006379A27903EB0223E27903EB0243227A85
:1097B00003EB02637B4A13604B207B4B984760E6C8
:1097C0005420794B984760E609227849E01C784B91
:1097D000984748B96278774B1A70A278764B1A701E
:1097E0004420714B984754E60122744B1A7045206F
:1097F0006D4B98474DE66278531EDBB21F2B06D99E
:1098000001226E4B1A704520674B984745E6654B21
:109810001A60A378E17803EB0123217903EB01437C
:10982000617903EB01635E490B60A11D6448654BE0
:10983000984741205C4B98472FE6002604AD45F839
:10984000046D614B984700953346012204215F4D1A
:10985000A847039B002B3FF424AE4FF080525C4B93
:109860001A60BFF34F8FBFF36F8F1AE64E204E4B37
:1098700098471AE6607800024A304B4B984718E642
:109880000120544B9847504B984703AB009300235B
:10989000012204214D4DA847039B002B3FF40DAE40
:1098A0004FF080524A4B1A60BFF34F8FBFF36F8F58
:1098B00003E6E21C6178A078474B98470620474BA7
:1098C000984720B904223D4B1A70452000E024201F
:1098D000354B9847F5E56078414B9847012803D010
:1098E0004520314B9847F0E524202F4B9847364BC5
:1098F000984703AB0093002301220421334DA8476E
:10990000039B002B3FF4E1AD4FF08052304B1A60C7
:10991000BFF34F8FBFF36F8FD7E5324B98472A4B7A
:10992000984703AB0093002301220821274DA84745
:10993000039B3BB14FF08052254B1A60BFF34F8F12
:10994000BFF36F8F2420184B9847C2E5264B9847EA
:109950002420154B9847C0E53D20134B9847C0E5A0
:109960007320114B9847C0E508222049601C104B1A
:10997000984700287FF4BDADFFDE08221B49601C1C
:109980000B4B984700287FF4B7AD194B4FF40042BA
:109990001A60402183F80F13C3F80021ACE500BF23
:1099A0001C2100202C210020259340003C42410036
:1099B00041144100B4200020182100202A21002059
:1099C000B8200020A1144100C99B400055F340007D
:1099D00004ED00E0299C4000D1A84000D9A9400036
:1099E000499C400015A3400021A34000484241008B
:1099F00000E100E08388B3F59F5F0DD0B3F5706F91
:109A00001DD0B3F5206F27D0B3F5A05F30D0B3F5EC
:109A1000706F39D000207047C288B2F51F6FEDD14A
:109A20004289A2F5E751093989B2C6293DD9A2F583
:109A3000DD521D3A92B2C62AE0D802207047C28891
:109A4000B2F5F06FDDD14289A2F50B52053A92B220
:109A5000C62AD6D803207047C288B2F5206FD3D16A
:109A60004289A2F6553292B2C62ACDD80520704757
:109A7000C288B2F5206FCAD14289A2F6553292B29D
:109A8000C62AC4D805207047C388B3F5F06F01D04B
:109A9000002070474389A3F5B8530D3B9BB2C62BFA
:109AA00001D8042070470020704701207047000053
:109AB00038B50125044B1D7000210846034CA04712
:109AC00000212846A04738BD390D0020B55440007C
:109AD00010B50024022C09D80B4B1A780021084637
:109AE0000A4B9847012801D00134F3E70024022CE7
:109AF00009D8054B1A7800210120044B984701280A
:109B000001D00134F3E710BD3A0D0020A953400005
:109B100010B5154B1B786BB90024022C15D8134BCC
:109B20001A78134B19880020124B984701280CD043
:109B30000134F2E7012100200F4CA0470121084623
:109B4000A04701200D4B9847E6E70024022C0AD8D5
:109B5000064B1A78064B19880120064B98470128B6
:109B600001D00134F2E710BD390D00203A0D00207C
:109B70002C010020A9534000B554400075EC400072
:109B8000F8B505460E460024204601E00134A4B293
:109B90002746B4EB960F14D215F8241005EB840376
:109BA0005A7801EB02219A7801EB0241DB7801EB54
:109BB00003610028EAD107F540608000014B984717
:109BC000E4E7F8BD4D654000014B1868704700BFE1
:109BD000400D0020014B1878704700BF3D0D00205C
:109BE00010B582B0074B01930023009380220649F1
:109BF0000648074CA047012802D00648064B984764
:109C000002B010BD400D002054474100959C40001B
:109C1000A1E9400060474100F50D4100014B187873
:109C2000704700BF380D002018B9044A044B1A6071
:109C30007047044A024B1A60704700BF5446410007
:109C40002801002054424100032817D8DFE800F023
:109C500002070C110A4A0B4B1A60012070470A4A8E
:109C6000084B1A6001207047084A064B1A60012011
:109C70007047074A034B1A60012070470020704765
:109C800054464100280100205445410054444100FD
:109C900054434100F0B585B001238DF80B309B4B48
:109CA000009300231A469A499A489B4CA0479B4B25
:109CB000186004A9502301F8063D0320984CA047E2
:109CC00004A9002301F8073D0D20A04710B9002387
:109CD00003930BE09DF80900924B9847F7E74FF08C
:109CE000FF3303AA002108468F4CA047039B13F0C3
:109CF000010FF4D040F213108C4B98478C4B9847CF
:109D00004FF480718B4B18688B4B984706E04FF0EF
:109D1000FF3303AA00210846834CA047039B13F09E
:109D2000020FF4D01920814B9847844B4FF4807276
:109D30001A63DB6B13F4004F19D0814B98470F2047
:109D4000804B984701467D487F4B984700227F4BC8
:109D50001A700DF10B010420714B984728B19DF842
:109D60000B3083F001038DF80B30002403E0784BB7
:109D70009847E4E7002414206C4B9847002303AA7B
:109D80001C211846684DA847039B13F0080F00D00C
:109D9000012413F0100F6FD1039B13F0040F2ED08A
:109DA0006A4B1B78002B40F0FF800F20654B9847D3
:109DB00001466248674B9847654B9847664B984702
:109DC0005B4B98475B4D4FF4807128685A4B98471E
:109DD0002A68624B9A4200F0F380584BDB6B13F415
:109DE000004F00F0F080564B98470F20554B984796
:109DF00001465248544B98472420594B9847534B9F
:109E00001B78002B40F0E280564B9847002840F02A
:109E1000FF8000224D4B1A709DF80B3093B1524BCE
:109E20001B787BB1514B1B78002B00F0D181504B3C
:109E3000984738B900224D4B1A704E4B984700286E
:109E400040F0B481002C96D0484B1D78002D91D164
:109E50003E4B1C78002C8ED00122474B1A70474B8A
:109E600098472E4B18680A23009300231A460321B3
:109E7000434CA0472C467EE70F20324B98472F4E8D
:109E800001463046334B9847314B98474FF4804753
:109E900077630A20254DA8473A4B98474FF4FA704C
:109EA000A847394B984777630120384B98471920CA
:109EB000A8474FF4807333630020354EB04701202C
:109EC000B04700210846334EB04700210120B0477B
:109ED00001210020304EB04701210846B04701273C
:109EE0001A4B1F702D4B98479DF80A100023032230
:109EF00041F480712A4EB0472A4B984700233A46D6
:109F00000221B0474FF0FF30A84745E7B19A400023
:109F1000E0930400884741003DF640007021002096
:109F200089794000499C400005F2400075EC4000F2
:109F3000A964400028010020819B4000000E0E40D3
:109F4000CD51400013D34000EFD240003D0D002022
:109F5000A9514000F3D24000E56440005442410062
:109F6000099340001D004100240100202E01002023
:109F7000C1574000D59B4000380D0020119B400088
:109F800079F6400039764000B5754000E175400033
:109F90004156400091544000B554400031AA400061
:109FA000A9F240003DAA40000022974B1A70974D3D
:109FB0004FF480766E631920954B98472E63F4E634
:109FC000944B984709E7944B98470EE7934B984773
:109FD00020B1934B984700287FF416AF00258A4B99
:109FE0001D70904B98472B4603224FF480718E4E84
:109FF000B0478E4B98472B4601220421B047834D32
:10A000004FF480766E631920814B98472E63FBE6F0
:10A01000834B984700283FF4FCAE7B4B1B78002B0A
:10A020007FF4FAAE0020824EB047824D28700120A6
:10A03000B047814B18702B78002B3FF4EDAE002811
:10A040003FF4EAAE0122704B1A707C4D28467C4BDF
:10A05000984728467B4B98470746052816D000228C
:10A06000794B1A704FF4FA70694B98470020704E84
:10A07000B047704D28700120B0476F4B18702B7897
:10A0800003B138B90022604B1A70C5E601226E4B4D
:10A090001A70E7E7634B98479DF80A1000230322E4
:10A0A00041F48071604DA847604B9847002301221E
:10A0B0000221A84739460020644DA84739460120AF
:10A0C000A8470A20624B9847D8B9624D002128461C
:10A0D000614B98472B78112B18D0002108465F4D13
:10A0E000A84700210120A8470025022D20D8564B63
:10A0F0001A78002108465A4B9847012818D0013594
:10A10000F3E758490A20584B9847DEE76B78002B55
:10A11000E3D1AB78002BE0D1EB78892BDDD12E4653
:10A1200029460020514DA84731460120A847D4E7D1
:10A130000025022D09D8444B1A7800210120484BF4
:10A140009847012801D00135F3E701210020484D4F
:10A15000A84701210846A8479DF80B3003B3454B9B
:10A160009847E8B1444B1B78D3B1444B1B782BB1D3
:10A170000122434B1A70434B98474DE60025404B54
:10A180001D70414B9847414B1E68414B98470A232D
:10A1900000932B460246012130463E4DA8473BE640
:10A1A0000122374B1A70374B984735E60025344B60
:10A1B0001D70354B9847354B1E68354B98470A2321
:10A1C00000932B46024601213046324DA84739E61E
:10A1D000314B984700283FF435AE0122274B1A70C7
:10A1E0002E4B984700283FF42DAE0122244B1A70C5
:10A1F000244B9847254B18680A23009300231A46DE
:10A200000321244DA8471DE63D0D0020000E0E4001
:10A2100075EC40008D674000A95140001D004100D1
:10A220002900410031AA4000A9F240003DAA4000A7
:10A23000456640003B0D00203C0D0020CC21002055
:10A2400081664000F59940003A0D0020B15540006C
:10A25000D5794000742100209D6540009154400054
:10A26000A95340002C010020897940009D554000F1
:10A27000B554400015574000240100202E01002055
:10A28000380D0020119B4000D19A40007021002021
:10A290009DEA400079F64000C1574000D59B400040
:10A2A00038B5114B1880114B1B786BB10446002553
:10A2B000022D0AD80E4B1A78214600200D4B9847E4
:10A2C000012802D00135F3E738BD0025022D09D859
:10A2D000074B1A7821460120064B9847012801D0E8
:10A2E0000135F3E738BD00BF2C010020380D0020F8
:10A2F0003A0D0020A953400010B5044B98470023A5
:10A3000003221021024CA047012010BDC99B400030
:10A31000A9F240000022014B1A707047240100206E
:10A320000122014B1A7070472401002038B5002427
:10A33000204609E000F47F43B3F5007F0CD000F421
:10A340007F43B3F5807F0CD00028F3D14FF0FF316D
:10A350000120134B9847EDE70020124B984700204F
:10A36000EDE7C5B2002008E00134A4B220460D4B51
:10A3700098470A2101200A4B984758B9AC42F3D3B9
:10A3800008E0013CA4B22046064B98470A21012070
:10A39000034B98470028D7D1AC42F2D8D4E700BF8E
:10A3A00081F14000F1504000F0B583B0022400205C
:10A3B00010F0010F0AD14FF0FF310120314B9847C7
:10A3C00000F00E03042BF3D10424F1E72E4B1B689D
:10A3D000ADF804301B0C8DF8063001A902202B4B80
:10A3E0009847042C07D02A4B984701A9294B984736
:10A3F00000252E4607E0264B98470021264B98471C
:10A40000F1E72E460225322101201E4B984700F02D
:10A410000E00042812D0022814D0042CF3D1C5B1A8
:10A42000022D22D0032DEED10136F6B2182EEAD934
:10A4300000252E46E7E703250026E4E700252E4603
:10A440000424E8E7124B98478021134B98470224D5
:10A45000E3E70F4B9847771CFFB2104B995D0E4B0B
:10A460009847632FCDD83E46CDE7094B9847771CD8
:10A47000FFB20B4B995D084B9847632FDBD83E46E4
:10A48000C1E700BF81F140009C474100897940004D
:10A49000CDFF4000795F4000295F4000940100201B
:10A4A0003001002008B5044B98476420034B9847BF
:10A4B000034B9847F7E700BF096A400075EC40007E
:10A4C0003D7B400070B582B0944B9847944B9847C1
:10A4D0000120944B984702A9002301F8013D052073
:10A4E000914B984728B19DF8073013B100208D4B50
:10A4F00098478E4B98478E4B98478E4A8E4B1A60E2
:10A5000001208E4B9847044690B98A4D8C4C0FCC55
:10A5100028606960AA60EB608A4B98478A4B98472D
:10A5200002228A4B1A638A4B98470546002416E09C
:10A53000814B196801207C4B984705E07E4B1B68D6
:10A5400000221A550134E4B20F2CF7D9E4E70520B4
:10A55000804B98477E4B984705460134E4B20DB9CD
:10A56000132CF4D97C4B984729467C4B98477C4B5D
:10A5700098477C4DA8470023012211467A4CA047FA
:10A5800001207A4B9847A847002301220221A047C7
:10A59000774B98476B4B9847764B9847002301229F
:10A5A000052175480068A04700252C4680E011462B
:10A5B000002341F8043B7148714B984738B9714BFF
:10A5C0005968013159606D486F4B98477BE0012114
:10A5D0006A486D4B984776E01146002341F8043BEA
:10A5E0006A48674B984798B9694B59680131596077
:10A5F0006648654B984767496748614B984760B91B
:10A60000634B59680131596063485F4B984768E074
:10A6100001215E485C4B9847EDE701215E485A4BAB
:10A6200098475EE0134600221A605A6801325A6069
:10A6300069465A48524B984750B9594B5968009B44
:10A64000994201D8002514E054484F4B9847F9E748
:10A65000534B596851484C4B9847F3E7514A13689C
:10A6600001331360052B44D94D4B00251D605D60FF
:10A6700015604D4BA3FB0423DB0803EB83035A0057
:10A68000944238D0494B9847002840F09D80484B71
:10A69000A3FB04235B09642202FB1343002B00F09D
:10A6A00096800A202B4B98470134632C00D9002454
:10A6B0000135B5F57A7FDCD3324A13680133136074
:10A6C0003B2B3FF674AF3B4B98470028C6D0002287
:10A6D000344B1A602E4A1368013313603B2B3FF64C
:10A6E0007BAF2F4A1368013313603B2B9AD80025A8
:10A6F000BFE70025BDE7304B984728B947232F4ACD
:10A7000013702F4A1370BDE700202E4EB0472B4B1D
:10A7100018700120B0472A4B1870B3E71980400029
:10A72000717A40009D51400089794000A951400054
:10A73000E54F4000FC210020DC210020D5794000BD
:10A7400054484100CDFF400011614000000E0E4012
:10A75000696A400075EC4000C5FF4000D9614000C7
:10A76000B5754000C99B4000A9F24000E17540006A
:10A7700051564000655E4000680D00200110FFFF4B
:10A78000AD7D4000580D0020F57D40000210FFFF18
:10A79000480D00204C0D00200410FFFF0310FFFFA8
:10A7A000500D0020440D0020CDCCCCCC15574000DE
:10A7B0001F85EB511D9C4000D59B4000F8010020F7
:10A7C000F901002025554000024B984769E7024BEC
:10A7D000984766E7215740005156400008B509E008
:10A7E000002108462D4CA04700210120A04700224F
:10A7F0002B4B1A704FF0FF3101202A4B9847284B02
:10A800001B78013B082BF2D801A252F823F000BFBD
:10A8100035A84000E1A740004FA840005FA84000D5
:10A8200045A8400087A840006FA840007BA84000D2
:10A8300081A8400001210020184CA04701210846B2
:10A84000A047D4E7184B1888184B9847CFE700214A
:10A850000846174CA04700210120A047C7E7012167
:10A860000020134CA04701210846A047BFE7114B29
:10A8700098471149114B9847B9E7114B9847B6E7EC
:10A88000104B9847B3E7104AD01E134612F8032C1A
:10A89000817840780D4CA047A9E700BF05554000DE
:10A8A000DB21002081F14000F6210020A1A2400020
:10A8B000B5544000CDFF4000D8210020795F400012
:10A8C00029794000E55740000F220020E95240005E
:10A8D00010B51446044B1870597002462146981C56
:10A8E000024B984710BD00BF0C220020A11441006C
:10A8F00010B582B0234B01930323009300238022E1
:10A9000021492248224CA047012802D02148224B4D
:10A910009847224B0193002300938022204921482D
:10A920001B4CA047012802D01F481B4B984700230F
:10A930000193009380221D491D48154CA047012812
:10A9400002D01C48144B98471B4B019300230093E3
:10A9500080221A491A480E4CA047012802D01948F3
:10A960000D4B9847184B0193002300938022174901
:10A970001748074CA047012802D01648064B9847B5
:10A9800002B010BD640D0020A0474100DDA74000CB
:10A99000A1E94000A4474100F50D41006C0D0020E5
:10A9A000C0474100C5A44000CC474100F4474100E6
:10A9B000A5A44000F8474100680D0020144841005C
:10A9C000A9A3400018484100600D00203448410010
:10A9D0002DA340003848410010B584B0104B1870CA
:10A9E0000022039204AB43F8082D0E4A106803AA14
:10A9F0000092042201210C4CA047029B5BB9039BEF
:10AA000063B14FF08052094B1A60BFF34F8FBFF311
:10AA10006F8F012000E0002004B010BD0120FBE793
:10AA2000DB210020640D002055F3400004ED00E020
:10AA3000014B1868704700BF600D0020014B18687B
:10AA4000704700BF680D00200023044A1370044AB9
:10AA500013700120034B1870704700BF780D002061
:10AA6000740D0020710D0020704700207047000019
:10AA70000D4B5B881A0A032A01D00020704713F09F
:10AA8000FF0F0ED1084BDB88402B01D00020704710
:10AA9000054B064A9A60064A1A6140229A810120B3
:10AAA00070470020704700BF702200207C0D0020FE
:10AAB000E5AA40000122014B1A707047710D002079
:10AAC00010B5034B034A04490448054CA04710BD88
:10AAD00071AA4000CC020020740D0020780D0020E7
:10AAE00029AC400008B5084B9B89402B00D008BD1D
:10AAF000064B1B781BB90648064B9847F7E70448F6
:10AB0000054B984708BD00BF70220020700D002043
:10AB10007C0D0020CD934000FD4E4000014B18708D
:10AB2000704700BF700D0020224B1B780BB91846F0
:10AB300070472DE9F04184B00746EFF31083B3FA74
:10AB400083F35B09039372B6BFF35F8F00211A4B47
:10AB50001970DDF80C80194D40222846184B984793
:10AB60003C4640372E4620686168A268E3680FC6FD
:10AB700010343546BC42F5D1124B009340230F4AA6
:10AB800000218120104CA04780F00100094B187073
:10AB9000B8F1000F05D00122074B1A70BFF35F8F89
:10ABA00062B6044B1B7883F00103184604B0BDE87D
:10ABB000F08100BF710D00202F030020BC0D00208C
:10ABC0009D164100B5AA400005CE400010B50446D0
:10ABD000134B9847837A212B01D0002010BD00F140
:10ABE0000902104B5B881B0A212B04D0C27B9342C5
:10ABF0000BD0002010BD0B4B9A60427AD9888A4254
:10AC000028BF0A469A81012010BD064B9C60028A2B
:10AC1000D9888A4228BF0A469A81012010BD00BF08
:10AC200001B2400070220020F8B5264C247865B2AD
:10AC3000002D07DB002D40DB04F06004202C22D027
:10AC40000020F8BD14F0600603D11E4F7F78062F58
:10AC50000BD0202EEED11B4A5278022A09D0032AAB
:10AC60000CD0012AE6D19847F8BD1046164B9847FC
:10AC7000F8BD144B986001209881F8BD114B996084
:10AC800001209881F8BD0F4A52780A2A07D00B2A72
:10AC90000BD0092A01D00020F8BD9847F8BD094B18
:10ACA0005B881B0A03700120F8BD064BDB8833B9B3
:10ACB000044B5B880B700120F8BD0020F8BD00201C
:10ACC000F8BD00BF70220020CDAB4000014B1868DA
:10ACD000704700BFDC210020024B1B681B685888AE
:10ACE00018447047080E002038B504460D46094B3D
:10ACF0009847024620782044904207D24378042B9C
:10AD000006D0AB4205D003781844F5E7002038BDE3
:10AD1000002038BDD9AC400038B5144B1B780BB3BC
:10AD2000134B1B681B681A7982421DD90D460446D5
:10AD3000104A1360104B984703E01A7813440D4AE9
:10AD400013600C4B1B6898420AD95A78042AF4D134
:10AD50009A789442F1D1DA78AA42EED1012038BD36
:10AD6000002038BD002038BD002038BD040E002072
:10AD7000080E00200C0E0020D9AC4000084BDB88E8
:10AD800063B9074B5B88012B01D000207047054A4F
:10AD9000138823F0020313800120704700207047BE
:10ADA00070220020FC0D002000207047044BDB883F
:10ADB00023B9044A024B1A610120704700207047F2
:10ADC00070220020F1B0400038B5134B1B7803B35C
:10ADD000124B1C79124B1B681B681B799C4201D3D8
:10ADE000002317E0002120460E4B9847034688B108
:10ADF0000B4B1B685B6853F82450EB68984701467F
:10AE00002046084B9847034620B1AB689847034655
:10AE100000E00023184638BD040E002070220020F8
:10AE2000080E002019AD400038B5104B1B78D3B187
:10AE300000240F4B1B681A681279944211D25B6888
:10AE400053F82450EB68984701462046094B984731
:10AE5000034648B1AB689847034628B90134E4B2C9
:10AE6000E7E7002300E00023184638BD040E002069
:10AE7000080E002019AD400070B504460021114BAA
:10AE80009847054608B9284670BD0F4B1B685B689C
:10AE900053F82460F368984701462046094B9847C9
:10AEA00005460028EFD0094B1C6805212046084BB9
:10AEB0009847044618B18078064B9847F5E77368C1
:10AEC0009847E0E719AD4000080E00200C0E002066
:10AED000E9AC400085CB400008B5064BDB88022B6F
:10AEE00001D0002008BD02210348044B98470120EF
:10AEF00008BD00BF70220020FC0D002069CA400080
:10AF000010B5184B9B78032B2AD8DFE803F0050215
:10AF1000100B0920144C0CE004211448144B9847E2
:10AF2000002006E0134B98470446102001E006205D
:10AF3000114C08B1002308E0012010BDE15C0F4A6C
:10AF400002EB430251800133DBB28342F6D3411C52
:10AF50004900C9B209480170054B9847012010BD4E
:10AF6000002010BD702200201C03002018030020C8
:10AF700069CA4000CDAC400028030020F402002044
:10AF800008B5234B5B88DAB21B0A013B0E2B38D87D
:10AF9000DFE803F0081731373737373737373737B8
:10AFA00037372A001B4B186801781B4B9847184B02
:10AFB000DA889B899A4228D2154B9A810123184638
:10AFC00008BD144B1B685B7C9A4201D30023F6E753
:10AFD000104B5B6853F8320041880F4B98470C4B7D
:10AFE0009B6802225A70E2E70A4B986858B1418880
:10AFF000094B9847DBE7094B984703460028D6D111
:10B00000DDE70023DBE70023D9E70123D7E700BF13
:10B0100070220020FC01002069CA400001AF4000FE
:10B0200008B5064BDB88012B01D0002008BD0121AB
:10B030000348044B9847012008BD00BF7022002040
:10B04000040E002069CA400038B5154BDB88012B7F
:10B0500002D00024204638BD124B1B78F3B1104BB0
:10B060001D79114B1B681B681B799D4201D300247D
:10B07000F0E7002128460D4B984704460028E9D008
:10B08000094B1B685B6853F82530DB689847084B11
:10B09000187001211846074B9847DBE70024D9E7D1
:10B0A00070220020040E0020080E002019AD400080
:10B0B000000E002069CA400008B5094BDB88022B4E
:10B0C00001D0002008BD064B1879064B9847064B67
:10B0D000188002211846054B9847012008BD00BF83
:10B0E00070220020D5CB4000FE0D002069CA400030
:10B0F00008B5034B588800F07F00024B984708BD05
:10B100007022002011CA400038B505460F4B984701
:10B110000346C0B10E4B1C68052120460D4B9847D5
:10B12000044640B18288C17880780B4B984703462B
:10B130000028F1D107E0094B1B685B6853F8253004
:10B140001B6898470346184638BD00BF19AD40003C
:10B150000C0E0020E9AC400075CA4000080E00202B
:10B1600038B50C4BDB8893B90B4B1B780BB900231C
:10B170000EE0084B1C799D782046084B9847034603
:10B1800030B129462046064B9847034600E000238D
:10B19000184638BD70220020040E002079AE400011
:10B1A00009B1400008B5074BDB884BB9054B5B88FC
:10B1B0000BB1002008BD034B1879034B984708BD1D
:10B1C000002008BD7022002011CD4000094BDB8813
:10B1D0006BB9084B5B880BB10020704710B5054C6C
:10B1E0002079054B98472079044B984710BD0020E3
:10B1F000704700BF7022002081CF400019CC400072
:10B20000014B1868704700BF0C0E002008B5014BB9
:10B21000984708BDB1C8400010B50B4B1B7863B10F
:10B22000002404E02046094B98470134E4B2084B5F
:10B230001B681B681B799C42F4D30022024B1A70D6
:10B240000122044B1A8010BD040E002079AE40008C
:10B25000080E0020FC0D002008B5024B9847024B59
:10B26000984708BD99C9400019B240001C4BDB88C3
:10B2700013B100231846704710B51A4B984750B3C6
:10B28000174B9A78184B1B685B7C9A4201DD0023B0
:10B2900022E0164B9847124B9B78154A1370EBB17E
:10B2A000114A526803F10053013B02EBC303114AF8
:10B2B000136000240F4B1B681B681B799C4208D24B
:10B2C000002120460C4B9847034628B10134E4B2D4
:10B2D000F0E7012300E00023184610BD0123FBE73F
:10B2E000702200204DCA4000FC01002019B240002D
:10B2F000040E0020080E002009B1400008B5344BB0
:10B300001B7813F0800F0ED113F01F0343D1304A86
:10B310005278013A082A3ED8DFE802F0343D373D42
:10B32000313D3D3D3A002A4AD288002A4ED013F0E2
:10B330001F0306D1264A5278062A0BD0082A0CD0C1
:10B340002AB1012B0CD0022B11D0002008BD214BBB
:10B35000984708BD204B984708BD204B984708BD2B
:10B360001B4A52780A2AEED11D4B984708BD184B4C
:10B370005B780BB1002008BD1A4B984708BD1A4BEB
:10B38000984708BD194B984708BD194B984708BD09
:10B39000184B984708BD012B03D0022B08D0002082
:10B3A00008BD0B4A52780B2AF7D1134B984708BDBA
:10B3B000074B5B78012B03D0032B04D0002008BD82
:10B3C0000E4B984708BD0E4B984708BD002008BD9E
:10B3D00070220020D9AE400081AF400021B0400073
:10B3E00049B04000B9B04000ADAD40007DAD400077
:10B3F000A9AD40006DB2400061B14000A5B1400070
:10B40000CDB140000B4B1B7813B110B5002402E006
:10B4100070470134E4B2084B1B681A6812799442F1
:10B4200007D25B6853F824301B69002BF1D0984792
:10B43000EFE710BD040E0020080E002008B5184BE1
:10B4400000229A811A615A611B7813F0800F11D182
:10B4500013F0600F14D0124B1B7803F01F03012B65
:10B4600014D00F4B1B7803F01F03022B14D00023C2
:10B47000184608BD0A4AD288002AE9D10023F7E716
:10B48000084B984703460028E5D0F1E7064B98475C
:10B4900003460028E5D0EBE7044B98470346E7E76F
:10B4A00070220020FDB24000C9AD400029AE40002E
:10B4B000F8B504460E46114B984705462046104BFA
:10B4C0009847054001D0002403E0F8BD0134062C64
:10B4D00011D88DB123010B4AD058B042F6D102EBFE
:10B4E000041359680D42F1D01F46DB6898477B680A
:10B4F00025EA0305EAE7F8BDF8BD00BFF7D2400032
:10B50000FBD24000100E0020F8B5164C2768062F1D
:10B5100026D8002401E00134E4B2A446A7420AD3AD
:10B52000114E250106EB050E75598D42F3D1DEF85B
:10B5300004509542EFD1CEF80010CEF80420CEF89A
:10B5400008300699CEF80C100137BC4505D01146DD
:10B550001A46064B98470020F8BD02490F60F6E7EF
:10B560000120F8BD800E0020100E0020BDD240004A
:10B570002DE9F04182B004460F4690460A4B9847A9
:10B5800005462046094B984706462046084B9847F3
:10B59000CDF800803B46024631462846054CA04780
:10B5A00002B0BDE8F08100BFFFD240000DD34000E3
:10B5B00013D3400009B5400008B50B210148024BE8
:10B5C000984708BD000E0E40B1B4400008B50C21EC
:10B5D0000148024B984708BD00100E40B1B440002E
:10B5E000F8B506460C461546224B984707464FF0DD
:10B5F000FF313046204B98473046204B9847002C6F
:10B600000CDB630904F01F0101228A4020331C492E
:10B6100041F82320BFF34F8FBFF36F8F002C08DB5F
:10B62000630904F01F0101228A406033144941F884
:10B630002320002C17DB2D01EDB204F1604303F54C
:10B64000614383F80053002C08DB620904F01F04F7
:10B65000012303FA04F40A4B43F8224039463046EA
:10B66000084B9847F8BD04F00F022D01EDB2064BD0
:10B670009D54E8E7FBD24000F3D24000F7D24000EF
:10B6800000E100E0EFD2400014ED00E082B002469D
:10B6900010B9244B1B783BB912B1224B1B780BB36A
:10B6A000204B1A7002B070471F4B1B7803B9FEE79E
:10B6B000EFF31083B3FA83F35B09009372B6BFF321
:10B6C0005F8F0021194B1970009817490B78013BC7
:10B6D0000B700028E0D00121144B1970BFF35F8F6D
:10B6E00062B6D9E7104B1B78FF2B19D0EFF310830C
:10B6F000B3FA83F35B09019372B6BFF35F8F002146
:10B700000A4B1970019808490B7801330B70002817
:10B71000C6D00121054B1970BFF35F8F62B6BFE73A
:10B72000FEE700BF850E0020882200202F030020A6
:10B7300084B02A4B9A6842F480729A609A6822F028
:10B740007F029A601A6B0192019A42F04F020192B5
:10B75000019A22F4074222F080020192019A42F4F7
:10B7600000420192019A1A631C4B1B6B13F4004FA9
:10B77000FAD01A4A136B0293029B43F04F030293D1
:10B78000029B43F400430293029B136300238DF852
:10B79000033006E000BF9DF803300133DBB28DF8C3
:10B7A00003309DF80330DBB2132BF3D9EFF3108392
:10B7B000B3FA83F35B09039372B6BFF35F8F002282
:10B7C000074B1A70039B0121044A116123B1044BFA
:10B7D0001970BFF35F8F62B604B070470040044039
:10B7E0002F030020034A0023136153619381024A0F
:10B7F00013707047702200208A0E002082B005224C
:10B80000104B1A70104A136B0193019B43F04F03C6
:10B810000193019B43F020030193019B13630023D9
:10B820008DF8033006E000BF9DF803300133DBB232
:10B830008DF803309DF80330DBB2132BF3D902B03F
:10B84000704700BF8A0E00200040044082B00322EF
:10B85000104B1A70104A136B0193019B43F04F0376
:10B860000193019B43F010030193019B1363002399
:10B870008DF8033006E000BF9DF803300133DBB2E2
:10B880008DF803309DF80330DBB2132BF3D902B0EF
:10B89000704700BF8A0E0020004004400422014B84
:10B8A0001A7070478A0E002008B5024B1B6903B15D
:10B8B000984708BD7022002030B589B06A4B1B78CC
:10B8C000032B29D0694B9C89694B1B88E41AA4B2CD
:10B8D000002C43D1674A11880B449BB21380634A02
:10B8E000D288934203D0644B1B78002B2CD0634B3F
:10B8F0009847634A136B0393039B43F04F030393EF
:10B90000039B23F001030393039B13635C4B1B6BAB
:10B9100013F0010FFAD115E0594A136B0293029B01
:10B9200043F04F030293029B23F001030293029B17
:10B930001363534B1B6B13F0010FFAD1514B984714
:10B94000514B984709B030BD484B5B6933B19847BC
:10B9500020B10022464B1A80444B9C893F2C37D99A
:10B960000022454B1A704024404B9A68404B1B887C
:10B970001A44EFF31083B3FA83F35B09079372B6AB
:10B98000BFF35F8F0021414B197007983C4B1B6B35
:10B9900013F0020F3ED028B101223C4B1A70BFF3C6
:10B9A0005F8F62B60422304B1A70354A136B0493D2
:10B9B000049B43F04F030493049B23F0010304937F
:10B9C000049B13632E4B1B6B13F0010FFAD1B9E7E5
:10B9D0000122294B1A70C7E7157829490D650133F3
:10B9E000DBB2013299B28C42F6D8214B1A8814444A
:10B9F0001C80234A136B0593059B43F04F0305936B
:10BA0000059B43F010030593059B136300238DF8FA
:10BA1000073008E00023E5E700BF9DF80730013359
:10BA2000DBB28DF807309DF80730DBB2132BF3D96A
:10BA3000134A136B0693069B43F04F030693069B32
:10BA400023F001030693069B13630D4B1B6B13F04E
:10BA5000010FFAD100283FF475AF01220B4B1A7089
:10BA6000BFF35F8F62B66DE78A0E00207022002060
:10BA7000860E0020880E0020840E00209DB8400015
:10BA800000400440A9B84000E5B740002F03002063
:10BA900010B586B0654B1B78012B1ED0022B04D04D
:10BAA000042B02D0624B984701E0624B9847624AF0
:10BAB000136B0093009B43F04F030093009B23F014
:10BAC00002030093009B13635B4B1B6B13F0020F8D
:10BAD000FAD15A4B984706B010BD574B186BC0F3BC
:10BAE0000A40574B9B89574A14882218934201DA1F
:10BAF000181B80B2524B9A682244002305E04E493D
:10BB0000096D11700133DBB2013299B28842F6D867
:10BB10000444A4B24B4B1C8040281BD0484B9C8152
:10BB20005B6913B19847002832D0434A136B0293E4
:10BB3000029B43F04F030293029B23F00203029304
:10BB4000029B13633C4B1B6B13F0020FFAD13E4B6D
:10BB50009847C0E73A4BDA883C4B1B8823449A420B
:10BB6000DCDD374B9B899C4227D0334A136B05930E
:10BB7000059B43F04F030593059B23F002030593B8
:10BB8000059B13632C4B1B6B13F0020FFAD1A2E73A
:10BB9000274B9847284A136B0193019B43F04F03AF
:10BBA0000193019B23F002030193019B1363224B3A
:10BBB0001B6B13F0020FFAD18DE7214B5B6953B178
:10BBC0009847E8B121491F4A0B88108803440B802D
:10BBD00000231380C9E7164B9847174A136B03934A
:10BBE000039B43F04F030393039B23F00203039350
:10BBF000039B1363104B1B6B13F0020FFAD16AE720
:10BC00000B4B98470C4A136B0493049B43F04F0370
:10BC10000493049B23F002030493049B1363064BD9
:10BC20001B6B13F0020FFAD155E700BF8A0E0020FC
:10BC3000FDB74000A9B8400000400440E5B740000F
:10BC400070220020860E00204DB84000880E002093
:10BC50000023042B14D810B40A499A00D418A00069
:10BC600004460844407C214400F083026FF3C7126D
:10BC70004A740133DBB2042BEED95DF8044B7047F4
:10BC8000704700BF8C0E002038B5437C13F0100FB6
:10BC900016D00D46437C6FF30413437404687CB1E3
:10BCA00002F10C03074951F8233013F4806F01D0DF
:10BCB00042F080028168012D14BF00200120A047BE
:10BCC00038BD00BF0040044010B500240BE02346FF
:10BCD0000134E4B203EB8303980022460121034BB5
:10BCE0001844034B9847042CF1D910BD8C0E00204A
:10BCF00089BC400010B500F00F02531E03EB830314
:10BD00009C00012102482044024B984710BD00BF0F
:10BD10008C0E002089BC400030B482B00246441E24
:10BD20003B4900F10C0551F8253051F8251013F06E
:10BD3000020302D001F0400151B9002B39D004EBCD
:10BD400084039900334B0B44597C6FF3830159747E
:10BD500004EB840399002F4B0B445B7C13F00C0F16
:10BD600032D12B4900F10C0551F825300093009B8E
:10BD700043F04F030093009B23F002030093009BCA
:10BD800041F8253002F10C03214951F8233013F01A
:10BD9000020FF7D1002838D0032836D004EB8404F2
:10BDA000A2001C4B13445A7C012161F383025A7494
:10BDB0002BE004EB84039900164B0B44597C0125BE
:10BDC00065F383015974C3E711490C3051F82030F1
:10BDD0000193019B43F04F030193019B23F0400328
:10BDE0000193019B41F8203002F10C03084951F8FE
:10BDF000233013F0400FF7D104EB8404A200054B6D
:10BE000013445A7C6FF383025A7402B030BC7047FB
:10BE1000004004408C0E0020F0B4461EB3003344B2
:10BE200099002A4A0A445368D1680B449468641AFA
:10BE3000128AC2F30902944209D31446002706EB82
:10BE400086029500214A2A442144D1601EE0012740
:10BE5000F5E71D781E4A00F1140142F821505D7883
:10BE600042F821509D7842F82150DD7842F8215067
:10BE70001D7942F821505D7942F821509D7942F8B0
:10BE80002150DD7942F82150083C0833072CE0D8D6
:10BE900007E01D7800F114020D4941F82250013CE1
:10BEA0000133002CF5D1094BB100881982001046EE
:10BEB0001A44527CC2F3810203440132597C62F37A
:10BEC000830159743846F0BC704700BF8C0E0020C7
:10BED0000040044070B582B0441E04EB84039A0015
:10BEE000364B13445B7CC3F3810328B1032801D094
:10BEF000022202E0012200E001229A4254DDA20067
:10BF0000224495002D4B2B44DA689B689A4205D356
:10BF10002A4B2B445B7C13F0400F48D00E4605465D
:10BF2000274B9847FEB1274A0C3552F8253001932C
:10BF3000019B43F04F030193019B43F010030193D6
:10BF4000019B42F8253000238DF8033006E000BF46
:10BF50009DF803300133DBB28DF803309DF80330D8
:10BF6000DBB2132BF3D940B104EB84039A00134BDB
:10BF700013445A7C6FF386125A74A2002244910033
:10BF80000E4B0B44DA689B689A4212D30B4B0B445E
:10BF90005B7C13F0400F0ED1084B0B445A7C42F0EF
:10BFA00080025A74002000E0012002B070BD002021
:10BFB000FBE70120F9E70120F7E700BF8C0E002026
:10BFC00019BE4000004004402DE9F8430546844670
:10BFD000471EBB003B449A002A4C1444A268E36805
:10BFE000A2EB030EB4F81080C8F3090862681A4483
:10BFF0000C30254951F82060C6F30A4666B3B645B1
:10C000000BD9B6464FF0000907EB870188001D49A0
:10C0100001447344CB6000210AE04FF00109F3E7CB
:10C020000CF11403184850F8233013700131013219
:10C030008E45F5D82846154B9847B9F1000F01D128
:10C04000B04507D905F10C030F4A52F8233013F01D
:10C05000200F04D0BDE8F8834FF00009EAE7012380
:10C06000AB405361074ABB00D81981000846114410
:10C07000C968024491602A4600212046044B984733
:10C08000E8E700BF8C0E00200040044019BD4000CE
:10C0900089BC40002DE9F0418CB00124ADE120467F
:10C0A000B34B98470120FAE1BB003B449900B14AE9
:10C0B0000A44537CC3F38101033161F38303537456
:10C0C000537C13F0200F00F0848013F00C0F3BD052
:10C0D000A94A04F10C0152F821300193019B43F06D
:10C0E0004F030193019B43F010030193019B42F81E
:10C0F000213000238DF8013006E000BF9DF80130AB
:10C100000133DBB28DF801309DF80130DBB2132B27
:10C11000F3D9994A06F10C0152F821300293029B9F
:10C1200043F04F030293029B23F001030293029B0F
:10C1300042F8213006F10C038F4A52F8233013F0F5
:10C14000010FF7D10120AAE18B4A04F10C0152F84A
:10C1500021300393039B43F04F030393039B23F08E
:10C1600001030393039B42F8213006F10C03824A3A
:10C1700052F8233013F0010FF7D1114606F10C03EA
:10C1800052F823200492049A42F04F020492049A37
:10C1900042F020020492049A41F8232000238DF8F3
:10C1A000023006E000BF9DF802300133DBB28DF8AB
:10C1B00002309DF80230DBB2132BF3D907EB87076F
:10C1C000BA006C4B13445A7C6FF345125A74012029
:10C1D00065E113F0800F42D1BB003B449A00654BF0
:10C1E0001344DA689B689A424CD307EB87039A00A2
:10C1F000604B13445B7C13F04C0F43D1EFF310837F
:10C20000B3FA83F35B090B9372B6BFF35F8F00221F
:10C210005A4B1A700B9B584A55612BB10122574B50
:10C220001A70BFF35F8F62B6534A06F10C0152F8E1
:10C2300021300593059B43F04F030593059B23F0A5
:10C2400001030593059B42F8213006F10C034A4A8D
:10C2500052F8233013F0010FF7D101201FE1BB008A
:10C260003B449A00434B1344597C6FF3C7115974F4
:10C27000DA689A60404B5D61224600214046404B9F
:10C280009847A9E7002C4AD0032C48D007EB870336
:10C290009A00384B13445B7C13F00C0F3FD0364AA6
:10C2A00006F10C0152F821300693069B43F04F0330
:10C2B0000693069B43F010030693069B42F8213039
:10C2C00000238DF8033006E000BF9DF803300133F2
:10C2D000DBB28DF803309DF80330DBB2132BF3D9BA
:10C2E000254A06F10C0152F821300793079B43F0D1
:10C2F0004F030793079B23F001030793079B42F823
:10C30000213006F10C031C4A52F8233013F0010FC0
:10C31000F7D1002120461B4B98470120BFE0002C9D
:10C320004AD0032C48D001212046164B984758B3D9
:10C33000114A06F10C0152F821300893089B43F092
:10C340004F030893089B23F001030893089B42F8CE
:10C35000213006F10C03084A52F8233013F0010F84
:10C36000F7D100212046074B9847012097E000BFF6
:10C37000C9BF40008C0E0020004004402F03002065
:10C3800089BC4000D5BE40004749BB00D819820097
:10C390000A4492F811E06FF3C71E82F811E0D268E8
:10C3A0001F44BB0019448A60404B5D612246002156
:10C3B00040463F4B9847BBE7012120463D4B9847FD
:10C3C0003A4A06F10C0152F821300993099B43F0D7
:10C3D0004F030993099B23F001030993099B42F83A
:10C3E000213006F10C03314A52F8233013F0010FCB
:10C3F000F7D1012053E00134E4B2052C4ED82B4B89
:10C400009B6926460125A5402B42F4D0671E07EB09
:10C4100087029300244A02EB030804F10C03234A29
:10C4200052F8233013F0420F7FF439AE04F10C03BD
:10C430001E4A52F8233013F0010F7FF435AE04F199
:10C440000C031A4A52F8233013F0080FD3D004F12A
:10C450000C0152F821300A930A9B43F04F030A93D0
:10C460000A9B23F008030A930A9B42F8213006F145
:10C470000C030E4A52F8233013F0080FF7D106F1DF
:10C480000C0352F8233003F4E063B3F5807F09D046
:10C4900006F10C0352F82330012000E000200CB01C
:10C4A000BDE8F0810120FAE78C0E00200040044036
:10C4B00089BC4000D5BE400000B587B0534B1B7807
:10C4C000E3B9534B1B6BC3F30A43082B3BD0504AD1
:10C4D000136B0193019B43F04F030193019B23F0E6
:10C4E00004030193019B1363494B1B6B13F0040F6F
:10C4F000FAD1484B984707B05DF804FB464B984784
:10C50000464B9847DDE7424A116D454A995401333D
:10C51000DBB2072BF7D9434B9847B0B93C4A136BB2
:10C520000293029B43F04F030293029B23F0040308
:10C530000293029B1363364B1B6B13F0040FFAD16B
:10C54000344B9847D7E70023E3E7354B93F90030A6
:10C55000002B1EDB2E4A136B0593059B43F04F0304
:10C560000593059B23F004030593059B1363284B58
:10C570001B6B13F0040FFAD1294BDB88002B42D040
:10C580000023294A1380294A138001221F4B1A7065
:10C59000B1E71F4A136B0393039B43F04F030393CD
:10C5A000039B43F080030393039B136300238DF8E5
:10C5B000033006E000BF9DF803300133DBB28DF895
:10C5C00003309DF80330DBB2132BF3D9104A136B01
:10C5D0000493049B43F04F030493049B23F0040350
:10C5E0000493049B13630A4B1B6B13F0040FFAD1E3
:10C5F00000230D4A13800D4A13800222034B1A7048
:10C600000B4B984777E70B4B984774E78A0E00204F
:10C6100000400440FDB74000A9B84000E5B7400025
:10C62000702200203DB44000880E0020860E0020BD
:10C63000B9B840004DB84000204BDB6913F0010F42
:10C6400037D000B583B01D4B1B6B13F0040F24D102
:10C650001A4B1B6B13F0010F23D1184B1B6B13F0FC
:10C66000020F22D1154B1B6B13F0080F23D0134A76
:10C67000136B0193019B43F04F030193019B23F044
:10C6800008030193019B13630C4B1B6B13F0080F02
:10C69000FAD1012003B05DF804FB094B9847012053
:10C6A000F8E7084B98470120F4E7074B984701202B
:10C6B000F0E7002070470020ECE700BF0040044096
:10C6C000B9C44000B9B8400091BA400010B54C4B15
:10C6D000984720B94B4BDB6913F4807F10D0302092
:10C6E000494B9847474B9B6913F4006F04D0454B67
:10C6F000DB6913F4006F0AD1444B984770B110BD49
:10C7000072B6BFF35F8F0022414B1A7010BD4FF419
:10C7100000623C4B1A623F4B984710BD3E4B984716
:10C720000028ECD1374B9B6913F4005F04D0354BE4
:10C73000DB6913F4005F3DD1324B9B6913F4007F3A
:10C7400004D0304BDB6913F4007F33D12D4B9B6950
:10C7500013F4806F04D02B4BDB6913F4806F29D165
:10C76000284B9B6913F4807F04D0264BDB6913F4BC
:10C77000807F2FD1234BDB6913F4805FBFD0214C26
:10C780004FF480532362254B9847254B98476368A5
:10C7900023F001036360636823F002036360214BAD
:10C7A0009847214B98474FF4807323614FF40063FF
:10C7B0002361A4E7134C4FF41853236263610120F3
:10C7C0001A4B98474FF48073236223614FF4006340
:10C7D000236110BD0B4B4FF480721A625A614FF403
:10C7E00000521A614FF400721A614FF480621A61AC
:10C7F00030200F4B984700200C4B984710BD00BFCE
:10C800006DD840000040044035D7400039C6400094
:10C810002F03002005B4400095C04000C9BC400073
:10C8200019B2400031B74000E5B740008DB6400076
:10C8300089D7400010B582B0EFF31083B3FA83F3C9
:10C840005B09019372B6BFF35F8F0022144B1A701D
:10C85000019C0120134B98473020134B9847134BF2
:10C860005A6F22F480725A675A6F42F400725A6704
:10C870004FF480721A614FF400521A614FF4007243
:10C880001A614FF480621A614FF400621A612CB190
:10C890000122034B1A70BFF35F8F62B602B010BD66
:10C8A0002F0300208DB6400035D7400000400440E3
:10C8B00030B583B0EFF31083B3FA83F35B090093D1
:10C8C00072B6BFF35F8F0024204B1C70009D204B7D
:10C8D000984730201F4B98471F4B98471F4B5022BB
:10C8E00083F830234FF480325A601D4B98474FF441
:10C8F00080201C4B98471C4B1C701C4B1B78FF2B3B
:10C9000022D0EFF31083B3FA83F35B09019372B67D
:10C91000BFF35F8F00220D4B1A700199134A1378F1
:10C920000133137029B10122084B1A70BFF35F8FD6
:10C9300062B60F4B98472DB10122044B1A70BFF31A
:10C940005F8F62B603B030BDFEE700BF2F0300204B
:10C9500039D1400035D7400021D3400000E100E04C
:10C9600051BC400059D84000850E0020882200208C
:10C9700035C8400008B5064B5A6F42F480725A67BA
:10C980005A6F22F400725A670020024B984708BD84
:10C99000004004408DB6400010B582B0EFF3108324
:10C9A000B3FA83F35B09009372B6BFF35F8F002283
:10C9B000144B1A70009C144B9847144B1B7803B906
:10C9C000FEE7EFF31083B3FA83F35B09019372B6CA
:10C9D000BFF35F8F00220B4B1A7001990B4A13783B
:10C9E000013B137029B10122064B1A70BFF35F8F10
:10C9F00062B62CB10122034B1A70BFF35F8F62B68F
:10CA000002B010BD2F03002075C94000882200200D
:10CA10000D4B5A6822F001025A609A6822F4807223
:10CA20009A60024670B1986820F07F0002F07F02A1
:10CA3000104398609A6842F480729A605A6842F093
:10CA400001025A60704700BF00400440054B5B681C
:10CA500013F0010F04D0034B986800F07F0070477B
:10CA60000020704700400440014B98609981704756
:10CA700070220020F0B583B045B200F00F00052809
:10CA800073D801F00306044600F10C033B4F57F83E
:10CA9000233013F4004F6BD1012E53D0031FDBB2B0
:10CAA000012B54D94023934266DB461E06EB8607D2
:10CAB000334B03EB870303F11007B3F810E062F385
:10CAC000090EA3F810E05B7C03F07F036FF34513BE
:10CAD0007B70002D3EDB294EB36A01228240134356
:10CAE000B362264B9B6A1A42FBD0244B9E6A26EA0D
:10CAF00002029A6200F10C0253F822300193019B6A
:10CB000043F04F030193019B23F4074323F0800379
:10CB10000193002D23DB0A0202F4407242F400422A
:10CB2000019B1343019301990C30144B43F82010DF
:10CB300004F10C03114951F8233032EA0303F7D111
:10CB4000012013E0B0B10328A8D100200EE04FF47B
:10CB50000073A8E77B786FF383037B70BBE70A025F
:10CB600002F4407242F40442DAE7002003B0F0BD60
:10CB70000020FBE70020F9E70020F7E70040044031
:10CB80008C0E002000F00F03052B1ED810B582B0CC
:10CB900019460E4C0C3354F823200192019A42F0AE
:10CBA0004F020192019A22F400420192019A44F844
:10CBB000232001F10C03054A52F8233013F4004FEF
:10CBC000F7D1034B984702B010BD704700400440B6
:10CBD000F5BC400000F00F00431E052815D803EBFC
:10CBE00083039A000A4B13445B7C13F0200F08D197
:10CBF0000C30084B53F8203013F0280F03D00120DD
:10CC0000704701207047002070470020704700BF28
:10CC10008C0E00200040044010B485B044B200F0F7
:10CC20000F00052865D8421EEFF31083B3FA83F393
:10CC30005B09039372B6BFF35F8F0021314B19700C
:10CC40000399002C14DB304A00F10C0452F8243014
:10CC50000293029B43F04F030293029B43F0200395
:10CC60000293029B42F8243000238DF807302EE017
:10CC700000F10C03244C54F8233013F0100F09D1A9
:10CC800002EB82039C00214B23445B7CC3F38103B2
:10CC9000012BD8DD02EB820294001C4B23445A7C0A
:10CCA00042F020025A74012303FA00F0164B186177
:10CCB00021B30120134B1870BFF35F8F62B619E0E8
:10CCC00000BF9DF807300133DBB28DF807309DF8C7
:10CCD0000730DBB2132BF3D9012303FA00F00A4B20
:10CCE000186169B10120074B1870BFF35F8F62B6FE
:10CCF00000E0002005B05DF8044B70470120F9E723
:10CD00000120F7E72F030020004004408C0E002094
:10CD100000F00F0005286CD830B583B00246441EE1
:10CD200004EB84039900354B0B44597C6FF3451198
:10CD3000597400F10C03324951F8233013F0200FDD
:10CD400059D000F10C0551F825300093009B43F0B9
:10CD50004F030093009B23F020030093009B41F8B6
:10CD6000253002F10C03264951F8233013F0200F2F
:10CD7000F7D10D468B6A012181400B43AB62204BFA
:10CD80009B6A1942FBD01E4B9D6A25EA01019962FC
:10CD90000C3053F820100191019941F04F0101919D
:10CDA000019921F008010191019943F8201002F145
:10CDB0000C03134951F8233013F0080FF7D104EB9B
:10CDC00084039A000D4B13445B7C13F0100F01D1C8
:10CDD000012011E00949A200101983000B44587C7E
:10CDE0006FF3041058741444A300CB5898470120E3
:10CDF00002E000207047012003B030BD8C0E0020FF
:10CE000000400440F0B583B000F00F04052C00F2A0
:10CE1000A28047B2651E04F10C00554E56F8200062
:10CE200010F4004F00F09A8005EB8500514E06EBA0
:10CE30008000407C10F0200F40F0928004F10C0044
:10CE40004B4E56F8200010F0200F40F08B80EFF38F
:10CE50001080B0FA80F04009009072B6BFF35F8F87
:10CE6000002645480670DDF800E005EB8500414EE0
:10CE700006EB8000407C10F0100F0AD0BEF1000FCE
:10CE800072D001223C4B1A70BFF35F8F62B6002054
:10CE900062E005EB8500374E06EB8000467C46F0ED
:10CEA00010064674BEF1000F05D001263248067008
:10CEB000BFF35F8F62B6DFF8BCE005EB8500800052
:10CEC0000EEB00067260B3600022F260089A4EF822
:10CED000002011B95BBB012000E00120254AA90018
:10CEE0004B1902EB83035B7C60F386130D4402EB6A
:10CEF00085026FF3C7135374EFF31083B3FA83F310
:10CF00005B09019372B6BFF35F8F00221A4B1A7050
:10CF1000019D0123A340164A1361002F09DB2DB3A5
:10CF20000120154B1870BFF35F8F62B614E000202C
:10CF3000D4E704F10C0352F8233013F0110FEED1B3
:10CF4000012120460D4B98470028E8D000212046BB
:10CF50000A4B9847E3E7002003B0F0BD0020FBE751
:10CF60000020F9E70020F7E70020F5E70120F3E7CC
:10CF7000004004408C0E00202F030020D5BE40004E
:10CF800070B586B000F00F04052C00F2C98042B2E3
:10CF9000EFF31083B3FA83F35B09059372B6BFF323
:10CFA0005F8F00215F4B1970059B26460125A54028
:10CFB0005D494D612BB101215A4B1970BFF35F8F51
:10CFC00062B6002A80F2948004F10C03564A52F8AB
:10CFD000233013F0100F64D0002C49D0032C47D01D
:10CFE00004F10C0152F821300193019B43F04F03EF
:10CFF0000193019B23F010030193019B42F8213020
:10D0000006F10C03484A52F8233013F0100FF7D101
:10D0100006F10C03444A52F8233013F0100FF7D1F5
:10D0200004F10C0152F821300293029B43F04F03AC
:10D030000293029B43F010030293029B42F82130BB
:10D0400000238DF8033006E000BF9DF80330013364
:10D05000DBB28DF803309DF80330DBB2132BF3D92C
:10D0600006F10C03304A52F8233013F0100FF7D0BA
:10D070002D4A04F10C0152F821300393039B43F035
:10D080004F030393039B23F010030393039B42F886
:10D09000213006F10C03244A52F8233013F0100F0C
:10D0A000F7D1214A04F10C0152F821300493049B7A
:10D0B00043F04F030493049B23F001030493049B68
:10D0C00042F8213006F10C03174A52F8233013F0CE
:10D0D000010FF7D1621E02EB82029100134B0B4449
:10D0E0005A7C6FF383025A740AE02046104B98472B
:10D0F00006F10C030C4A52F8233013F0420FF4D11E
:10D10000094A936A2B439362074B9B6A1D42FBD0EB
:10D11000054A936A23EA050595622046054B984720
:10D1200006B070BD2F030020004004408C0E00208C
:10D1300019BD4000F5BC4000064BD3F8142122F481
:10D140004062C3F81421D3F8202142F00102C3F851
:10D150002021704700020E400B4619B1096801609A
:10D160005B6843601AB11368036153684361704799
:10D1700021F0FE01C905C90D0162704710B51E4BB3
:10D1800053F820402268536A13F0805F11D00223C5
:10D19000C2F8203123684FF0FF32DA610023237593
:10D1A000236913F0010F26D0636823B32046984704
:10D1B00010BD13F0006F13D00223C2F82031236892
:10D1C0004FF00062DA61236913F0020F03D0A36805
:10D1D0000BB12046984723680122C3F8202110BDD7
:10D1E00013F0007F07D0236913F0040F03D0E36826
:10D1F0000BB12046984710BDF00E002008B5002066
:10D20000014B984708BD00BF7DD1400008B5012003
:10D21000014B984708BD00BF7DD1400070B5054661
:10D220000E461446016001230B60214B99422BD01E
:10D230000D20204B9847204B1D6023781B0203F4E0
:10D24000FE43736063782BBB0022A3780BB142F0DE
:10D250000402E3780BB142F0080223790BB142F0EB
:10D26000100263791B0203F47063A179090389B288
:10D270000B431343B3652389C3F30E03628943EA67
:10D280000243F36500230CE012200A4B98470A4B37
:10D290005D60D2E70222D8E705EB830200215160EE
:10D2A0000133022BF8D900202861287570BD00BF1A
:10D2B0000000034035D74000F00E002012F0100FA0
:10D2C00012D0C0F8B01012F0200F07D0C0F8D41060
:10D2D00012F0400F05D0C0F8C0107047C0F8D01051
:10D2E000F6E7C0F8C4107047C0F8B4107047016486
:10D2F000704741647047C06C7047806C704740094C
:10D3000000F5001000F207704002704740090B3032
:10D31000704700F01F00012303FA00F0704700007F
:10D3200008B500200A4B98470A4B98470028FBD0C5
:10D33000094B9847094A0A4BDA620A4B984700287A
:10D34000FBD00020084B9847084B984708BD00BF0A
:10D35000B1D64000D5D6400019D74000013FB805EE
:10D3600000040E4025D7400039D840004DD8400079
:10D3700010B5A2B01848194B98470020184B984791
:10D38000184B98470028FBD0174B9847174A184B63
:10D390009A62184B98470028FBD00020164B9847FC
:10D3A000164B984716480D4B9847164B1A68164B64
:10D3B0001344164A934201D922B010BD2023009392
:10D3C00002AB0F220E211248124CA047BDF84810A4
:10D3D0001148124B9847EFE7000E2707BDDB4000CE
:10D3E000B1D64000D5D64000FDD64000013FB70B76
:10D3F00000040E4009D740005DD64000C9DA400065
:10D400000000DC0530030020C0D3BDF980C3C90192
:10D41000000A0E401100002010140E407DD840007C
:10D4200070B50D461446064658B14FF0FF360AE077
:10D43000064B1868064B1B6829469847013501368C
:10D44000013C002CF4DC304670BD00BF9822002067
:10D450009022002070B5013802280FD8144600250C
:10D460008CB10A4B18684E1C094B1B680978984709
:10D47000002806DB0135013C3146F1E74FF0FF356E
:10D4800001E04FF0FF35284670BD00BF9822002014
:10D4900094220020A1F10E03012B02D84FF0FF309F
:10D4A000704710B582B0EFF31083B3FA83F35B09D2
:10D4B000019372B6BFF35F8F00240B4B1C70019C6D
:10D4C000120222F07F4222F0FF02C9B2114341F062
:10D4D000B441064B98472CB10122034B1A70BFF39D
:10D4E0005F8F62B602B010BD2F03002079000020CC
:10D4F0004C4B1B78FF2B31D000B583B0EFF310837A
:10D50000B3FA83F35B09019372B6BFF35F8F002216
:10D51000454B1A700199434A13780133137029B1AE
:10D520000122414B1A70BFF35F8F62B63F4A9042AF
:10D5300015D03F4A904220D03E4A90422BD03E4ADE
:10D54000904236D03D4A904241D03D4A90424CD024
:10D550003C4A904257D003B05DF804FBFEE716202A
:10D56000394B98470720394B984700210720384B03
:10D5700098470720374B9847EDE71520324B9847DF
:10D580000720324B984700210720314B984707204E
:10D59000304B9847DFE714202B4B984707202B4B45
:10D5A0009847002107202A4B98470720294B984786
:10D5B000D1E71320244B98470620244B984700219D
:10D5C0000620234B98470620224B9847C3E70E209E
:10D5D0001D4B984706201D4B9847002106201C4BE9
:10D5E000984706201B4B9847B5E70920164B9847EC
:10D5F0000620164B984700210620154B9847062019
:10D60000144B9847A7E708200F4B984706200F4B6D
:10D610009847002106200E4B984706200D4B98474F
:10D6200099E700BF882200202F030020000004405B
:10D630000080004000C001400080014000400240E6
:10D640000000024000C0004035D7400025D840000F
:10D65000DDD7400011D8400001607047134A136BBA
:10D6600023F07003184310634FF400630F4A926E67
:10D6700012F0080F02D1A3B1013BF7E70B4A136B7D
:10D6800023F0030343F0020313634FF40063074ADC
:10D69000926E12F0080F02D12BB1013BF7E7002088
:10D6A0007047012070470120704700BF00040E4002
:10D6B000012803D0054A064B1A607047044A936854
:10D6C00043F0254343F480139360F3E7080000A57B
:10D6D00010140E40074B5B6913F0800F06D0064B09
:10D6E0009B6E13F0800F03D100207047002070471D
:10D6F0000120704710140E4000040E400022014B20
:10D700009A62704700040E40024B986E00F00200CF
:10D71000704700BF00040E400022014BDA627047E0
:10D7200000040E40024B986E00F00400704700BFEA
:10D7300000040E4032281ED81F280CD8114B9A69BD
:10D7400001238340934318D0012303FA00F00D4BCB
:10D7500018610020704720380A4BD3F808210123B4
:10D76000834093430BD0012303FA00F0054BC3F829
:10D770000001002070470120704700207047002002
:10D78000704700BF00040E40322822D81F280ED850
:10D79000114B9A6901238340934301D000207047C5
:10D7A000012303FA00F00C4B586100207047203829
:10D7B000094BD3F8082101238340934301D0002073
:10D7C0007047012303FA00F0034BC3F80401002063
:10D7D00070470120704700BF00040E4041F0040173
:10D7E00000F11002094B43F822104FF40062074B7E
:10D7F000996E4FF480738340194202D11AB1013AF5
:10D80000F5E7002070470120704700BF00040E407C
:10D810004FF4807303FA00F0014B1860704700BFAB
:10D8200000040E404FF4807303FA00F0014B58607F
:10D83000704700BF00040E40000200F4706040F02A
:10D840000100014B9863704700040E408022014B99
:10D850001A60704700040E40C0F31200024B1A6FAA
:10D8600010431867704700BF00040E40024B187841
:10D8700080F00100704700BFF80E0020C36923F458
:10D88000F053490201F4F051194341F0B44141F41D
:10D890008071C161704730B4B2EB011F17D31024FF
:10D8A00001FB04F14B0803EBC202B2FBF1F2D30817
:10D8B0005D1E4FF6FE718D4210D8082C09D012045F
:10D8C00002F4E0221A430262002030BC70470824B0
:10D8D000E6E7416841F400214160F0E70120F4E708
:10D8E0004023036070478823036070471023036060
:10D8F00070472423036070474FF4807303607047C0
:10D900004FF4002303607047436913F0020F04D003
:10D91000C1F30801C16100207047012070474369CD
:10D9200013F0020FFBD0C1F30801C1610020704762
:10D93000436913F0010F05D08369C3F308030B603B
:10D940000020704701207047014BC0F8E430704759
:10D950000041535510B50446094B984700236360B6
:10D960006362A3622046074B98472046064B9847C0
:10D970002046064B98472046054B984710BD00BFF0
:10D9800049D94000E7D84000F3D84000F9D840001A
:10D9900001D9400070B505460C461646104B984715
:10D9A0000022104B1A60B4B13246216828460E4B53
:10D9B0009847024688B96368A1680B4321690B4305
:10D9C000E1680B430749086803430B6069680B4330
:10D9D0006B60104670BD0122FBE70122F9E700BF32
:10D9E00055D94000FC0E002097D8400000B583B008
:10D9F000234B244A9A4209D0214B224A03E0116862
:10DA000019600433043220498B42F8D31F4B02E0E3
:10DA100000221A6004331E4A9342F9D31D4A22F0B1
:10DA20007F011D4B9960EFF31083B3FA83F35B0919
:10DA3000019372B6BFF35F8F0021184B19700198E4
:10DA400017490B6843F470030B60BFF34F8FBFF3AC
:10DA50006F8F28B10121114B1970BFF35F8F62B630
:10DA600002F16042B2F5203F04D20B4A936843F0C2
:10DA7000005393600B4B98470B4B9847FEE700BF52
:10DA800010000020F84A4100E80C0020E80C0020BB
:10DA90007C2300200040400000ED00E02F03002028
:10DAA00088ED00E0A50D41004DFD400008B50120C6
:10DAB000034B9847EFF30580024B9847FFDE00BF0A
:10DAC000214D40002D4D4000344B1B6B03F00303F0
:10DAD000012B20D083B1022B39D0304B1B6B03F0CC
:10DAE0007003702B51D02D4B1A6BC2F302122C49CC
:10DAF0000B68D3400B6070472A4B5B6913F0800FB3
:10DB000004D04FF40042264B1A60E6E74FF4FA4285
:10DB1000234B1A60E1E7214B1B6A13F0807F03D08F
:10DB2000214A1F4B1A60D8E7204A1D4B1A601B4B35
:10DB30001B6A03F07003102B05D0202BCDD11C4A9B
:10DB4000174B1A60C9E71B4A154B1A60C5E7154BFE
:10DB50005B6913F0800F13D04FF40042104B1A6032
:10DB60000E4B1B6B03F00303022BB6D10B4B9A6ACF
:10DB7000C2F30C420A490B6802FB03330B60ACE7AB
:10DB80004FF4FA42064B1A60EAE7054A13680A495D
:10DB9000A1FB03135B081360704700BF00040E4035
:10DBA0003003002010140E40001BB70000127A0052
:10DBB00000366E010024F400ABAAAAAA144B9842C6
:10DBC0000FD9144B984211D9134B984212D9134BC9
:10DBD000984213D9124B984214D9124A124B1A6028
:10DBE00070474FF08062104B1A6070470F4A0E4B1F
:10DBF0001A6070470E4A0C4B1A6070470D4A0A4B68
:10DC00001A6070474FF00422074B1A60704700BF3C
:10DC1000FF2C3101FF596202FF869303FFB3C40456
:10DC2000FFE0F50500050004000A0E4000010004B5
:10DC300000020004000300040A4B1B6853B1094BA7
:10DC40001B681A180849914208DB1046054A106003
:10DC500018467047054A034B1A60F0E74FF0FF3053
:10DC6000704700BF000F0020FC7F0220805300207F
:10DC70004FF0FF3070474FF400534B600020704767
:10DC8000012070470020704700F1080343604FF007
:10DC9000FF328260C360036100230360704700238A
:10DCA0000361704743684B609A688A609A68516064
:10DCB00099600861036801330360704730B40D68F0
:10DCC000B5F1FF3F02D000F1080202E0026904E072
:10DCD0001A4653681C68A542FAD253684B60996093
:10DCE0008A605160086103680133036030BC70478B
:10DCF00003694268816891608268416851605A682E
:10DD0000904206D0002202611A68013A1A6018682F
:10DD1000704782685A60F5E782B0002301934FF0A4
:10DD2000500383F31188BFF36F8FBFF34F8F019BB5
:10DD3000002BFCD002B0704708480068006880F3F0
:10DD400008884FF0000080F3148862B661B6BFF314
:10DD50004F8FBFF36F8F00DF00BF000008ED00E0C2
:10DD6000DFF80C00016841F47001016070470000A9
:10DD700088ED00E04FF0807340F8043C21F0010191
:10DD800040F8081C054B40F80C3C40F8202C6FF084
:10DD9000020340F8243C4438704700BF19DD4000BE
:10DDA000074B19680868B0E8F04F80F30988BFF3A3
:10DDB0006F8F4FF0000080F311887047AFF3008041
:10DDC000040F00204FF0500383F31188BFF36F8FCF
:10DDD000BFF34F8F024A136801331360704700BFCF
:10DDE00034030020034A1368013B13600BB983F32B
:10DDF000118870473403002000000000000000007C
:10DE0000EFF30980BFF36F8F154B1A681EF0100FE8
:10DE100008BF20ED108A20E9F04F10602DE90900BD
:10DE20004FF0500080F31188BFF34F8FBFF36F8F17
:10DE300000F07CFF4FF0000080F3118809BC1968E6
:10DE40000868B0E8F04F1EF0100F08BFB0EC108A61
:10DE500080F30988BFF36F8F704700BFAFF3008076
:10DE6000040F002008B54FF0500383F31188BFF36F
:10DE70006F8FBFF34F8F054B984718B14FF080520B
:10DE8000034B1A60002383F3118808BDA9EA400000
:10DE900004ED00E0054B00221A6005490A600549BF
:10DEA000054A116007221A60704700BF10E000E0C9
:10DEB00018E000E0FF7F010014E000E010B50E4B19
:10DEC0001A6842F470021A601A6842F070421A60CE
:10DED0000A4B984700240A4B1C600A4B98470A4A91
:10DEE000136843F040431360084B9847084B98472A
:10DEF000084B9847204610BD20ED00E095DE40001D
:10DF00003403002061DD400034EF00E039DD4000E3
:10DF10002DED400019DD400010B50446044B984734
:10DF20002046044B98470446034B9847204610BDB3
:10DF30008DEA40001D0E41009DEB400048B110B538
:10DF40000446044B98472046034B9847034B984799
:10DF500010BD70478DEA40002D0E41009DEB400042
:10DF6000436A23B1036B1868C0F1050070470020B5
:10DF70007047000010B50446064B9847A26BE36B50
:10DF80009A4204D00024044B9847204610BD012437
:10DF9000F9E700BFC5DD4000E5DD400010B50446EF
:10DFA000054B9847A36B23B10024044B98472046A8
:10DFB00010BD0124F9E700BFC5DD4000E5DD4000EC
:10DFC00070B504461646856B026C5AB903681BB1DE
:10DFD00000200135A56370BD4068174B98470023AA
:10DFE0006360F6E76EB98068144B9847226CA368AB
:10DFF0001344A3606268934219D32368A36000208E
:10E00000E7E7C0680D4B9847226C5242E36813441F
:10E01000E36021688B4202D263681A44E260022EF8
:10E0200001D00020D5E725B1013D0020D1E7002037
:10E03000CFE70020CDE700BF3DF04000A114410034
:10E04000026C72B110B5C3681344C3604468A34244
:10E0500001D30368C3600C46C1682046014B984752
:10E0600010BD7047A114410038B505461A4B9847BA
:10E0700095F8454064B201E0013C64B2002C0ADD31
:10E080006B6A43B105F12400144B98470028F3D084
:10E09000134B9847F0E7FF2385F84530114B98471D
:10E0A0000D4B984795F8444064B201E0013C64B2DE
:10E0B000002C0ADD2B6943B105F11000074B98478E
:10E0C0000028F3D0064B9847F0E7FF2385F844304B
:10E0D000044B984738BD00BFC5DD400031EE40001D
:10E0E0002DEF4000E5DD400038B504460D46144BE9
:10E0F00098472168E26B236C03FB021060600020EC
:10E10000A063A160013A02FB0313E360FF2384F8DC
:10E11000443084F8453055B923691BB9094B9847F9
:10E12000012038BD04F11000074B9847F6E704F1D1
:10E130001000064DA84704F12400A847EEE700BFF1
:10E14000C5DD4000E5DD400031EE400089DC4000E7
:10E1500038B51D46049C0B4649B12260E063236438
:10E1600001212046034B984784F84C5038BD246069
:10E17000F4E700BFE9E04000F0B583B0054617467C
:10E180000E4689B100FB01F05030084B9847044619
:10E1900038B100903B4600F1500231462846044D0C
:10E1A000A847204603B0F0BD0020EDE719DF40008E
:10E1B00051E14000F0B585B004460F4601921E467D
:10E1C000002526E0324639462046354B9847636A9B
:10E1D00023B9344B9847012005B0F0BD04F1240069
:10E1E000314B9847F5E72F4B98470020F4E702A8FA
:10E1F0002E4B9847012519E0002384F8443021E094
:10E20000002384F8453023E02046294B9847294BCA
:10E210009847294B9847A26BE36B9A42D2D3022EC0
:10E22000D0D0019B002BDED0002DE0D01D4B9847B5
:10E23000224B9847204B984794F844305BB2B3F197
:10E24000FF3FD9D094F845305BB2B3F1FF3FD7D050
:10E25000144B984701A902A8194B9847C8B9204602
:10E26000184B98470028CFD0019904F11000164BA5
:10E27000984720460E4B98470E4B98470028C8D128
:10E280004FF08052114B1A60BFF34F8FBFF36F8F67
:10E29000BFE72046064B9847064B984700209BE770
:10E2A000C1DF4000E5DD400031EE4000B1EE40004E
:10E2B00069E040009DEB4000C5DD40008DEA400074
:10E2C000C9EE400075DF4000E1ED400004ED00E0E4
:10E2D00048B110B5002141600160C1600B460A469B
:10E2E000014CA04710BD7047B5E1400010B5024693
:10E2F00000210120034B98470446034B98472046D2
:10E3000010BD00BF79E14000D1E24000F8B5EFF365
:10E3100011864FF0500484F31188BFF36F8FBFF361
:10E320004F8F856BC46BA54205D3022B03D0002011
:10E3300086F31188F8BD1746054690F8454064B24B
:10E340001A460E4B9847B4F1FF3F05D0013464B232
:10E3500085F845400120EBE76B6A0BB90120E7E740
:10E3600005F12400064B984718B127B10120386009
:10E37000DEE70120DCE70120DAE700BFC1DF400073
:10E3800031EE4000F0B585B004460F4601920026FC
:10E3900032E039462046384B9847013DA563236952
:10E3A00023B9364B9847012005B0F0BD04F11000A9
:10E3B000334B9847F5E7314B98470020F4E702A824
:10E3C000304B9847012621E0002384F8443029E0AF
:10E3D000002384F845302BE020462B4B98472B4BED
:10E3E000984709E02046284B9847284B98472046F5
:10E3F000274B984700283DD1264B9847A56B002D09
:10E40000C7D1019B002BD6D0002ED8D01B4B9847EC
:10E41000214B98471F4B984794F844305BB2B3F1B7
:10E42000FF3FD1D094F845305BB2B3F1FF3FCFD07E
:10E43000124B984701A902A8184B98470028D1D140
:10E440002046134B98470028C6D0019904F12400B8
:10E45000134B984720460C4B98470C4B9847002885
:10E46000CAD14FF080520F4B1A60BFF34F8FBFF3EA
:10E470006F8FC1E7002097E741E04000E5DD4000F5
:10E4800031EE4000B1EE400069E040009DEB4000FD
:10E490009DDF4000C5DD40008DEA4000C9EE400030
:10E4A000E1ED400004ED00E070B584B00446019158
:10E4B000002635463EE0013BA36323683BB1236958
:10E4C0004BB9444B98470126304604B070BD424BCF
:10E4D00098476060F3E704F11000404B9847F0E77D
:10E4E0003C4B98470026EFE702A83D4B9847012593
:10E4F0002AE0002384F8443032E0002384F84530D9
:10E5000034E0384B98476068374B98470646314BA4
:10E5100098473BE02046354B9847354B984709E0F4
:10E520002046324B9847324B98472046314B98470C
:10E53000002840D12B4B9847A36B002BBBD1019BEC
:10E54000002BCDD0002DCFD0224B98472A4B984797
:10E55000244B984794F844305BB2B3F1FF3FC8D0E6
:10E5600094F845305BB2B3F1FF3FC6D0194B9847E2
:10E5700001A902A8214B98470028D1D120461D4B64
:10E5800098470028C6D02368002BBAD0019904F11F
:10E5900024001B4B98472046144B9847144B984730
:10E5A0000028C7D14FF08052164B1A60BFF34F8F2F
:10E5B000BFF36F8FBEE7002E86D00A4B98472046E8
:10E5C000114B984701466068104B9847014B98479C
:10E5D000002679E7E5DD400065F1400031EE4000BE
:10E5E000B1EE4000C5DD400075EF400069E040003D
:10E5F0009DEB40009DDF40008DEA4000C9EE4000E9
:10E60000E1ED400004ED00E061DF4000C5F04000B6
:10E610000023092B0CD8074A52F833200AB10133E2
:10E62000F7E7044A42F8331002EBC303586070471F
:10E63000704700BF9C22002070B504460D46164668
:10E64000124B984794F844305BB2B3F1FF3F0DD0C2
:10E6500094F845305BB2B3F1FF3F0BD00C4B9847B9
:10E66000A36B5BB120460B4B984770BD002384F829
:10E670004430EDE7002384F84530EFE73246294681
:10E6800004F12400044B9847ECE700BFC5DD4000CF
:10E69000E5DD400069E0400005EE4000F0B50368AC
:10E6A0004BB343685B68436000F10807BB4204D08A
:10E6B0004368D3F80CE0002609E05B684360F7E7A5
:10E6C0005B68436008E02E46B6B9AE4514D0436897
:10E6D0005B6843609F42F3D04368DD6800230F2BE3
:10E6E000F2D8EA1892F83420CC5CA242ECD1002A8D
:10E6F000E9D00133F3E700263046F0BD002301E006
:10E70000013001330278A52AFAD0C3F38F00704795
:10E710000A4B1B681B684BB901234BB9074B1B689D
:10E72000DB68DB685A68064B1A6070470023F4E721
:10E730004FF0FF32024B1A60704700BF080F0020F5
:10E74000B40F00202DE9F84F81460D4617469A4632
:10E750000A9EDDF82C800C9C9200A521206B1D4B9D
:10E760009847236B07F18042013A03EB820727F0B9
:10E77000070700230F2B07D8E95CE21882F8341052
:10E78000EA5C0AB10133F5E7002384F84330042E34
:10E7900000D90426E662E66400252565201DDFF821
:10E7A0003CB0D84704F11800D8472461C6F10506EB
:10E7B000A6616462656584F85850524649463846F9
:10E7C000054B98472060B8F1000F01D0C8F8004011
:10E7D000BDE8F88F9D16410075DD40009FDC4000CC
:10E7E00070B5002407E004EB840293000B48184442
:10E7F0000B4B98470134042CF5D90A4E3046084C8F
:10E80000A047094D2846A0470848A0470848A04708
:10E81000084B1E60084B1D6070BD00BF100F00202C
:10E8200089DC4000880F00209C0F0020BC0F0020D6
:10E83000D40F0020080F00200C0F002010B5044654
:10E840001C4B98471C4A1368013313601B4B1B6811
:10E85000002B26D01A4B1B683BB9184B1B68DA6A91
:10E86000E36A9A4201D8154B1C60164A13680133BB
:10E8700013606364E36A01229A4013490868024303
:10E880000A6003EB83039A00211D10481044104BCB
:10E890009847104B98470A4B1B680BB1074B1B68F6
:10E8A00010BD064B1C601368012BDED10A4B984744
:10E8B000DBE700BFC5DD4000740F0020040F00201F
:10E8C000D00F0020800F0020840F0020100F0020A8
:10E8D000A5DC4000E5DD4000E1E7400070B50446FE
:10E8E0000E461D4B1D681D4B186804301C4B984785
:10E8F00050B91A4B1B68DA6A012303FA02F219496C
:10E900000B6823EA02030B60B4F1FF3F13D02C44E1
:10E91000124B1B685C60A54216D8134B18680F4B4E
:10E9200019680431114B9847114B1B689C4201D266
:10E930000F4B1C6070BD002EE9D0084B19680431E4
:10E940000C480D4B984770BD0C4B1868034B196869
:10E950000431064B984770BDE80F0020040F0020DB
:10E96000F1DC4000840F0020080F0020BDDC4000D7
:10E97000B40F0020D40F0020A5DC40000C0F0020B5
:10E9800008B54FF08052044B1A60BFF34F8FBFF3AE
:10E990006F8F024B9847F4E704ED00E085FC4000E0
:10E9A0002DE9F04385B006460F461546984690007F
:10E9B000144B984700B381465C20124B984704469D
:10E9C000B0B1C0F83090CCB10023039302940D9BFA
:10E9D00001930C9B009343462A46394630460A4D24
:10E9E000A8472046094B9847012005B0BDE8F083B1
:10E9F0004846074B9847E6E70024E4E74FF0FF302E
:10EA0000F3E700BF19DF400045E740003DE8400064
:10EA10003DDF400010B582B0134B019300230093FB
:10EA2000462212491248134CA047012803D001285E
:10EA300004D002B010BD104B9847F8E74FF05003D8
:10EA400083F31188BFF36F8FBFF34F8F4FF0FF3207
:10EA50000A4B1A6001220A4B1A600022094B1A6005
:10EA6000094B9847E5E700BFB00F00206848410018
:10EA700081E94000A1E94000F9F54000B40F002011
:10EA8000D00F0020E80F0020BDDE4000024A1368CE
:10EA900001331360704700BF7C0F0020014B1868E2
:10EAA000704700BFE80F002070B52F4B1B68002B8C
:10EAB00052D12E4B1E6801361E604EB12C4B1B6886
:10EAC0009E422FD22B4B1B68002B42D0002070BDE2
:10EAD000294A1168294B186810601960284A136880
:10EAE00001331360274B9847E8E7012320E04FF0FC
:10EAF000FF321F4B1A60E5E71D4A1360E2E704F19D
:10EB00001800214B9847E36A01229A401F49086880
:10EB100002430A6003EB83039A0029461C48104411
:10EB20001C4B9847144B1B681B68002BDDD000233F
:10EB3000002BDCD1104B1B68DB68DC6863689E42ED
:10EB4000DAD3251D2846104B9847A36A002BD6D14F
:10EB5000D9E7114B9847B9E7064A136801331360A8
:10EB60000D4B9847B2E700BF7C0F0020E80F002054
:10EB7000B40F0020780F0020080F00200C0F002099
:10EB8000B80F002011E74000F1DC4000840F0020A6
:10EB9000100F0020A5DC400049FD400070B5274B58
:10EBA0009847274B1A68013A1A601B68002B32D12C
:10EBB000244B1B68002B2ED00024234B1B6813B35F
:10EBC000214BDB68DC6804F11800204EB047251D9E
:10EBD0002846B047E36A01229A401D49086802436B
:10EBE0000A6003EB83039A0029461A4810441A4B23
:10EBF0009847E26A194B1B68DB6A9A42DDD301220F
:10EC0000174B1A60D9E70CB1164B9847164B1C6886
:10EC10003CB9134B1B68154B9847002070BD013C55
:10EC200007D0134B98470028F9D001220C4B1A60EB
:10EC3000F5E700220C4B1A60EBE700BFC5DD400092
:10EC40007C0F0020740F0020BC0F0020F1DC40007E
:10EC5000840F0020100F0020A5DC4000040F0020CE
:10EC6000EC0F002011E74000780F0020E5DD4000A8
:10EC7000A9EA400010B550B9002038B94FF08052D1
:10EC8000084B1A60BFF34F8FBFF36F8F10BD044660
:10EC9000054B984700212046044B9847044B984762
:10ECA000EBE700BF04ED00E08DEA4000DDE8400046
:10ECB0009DEB400070B50646154B98470524013C76
:10ECC00004EB84029300314612481844124B9847D3
:10ECD000054608B9002CF2D12DB15DB18DB10F4BB5
:10ECE0009847284670BD0E4B186831460A4B984726
:10ECF0000546F2E70B4B18683146074B9847054627
:10ED0000ECE731460848044B98470546E7E700BF63
:10ED10008DEA4000100F00209DE640009DEB400072
:10ED2000080F00200C0F0020D40F0020264B1B687A
:10ED3000002B2FD110B50022244B1A60244B1B68E6
:10ED40001B6B1A68B2F1A53F28D0214B18681968CF
:10ED50003431204B9847204B1B68B3FA83F3DBB266
:10ED6000C3F11F031D489A00D418A10001444C6848
:10ED700064684C601A4491000831084484421AD0F7
:10ED800003EB83039A00154B13445B68DA68104B5E
:10ED90001A6010BD01220D4B1A6070475A68B2F11B
:10EDA000A53FD2D19A68B2F1A53FCED1DB68B3F1CD
:10EDB000A53FCAD1CFE7606803EB83029100074A01
:10EDC0000A445060DCE700BF7C0F0020EC0F0020FD
:10EDD000040F002049FC4000840F0020100F002089
:10EDE00010B50C46044B19681831044B98470121A3
:10EDF0002046034B984710BD040F0020BDDC4000A7
:10EE0000DDE8400038B50D461446064B1968183148
:10EE1000054B98470CB14FF0FF3521462846034B70
:10EE2000984738BD040F0020A5DC4000DDE8400015
:10EE300038B5C368DC6804F118052846144B9847B8
:10EE4000144B1B68E3B9251D2846114B9847E36A0C
:10EE500001229A401049086802430A6003EB8303C9
:10EE60009A0029460D4810440D4B9847E26A0D4B15
:10EE70001B68DB6A9A4208D901200B4B186038BD29
:10EE800029460A48064B9847F0E7002038BD00BFE6
:10EE9000F1DC40007C0F0020840F0020100F0020C8
:10EEA000A5DC4000040F0020EC0F0020BC0F002068
:10EEB000034B1B680360034B1B684360704700BF34
:10EEC000B80F0020E80F0020F8B504460D46124B9D
:10EED0009847124B19686268881A2B68B3F1FF3F94
:10EEE00016D027680E4E3668B74201D0914211D233
:10EEF000984206D300232B6001240A4B98472046F2
:10EF0000F8BD1B1A2B602046074B98470024F4E7F6
:10EF10000024F2E70124F0E7C5DD4000E80F0020FF
:10EF2000B80F0020E5DD4000B1EE40000122014BAA
:10EF30001A607047EC0F002008B5034618B1186B33
:10EF4000024B984708BD024B1B68F8E7FDE64000FE
:10EF5000040F0020054B1B6823B1054B1B681BB930
:10EF6000022070470120704700207047D00F00201A
:10EF70007C0F0020002854D038B50446C26A2A49C4
:10EF80000968C96A8A4242D28169002905DB26499B
:10EF90000968C96AC1F105018161606902EB8202F9
:10EFA0009100224A0A44904207D000223AB91E4AF0
:10EFB0001268D26AE262012038BD0122F6E7251DFF
:10EFC00028461B4B984768B9E36A03EB83018A0024
:10EFD00016498A5832B901229A4016490B6823EA29
:10EFE00002030B60104B1B68DB6AE362012404FA26
:10EFF00003F21049086802430A6003EB83039A0096
:10F0000029460A4810440C4B9847204638BDC26C2C
:10F01000054B1B68DB6A9A4201D2012038BD0020F3
:10F0200038BD0020704700BF040F0020100F0020E3
:10F03000F1DC4000840F0020A5DC4000002834D023
:10F0400038B50446026D013A0265C06AE16C884237
:10F050002DD00AB1002038BD251D2846154B9847F4
:10F0600068B9E36A03EB83018A0013498A5832B90D
:10F0700001229A4011490B6823EA02030B60E36CFA
:10F08000E362C3F10502A261012404FA03F20B4911
:10F09000086802430A6003EB83039A002946064886
:10F0A0001044074B9847204638BD00207047002089
:10F0B00038BD00BFF1DC4000100F0020840F00209D
:10F0C000A5DC4000002843D038B50446C26C8A4213
:10F0D00000D20A46E16A8A4202D0206D012800D09F
:10F0E00038BDE262A069002802DBC2F10502A2611C
:10F0F000636901EB81018800164A0244934225D0DE
:10F100000022002AECD0251D2846134B984768B9E9
:10F11000E36A03EB83018A000E498A5832B901225F
:10F120009A400E490B6823EA02030B60E36A01224E
:10F130009A400A49086802430A6003EB83039A0075
:10F14000294604481044064B9847C9E70122D8E7EE
:10F15000704700BF100F0020F1DC4000840F00203A
:10F16000A5DC4000054B1B6823B1044B1A68136DE6
:10F1700001331365014B1868704700BF040F00206E
:10F1800038B505460C461A4B98471A4B1B685B6D01
:10F190002BB9184B1B68012283F85820ACB9164BC9
:10F1A0009847134B9847134B1B685C6D24B1CDB93E
:10F1B000104B1B68621E5A650E4B1B68002283F8B9
:10F1C00058200D4B9847204638BD114620460B4B22
:10F1D00098474FF080520A4B1A60BFF34F8FBFF32E
:10F1E0006F8FDCE7034B1B6800225A65E4E700BF22
:10F1F000C5DD4000040F0020E5DD4000DDE84000F3
:10F2000004ED00E0F8B507460D4614461E46214BB6
:10F210009847214B1B6893F85830DBB2022B0AD079
:10F220001D4B1A68506D20EA070050651B680122CB
:10F2300083F85820CEB9194B9847164B98471CB104
:10F24000154B1B685B6D2360134B1B6893F858309C
:10F25000DBB2022B16D000240F4B1B68002283F870
:10F2600058200E4B98472046F8BD114630460C4BAF
:10F2700098474FF080520B4B1A60BFF34F8FBFF38C
:10F280006F8FD8E7044B1A68536D23EA050555655F
:10F290000124E1E7C5DD4000040F0020E5DD40006A
:10F2A000DDE8400004ED00E0F8B504460F461546E1
:10F2B0001E46214B98470EB1636D336094F8583069
:10F2C000DBB2022284F858206A1E032A1AD8DFE82B
:10F2D00002F0020C1114626D174367650125012BC2
:10F2E00014D0164B98472846F8BD626D013262650E
:10F2F0000125F4E767650125F1E7022B04D0676576
:10F300000125ECE70125EAE70025E8E7261D304660
:10F310000B4B9847E36A01229A400A490868024366
:10F320000A6003EB83039A00314607481044074BF9
:10F330009847074B1B68D4E7C5DD4000E5DD40007A
:10F34000F1DC4000840F0020100F0020A5DC4000FD
:10F35000040F0020F8B5EFF311854FF0500484F34B
:10F360001188BFF36F8FBFF34F8F0BB1446D1C60DB
:10F3700090F85830DBB2022480F85840013A032A52
:10F380001AD8DFE802F0020C1114426D11434165F6
:10F390000126012B14D085F311883046F8BD426D4B
:10F3A000013242650126F4E741650126F1E7022BAF
:10F3B00004D041650126ECE70126EAE70026E8E7EC
:10F3C0000446164B1B68F3B9071D3846144B984783
:10F3D000E36A01229A401349086802430A6003EB7A
:10F3E00083039A00394610481044104B9847E26A4C
:10F3F0000F4B1B68DB6A9A42CDD9069B4BB10123A8
:10F40000069A1360C7E700F118010A48074B9847AE
:10F41000EDE70122084B1A60BDE700BF7C0F00201A
:10F42000F1DC4000840F0020100F0020A5DC40001C
:10F43000040F0020BC0F0020EC0F0020F8B5EFF304
:10F4400011854FF0500383F31188BFF36F8FBFF323
:10F450004F8F90F85830DBB2022280F85820426D6E
:10F4600001324265012B02D085F31188F8BD0E46AA
:10F470000446154B1B68E3B9071D3846134B9847E4
:10F48000E36A01229A401249086802430A6003EBCA
:10F4900083039A0039460F4810440F4B9847E26A9D
:10F4A0000E4B1B68DB6A9A42DED946B101233360FA
:10F4B000DAE700F118010A48074B9847EFE7012205
:10F4C000084B1A60D0E700BF7C0F0020F1DC400041
:10F4D000840F0020100F0020A5DC4000040F002046
:10F4E000BC0F0020EC0F0020064B1A681368B3FA1B
:10F4F00083F35B09036013B9D36818687047002071
:10F50000704700BFF00F002008B5416000619142D4
:10F510000CD8D21A83699A4201D3012008BD011D7B
:10F52000094B1868094B9847002008BD9A4201D240
:10F53000994206D2011D064B1868044B98470020DB
:10F5400008BD012008BD00BFF40F0020BDDC400055
:10F55000F00F002070B5104B9847104B1B6813B18B
:10F560000F4B984770BD0F4D28460F4EB0470F4CBC
:10F570002046B0470E4B1D600E4B1C6000220C2134
:10F580000A200D4B9847054B18600028E8D00B491E
:10F590000B4B9847E4E700BFC5DD40002410002076
:10F5A000E5DD4000F80F002089DC40000C10002051
:10F5B000F00F0020F40F002079E140007048410076
:10F5C00011E640002DE9F041079C7CB198461546B4
:10F5D0000E460746064B98472760A661E561C4F8CA
:10F5E0002080069B6362201D024B9847BDE8F08196
:10F5F00055F540009FDC400010B582B0094B98479C
:10F60000094B1B6863B1094B01930323009300234B
:10F610004FF42F7206490748074CA04702B010BDAF
:10F620000020FBE755F540002410002028100020A2
:10F630007848410031F94000A1E940002DE9F0414E
:10F6400082B005460E46174698462C20084B984730
:10F65000044640B10190089B009343463A46314628
:10F660002846044DA847204602B0BDE8F08100BFFF
:10F6700019DF4000C5F5400030B585B0134C256852
:10F680000DB31C46019102920390052913DC104B27
:10F690009847022807D000231A4601A90B480068A2
:10F6A0000C4CA0470DE00023089A01A90748006808
:10F6B000084CA04705E00023224601A92846064C35
:10F6C000A04705B030BD0020FBE700BF241000209C
:10F6D00055EF4000B5E140000DE3400070B582B049
:10F6E000154B1B681A6802B3DB681E68DC68251DB1
:10F6F0002846124B9847636A20469847E369012BD6
:10F70000EED1A36933449E4207D263602461294647
:10F71000094B18680A4B9847E2E7002100910B4615
:10F7200032462046074CA047DAE7074A10680249EC
:10F730000860136002B070BDF00F0020F1DC4000E3
:10F74000BDDC400079F64000F40F002038B50546D6
:10F75000084B98470446084B1B68984205D3002382
:10F760002B60054B1C60204638BD044B9847012395
:10F770002B60F6E79DEA400020100020DDF64000F7
:10F7800070B582B005460E460F4B1B68DB68DC681F
:10F79000201D0E4B9847E369012B04D0636A204675
:10F7A000984702B070BDA1692B46324629442046D5
:10F7B000074EB0470028F1D0002100910B462A46A1
:10F7C0002046044DA847E9E7F00F0020F1DC400097
:10F7D00009F5400079F6400070B582B006460C4647
:10F7E000174B984701A8174B9847019B23BB054629
:10F7F0000CB9B04219D22CB1134B1B681C68B4FA77
:10F8000084F464092246711B104B1868104B98470A
:10F81000104B984738B94FF080520F4B1A60BFF326
:10F820004F8FBFF36F8F02B070BD0A4B98472946C8
:10F8300030460A4B9847F6E7064B9847F3E700BF78
:10F840008DEA40004DF74000F40F00202410002006
:10F8500039E640009DEB400004ED00E081F74000F8
:10F8600030B587B0002203A92A4B18682A4B984765
:10F8700000284CD0039B002BF4DB059C636913B17B
:10F88000201D264B984702A8254B9847039B092B20
:10F89000E8D801A252F823F0C1F84000C1F84000B6
:10F8A000C1F8400065F84000F5F8400007F9400055
:10F8B000C1F84000C1F8400065F84000F5F840008C
:10F8C0000499A5690B46024629442046154DA847D0
:10F8D0000028C7D0636A20469847E369012BC1D14D
:10F8E000A269002100910B460498024420460E4C68
:10F8F000A047B7E70499A1610346024601442046A8
:10F90000084CA047AEE72046084B9847AAE707B047
:10F9100030BD00BF2410002085E34000F1DC400032
:10F920004DF7400009F5400079F640003DDF40000A
:10F9300000B583B001A8044B98470199034B984741
:10F94000034B9847F6E700BFE9F44000D9F74000C1
:10F9500061F84000064BDB6BC3F30023054A1370CC
:10F96000054BDB6BC3F34033044A1370704700BF91
:10F9700000100E402C100020000E0E402D10002014
:10F9800008B5054BDB6B13F4004F02D1034B9847CE
:10F9900008BD034B984708BD000E0E40A95140001A
:10F9A000CD51400030B583B004460D46002301938D
:10F9B0002E4B984213D02E4B9C421AD02D4B9C427A
:10F9C00021D02D4B9C4228D02C4B9C422FD02C4B2D
:10F9D0009C4236D02B4B9C423DD003B030BD01A998
:10F9E0002046294B98470028F9D19DF804302B7008
:10F9F000E1E701A92046244B98470028F9D19DF85A
:10FA000004302B70DAE701A920461F4B98470028E5
:10FA1000F9D19DF804302B70D3E701A920461A4B89
:10FA200098470028F9D19DF804302B70CCE701A944
:10FA30002046154B98470028F9D19DF804302B70CB
:10FA4000C5E701A92046104B98470028F9D19DF839
:10FA500004302B70BEE701A920460B4B98470028C5
:10FA6000F9D19DF804302B70B7E700BF00C2004009
:10FA700000020240004202400082014000C20140F8
:10FA8000008200400002044031D9400038B50446ED
:10FA90000D46274B984213D0264B984218D0264B40
:10FAA00098421DD0254B984222D0254B984227D012
:10FAB000244B98422CD0244B984231D0002038BDA2
:10FAC00029462046214B98470028F9D1012038BD0E
:10FAD000294620461D4B98470028F9D1012038BD02
:10FAE00029462046194B98470028F9D1012038BDF6
:10FAF00029462046154B98470028F9D1012038BDEA
:10FB000029462046114B98470028F9D1012038BDDD
:10FB1000294620460D4B98470028F9D1012038BDD1
:10FB200029462046094B98470028F9D1012038BDC5
:10FB300000C2004000020240004202400082014038
:10FB400000C20140008200400002044009D9400088
:10FB500000B583B002A9002341F8043D084B1868A2
:10FB6000084B9847019B3BB14FF08052064B1A60FF
:10FB7000BFF34F8FBFF36F8F03B05DF804FB00BF7F
:10FB8000341000203DF4400004ED00E070B58AB070
:10FB90001D4B0FCB0AAC04E90F001C4D1C4B1D6024
:10FBA0001C4A1D4B1A601D4A1D4B1A60069B009390
:10FBB000079B0193089B0293099B039300240494E1
:10FBC000184E3046184B984701213046174B98473E
:10FBD000174A69462846174B98472846164B9847B8
:10FBE0002846164B9847164E336821469868154D9F
:10FBF000A847336821465868A84733682146986863
:10FC0000A8470AB070BD00BF804841000082014093
:10FC1000982200208DFA400094220020A5F940008F
:10FC20009022002000800140F1D4400059D64000CD
:10FC30000000DC0595D94000E1D84000EDD8400037
:10FC40003C0300207517410008B504460D460A46DE
:10FC500001460748074B98470220074B984729461B
:10FC60002046064B9847EFF30580054B9847FFDE8B
:10FC700044494100F50D4100214D40000D4D40002B
:10FC80002D4D400070B51F4B98471F4B1B68C31A82
:10FC9000632B00D870BD1C4B18601C4B18681C4DA2
:10FCA000A8471C4C20601C481C4EB047A847606009
:10FCB0001B48B047A847A0601A48B047A847E06073
:10FCC0001948B047A84720611848B047A847606165
:10FCD0001748B047A847A0611648B047A847E06159
:10FCE0001548B047A84720621448B047A84760624B
:10FCF0001348B047A847A0621248B047A847E0623F
:10FD0000C8E700BF9DEA40003010002034100020FA
:10FD100039EF40001423002038494100B5EC400081
:10FD2000FC414100A0474100C0474100F447410069
:10FD30001448410034484100544741009441410077
:10FD40006848410078484100704700002DE9F043C1
:10FD500083B04B4B98474B4A936843F0254343F499
:10FD600080139360484B9847484B9847484B9847B7
:10FD7000484B9847484B9847484B98470446484B50
:10FD80009847F02201462046464B9847464B9847F5
:10FD90004648474B03602223037123234371454D9B
:10FDA0002946454CA0474548454B03602B2303712A
:10FDB0002A2343712946A047424B9847424B984714
:10FDC0004248434B98474348434CA0474349444823
:10FDD000A04744494448A047444A45494548A047AC
:10FDE00000230193042200924FF480724249434859
:10FDF000434CA047012802D04248374B98473E4821
:10FE0000414B9847414B1860414B9847414B9847AD
:10FE1000414B9847414B9847414A00210F20414EA2
:10FE2000B047414C03220B212046404DA847DFF844
:10FE300010914A4600212820B0473D4F03220C2153
:10FE40003846A8472820DFF8FC80C04701463846DE
:10FE5000384FB8474A4600210D20B04703220B21F6
:10FE60002046A8470D20C04701462046B847324BE0
:10FE70009847324B9847002003B0BDE8F08300BF9D
:10FE80006945400010140E4071D340006D7640006B
:10FE9000A96A40008DFB4000797240003174400037
:10FEA00039744000F17240000D73400000230020BF
:10FEB00000000240A08601003D6F4000EC220020BF
:10FEC00000C001400DB240007169400051FB40008C
:10FED0005D45400090484100F50D4100A8484100B3
:10FEE000BC48410034424100C8484100DC48410060
:10FEF000E8484100F44841000C4941004574400085
:10FF0000A1E9400014494100B5EC40003410002044
:10FF100065934000F1A84000E19B4000898B4000C0
:10FF200081F9400071B54000000E0E40E1B540007F
:10FF300000100E40EFD24000FB4E400015EA40009A
:10FF400055F9400013D3400030B583B000248DF83C
:10FF500004408DF805408DF806400F4B98470F4B35
:10FF6000984720460E4B98470E4D01A928460E4B48
:10FF7000984772B60D480E4CA0472846A0470D4B37
:10FF800098470D4B98470D4B98470D4A136823F03F
:10FF90000103136003B030BD397640008DEA4000A4
:10FFA000F1504000EC220020795F40000023002047
:10FFB000D56F40009550400059B240008D7340000D
:10FFC00010E000E000487047002300200048704720
:10FFD000EC22002008B5014B984708BD4174400051
:10FFE00008B5014B984708BD437440007047012095
:10FFF0007047000008B50248024B984708BD00BF93
:020000040041B9
:10000000002300207570400008B50248024B984755
:1000100008BD00BFEC22002075704000014B18782D
:10002000704700BF2D100020014B1878704700BFAB
:100030002C10002070B58AB0044600F06FF8324BE7
:1000400093F900506B1C064609D02146204600F06B
:100050008DFE20B90021204600F07EFE10B1304612
:100060000AB070BD294B08902046019300F006FBB2
:10007000CDE90401CDE902012046CDB9244B4FF072
:1000800060420021CDE9062300F03EFE002833D077
:1000900002230093684600F085F9A8B1089BC3B914
:1000A000DDE9060100F03EFB064630460AB070BDB1
:1000B000184B00220021CDE9062300F025FE68B18F
:1000C00002239D420093E5D100F066FE22230360E7
:1000D000E4E700F061FE089B0360E1E70123022DE5
:1000E00000930BD100F058FE212303600A4800F072
:1000F0005BF9CDE90601D1E701230093684600F0E2
:1001000051F90028F2D1EDE7380300205C494100A5
:10011000FFFFEFC70000F0FF644841002DE9F84FF2
:1001200030F000432DD00028014604464ADBB0F1F0
:10013000FF4F3BDAB0F5000F3CDB00268D4AC4F3DD
:1001400016052A4402F40002E41582F07E507F3C3A
:1001500034444FF07E51284304EBD25400F036FB78
:1001600005F10F03C3F316030F2B064631DC002104
:1001700000F0CAFD002800F094804CB90020BDE8D2
:10018000F88F00214FF04C4000F0DEFCBDE8F88F06
:10019000204600F0D1FB7849054600F021FC774964
:1001A0000446284600F01CFC0146204600F010FBE7
:1001B000BDE8F88F4FF0984100F012FC6FF0180680
:1001C0000446BBE700F002FB002100F0BDFCBDE8E7
:1001D000F88F4FF0804100F0FBFA0146304600F006
:1001E000B3FC8046204600F0A7FB414681464046CE
:1001F00000F0F6FB0146834600F0F2FB6049DFF8B1
:10020000A0A1074600F0ECFB5E4900F0E1FA394698
:1002100000F0E6FB5C4900F0DBFA394600F0E0FB59
:100220005A4900F0D5FA594600F0DAFB584983469E
:10023000384600F0D5FB574900F0CAFA394600F0BD
:10024000CFFB554900F0C4FA394600F0C9FB01461E
:10025000584600F0BDFAC5F55713AA4403F52273BA
:1002600043EA0A03002B074665DD4FF07C51304618
:1002700000F0B6FB314600F0B3FB0546002C32D14E
:100280002946384600F0A4FA414600F0A9FB014691
:10029000284600F09BFA0146304600F097FABDE888
:1002A000F88F3E49304600F09BFB01464FF07C50F2
:1002B00000F08CFA31460546304600F091FB0146CD
:1002C000284600F08DFB0546002C2ED0204600F07D
:1002D00033FB2949074600F083FB2849044638468A
:1002E00000F07EFB14E02449484600F079FB2946E3
:1002F0000446384600F06CFA414600F071FB1F4995
:100300000746484600F06CFB0146384600F060FAAC
:100310000146284600F05AFA314600F057FA0146E5
:10032000204600F053FABDE8F88F0146304600F051
:100330004DFABDE8F88F7CB10F49484600F050FBFC
:1003400039460446304600F041FA414600F048FB89
:100350000A4905464846C3E70146304600F036FAEA
:10036000414600F03DFB0146304600F02FFABDE863
:10037000F88F00BF20FB4A008071313FD1F717375B
:100380009788173E25333A3E2549923EABAA2A3F2D
:100390004FD01C3E298E633ECDCCCC3EABAAAA3EAC
:1003A000305CCFFF0020704700200149704700BF3C
:1003B0000000F87F81F0004102E000BF83F00043BD
:1003C00030B54FEA41044FEA430594EA050F08BFF0
:1003D00090EA020F1FBF54EA000C55EA020C7FEAB4
:1003E000645C7FEA655C00F0E2804FEA5454D4EB31
:1003F0005555B8BF6D420CDD2C4480EA020281EAFB
:10040000030382EA000083EA010180EA020281EA32
:100410000303362D88BF30BD11F0004F4FEA013184
:100420004FF4801C4CEA113102D0404261EB410193
:1004300013F0004F4FEA03334CEA133302D0524219
:1004400063EB430394EA050F00F0A780A4F10104D5
:10045000D5F1200E0DDB02FA0EFC22FA05F280180F
:1004600041F1000103FA0EF2801843FA05F35941F5
:100470000EE0A5F120050EF1200E012A03FA0EFC74
:1004800028BF4CF0020C43FA05F3C01851EBE3719E
:1004900001F0004507D54FF0000EDCF1000C7EEBBB
:1004A00000006EEB0101B1F5801F1BD3B1F5001FF9
:1004B0000CD349085FEA30004FEA3C0C04F1010418
:1004C0004FEA445212F5800F80F09A80BCF1004F41
:1004D00008BF5FEA500C50F1000041EB045141EAC3
:1004E000050130BD5FEA4C0C404141EB010111F4C4
:1004F000801FA4F10104E9D191F0000F04BF01466F
:100500000020B1FA81F308BF2033A3F10B03B3F14C
:1005100020020CDA0C3208DD02F1140CC2F10C02DC
:1005200001FA0CF021FA02F10CE002F11402D8BF3A
:10053000C2F1200C01FA02F120FA0CFCDCBF41EA06
:100540000C019040E41AA2BF01EB0451294330BDD5
:100550006FEA04041F3C1CDA0C340EDC04F11404B2
:10056000C4F1200220FA04F001FA02F340EA030089
:1005700021FA04F345EA030130BDC4F10C04C4F1CF
:10058000200220FA02F001FA04F340EA03002946AF
:1005900030BD21FA04F0294630BD94F0000F83F4F9
:1005A000801306BF81F480110134013D4EE77FEADC
:1005B000645C18BF7FEA655C29D094EA050F08BF28
:1005C00090EA020F05D054EA000C04BF1946104609
:1005D00030BD91EA030F1EBF0021002030BD5FEA4D
:1005E000545C05D14000494128BF41F0004130BD75
:1005F00014F580043CBF01F5801130BD01F00045C9
:1006000045F0FE4141F470014FF0000030BD7FEA3B
:10061000645C1ABF194610467FEA655C1CBF0B4636
:10062000024650EA013406BF52EA033591EA030F4D
:1006300041F4002130BD00BF90F0000F04BF002145
:10064000704730B54FF4806404F132044FF0000578
:100650004FF0000150E700BF90F0000F04BF0021F1
:10066000704730B54FF4806404F1320410F0004557
:1006700048BF40424FF000013EE700BF42004FEA52
:10068000E2014FEA31014FEA02701FBF12F07F43CF
:1006900093F07F4F81F06051704792F0000F14BFCC
:1006A00093F07F4F704730B54FF4607401F0004510
:1006B00021F0004120E700BF50EA010208BF704767
:1006C00030B54FF000050AE050EA010208BF70475C
:1006D00030B511F0004502D5404261EB41014FF4C5
:1006E000806404F132045FEA915C3FF4DCAE4FF0C9
:1006F00003025FEADC0C18BF03325FEADC0C18BFB0
:10070000033202EBDC02C2F1200300FA03FC20FA00
:1007100002F001FA03FE40EA0E0021FA02F114444D
:10072000C1E600BF4FEA4102B2F1E04324BFB3F596
:10073000001CDCF1FE5C0DD901F0004C4FEAC00258
:100740004CEA5070B2F1004F40EB830008BF20F03C
:100750000100704711F0804F21D113F13872BCBFF6
:1007600001F00040704741F480114FEA5252C2F14B
:100770001802C2F1200C10FA0CF320FA02F018BF94
:1007800040F001004FEAC1234FEAD32303FA0CFCE7
:1007900040EA0C0023FA02F34FEA4303CCE77FEA76
:1007A000625307D150EA01331EBF4FF0FE4040F4C0
:1007B0004000704701F0004040F0FE4040F400006F
:1007C000704700BF80F0004002E000BF81F00041B0
:1007D00042001FBF5FEA410392EA030F7FEA226CE7
:1007E0007FEA236C6AD04FEA1262D2EB1363C1BF77
:1007F000D218414048404140B8BF5B42192B88BFE6
:10080000704710F0004F40F4000020F07F4018BF08
:10081000404211F0004F41F4000121F07F4118BF28
:10082000494292EA030F3FD0A2F1010241FA03FCD0
:1008300010EB0C00C3F1200301FA03F100F00043B8
:1008400002D5494260EB4000B0F5000F13D3B0F180
:10085000807F06D340084FEA310102F10102FE2AEF
:1008600051D2B1F1004F40EBC25008BF20F001005F
:1008700040EA03007047490040EB000010F4000F0D
:10088000A2F10102EDD1B0FA80FCACF1080CB2EBA0
:100890000C0200FA0CF0AABF00EBC25052421843FF
:1008A000BCBFD0401843704792F0000F81F40001A4
:1008B00006BF80F400000132013BB5E74FEA410377
:1008C0007FEA226C18BF7FEA236C21D092EA030FE3
:1008D00004D092F0000F08BF0846704790EA010F5D
:1008E0001CBF0020704712F07F4F04D1400028BF8A
:1008F00040F00040704712F100723CBF00F500006C
:10090000704700F0004343F0FE4040F400007047A1
:100910007FEA226216BF08467FEA2363014642024D
:1009200006BF5FEA412390EA010F40F48000704760
:100930004FF0000304E000BF10F0004348BF404206
:100940005FEA000C08BF704743F0964301464FF042
:1009500000001CE050EA010208BF70474FF000039E
:100960000AE000BF50EA010208BF704711F00043DF
:1009700002D5404261EB41015FEA010C02BF8446AF
:100980000146002043F0B64308BFA3F18053A3F50E
:100990000003BCFA8CF2083AA3EBC25310DB01FA55
:1009A00002FC634400FA02FCC2F12002BCF1004FD9
:1009B00020FA02F243EB020008BF20F0010070476A
:1009C00002F1200201FA02FCC2F1200250EA4C00BE
:1009D00021FA02F243EB020008BF20EADC70704704
:1009E0004FF0FF0C1CEAD0521EBF1CEAD15392EA12
:1009F0000C0F93EA0C0F6FD01A4480EA010C4002EE
:100A000018BF5FEA41211ED04FF0006343EA501047
:100A100043EA5111A0FB01310CF00040B1F5000F89
:100A20003EBF490041EAD3715B0040EA010062F138
:100A30007F02FD2A1DD8B3F1004F40EBC25008BF22
:100A400020F00100704790F0000F0CF0004C08BF40
:100A500049024CEA502040EA51207F3AC2BFD2F10D
:100A6000FF0340EAC250704740F400004FF000031B
:100A7000013A5DDC12F1190FDCBF00F00040704755
:100A8000C2F10002410021FA02F1C2F1200200FA93
:100A900002FC5FEA310040F1000053EA4C0308BF5A
:100AA00020EADC70704792F0000F00F0004C02BFAB
:100AB000400010F4000F013AF9D040EA0C0093F026
:100AC000000F01F0004C02BF490011F4000F013B80
:100AD000F9D041EA0C018FE70CEAD15392EA0C0FEE
:100AE00018BF93EA0C0F0AD030F0004C18BF31F059
:100AF000004CD8D180EA010000F00040704790F02F
:100B0000000F17BF90F0004F084691F0000F91F0D2
:100B1000004F14D092EA0C0F01D142020FD193EA98
:100B20000C0F03D14B0218BF084608D180EA010020
:100B300000F0004040F0FE4040F40000704740F0FC
:100B4000FE4040F4400070474FF0FF0C1CEAD052CA
:100B50001EBF1CEAD15392EA0C0F93EA0C0F69D026
:100B6000A2EB030280EA010C49024FEA402037D091
:100B70004FF0805343EA111143EA10130CF0004088
:100B80008B4238BF5B0042F17D024FF4000C8B4278
:100B900024BF5B1A40EA0C00B3EB510F24BFA3EB58
:100BA000510340EA5C00B3EB910F24BFA3EB910328
:100BB00040EA9C00B3EBD10F24BFA3EBD10340EA82
:100BC000DC001B0118BF5FEA1C1CE0D1FD2A3FF6C8
:100BD00050AF8B4240EBC25008BF20F0010070477D
:100BE0000CF0004C4CEA50207F32C2BFD2F1FF0320
:100BF00040EAC250704740F400004FF00003013A51
:100C000037E792F0000F00F0004C02BF400010F4F4
:100C1000000F013AF9D040EA0C0093F0000F01F008
:100C2000004C02BF490011F4000F013BF9D041EA2A
:100C30000C0195E70CEAD15392EA0C0F08D142025D
:100C40007FF47DAF93EA0C0F7FF470AF084676E730
:100C500093EA0C0F04D14B023FF44CAF08466EE709
:100C600030F0004C18BF31F0004CCAD130F00042D7
:100C70007FF45CAF31F000437FF43CAF5FE700BF2F
:100C80004FF0FF3C06E000BF4FF0010C02E000BF58
:100C90004FF0010C4DF804CD4FEA40024FEA4103FA
:100CA0007FEA226C18BF7FEA236C11D001B052EAB0
:100CB000530C18BF90EA010F58BFB2EB030088BF76
:100CC000C81738BF6FEAE17018BF40F001007047E5
:100CD0007FEA226C02D15FEA402C05D17FEA236CC7
:100CE000E4D15FEA412CE1D05DF8040B704700BF0E
:100CF000844608466146FFE70FB5FFF7C9FF0028A5
:100D000048BF10F1000F0FBD4DF808EDFFF7F4FFDD
:100D10000CBF012000205DF808FB00BF4DF808ED76
:100D2000FFF7EAFF34BF012000205DF808FB00BF99
:100D30004DF808EDFFF7E0FF94BF012000205DF8BB
:100D400008FB00BF4DF808EDFFF7D2FF94BF01206C
:100D500000205DF808FB00BF4DF808EDFFF7C8FF65
:100D600034BF012000205DF808FB00BF4FEA4002BD
:100D70004FEA41037FEA226C02D15FEA402C08D19E
:100D80007FEA236C02D15FEA412C02D14FF00000D0
:100D900070474FF001007047014B1868704700BF63
:100DA0003C03002070B50F4E0F4D761BB61018BFD8
:100DB000002405D0013455F8043B9847A642F9D1E8
:100DC0000A4E0B4D761B03F081FEB61018BF0024AF
:100DD00006D0013455F8043B9847A642F9D170BDBE
:100DE00070BD00BFD84A4100D84A4100E04A4100E6
:100DF000D84A41000FB400B5074983B004AB086876
:100E000053F8042B8168019300F066FE03B05DF88F
:100E100004EB04B0704700BF3C030020024B0146C6
:100E2000186800F00BB800BF3C030020024B0146DD
:100E3000186801F06DBF00BF3C0300202DE9F04FA2
:100E400001F10B06162E83B0054640F29E8036F067
:100E5000070600F1BD80B14200F2BA8000F06CFCE0
:100E6000B6F5FC7FC0F09382730A00F0B880042BC3
:100E700000F27981B30903F1390003F1380EC300A0
:100E8000BF4F3B44A3F108015C68A14206D10CE0CE
:100E9000002A80F2AA80E468A14206D0636823F0A9
:100EA00003039A1B0F2AF3DD70463C69DFF8E4E286
:100EB000744500F0AB81636823F003039A1B0F2A8B
:100EC00000F39081002AC7F814E0C7F810E080F220
:100ED0009D80B3F5007F80F06181DB0803F1010C98
:100EE00099107A6857F83C80C4F8088001238B4039
:100EF00007EBCC0113430839E1607B6047F83C40C5
:100F0000C8F80C408210012494409C4200F28B806F
:100F10001C4206D120F0030064001C4200F10400D2
:100F2000FAD007EBC009CC468046DCF80C309C4573
:100F300007D16DE1002A80F27B81DB689C4500F0DF
:100F40006781596821F003018A1B0F2AF2DDD3F86B
:100F50000CC0D3F8088000939C19284646F001067F
:100F600042F001055E60C8F80CC0CCF808807C61D6
:100F70003C61C4F80CE0C4F808E065605A5000F029
:100F8000E1FB009B03F108041EE0102920D800F0CB
:100F9000D3FB102618230220794F3B44A3F108020B
:100FA0005C68944200F03D816368E168A66823F0C4
:100FB0000303234428465A68F16042F001028E6020
:100FC0005A6000F0BFFB0834204603B0BDE8F08F44
:100FD00000240C2320462B6003B0BDE8F08F402096
:100FE0004FF400734FF03F0E4AE72344E1685A681C
:100FF000A66842F00102F16028468E605A6000F057
:10100000A1FB0834204603B0BDE8F08F23442846F6
:101010005A6842F001025A6000F094FB08342046FE
:1010200003B0BDE8F08FBC68636823F00308B045E7
:1010300004D3A8EB06030F2B00F38580DFF858914B
:10104000504BD9F800201B680132334404EB080AE6
:1010500000F0558103F580530F3323F47F6B2BF0A1
:101060000F0B5946284600F073FB411C024600F066
:10107000FC80824500F2F780434B1968594419609F
:1010800000F04D81D9F8000001301BBFA2EB0A0A25
:101090005144C9F80020196012F0070100F01581D1
:1010A000C1F10800C1F580510244083102EB0B097F
:1010B000C9F30B09A1EB090949462846019300929F
:1010C00000F046FB431C9DE80C0000F04381801AB1
:1010D000484440F001001968BA604944BC4250607D
:1010E000196017D0B8F10F0F40F2FB806068A8F1CB
:1010F0000C0222F0070204EB020E00F001004FF098
:10110000050C10430F2A6060CEF804C0CEF808C06A
:1011100000F217811D4BBC681A68914288BF1960A4
:101120001B4B1A689142626888BF196022F0030263
:101130009642A2EB060301D80F2B04DC284600F0F0
:1011400001FB002440E7A21943F0010346F0010629
:1011500066602846BA60536000F0F4FA083420460E
:1011600003B0BDE8F08F142B71D9542B00F2A3808B
:10117000330B03F16F0003F16E0EC30080E600BF76
:101180006807002068100020381000206010002040
:101190006410002070070020700B00205A0A042AF7
:1011A0005BD9142A00F2AE8002F15C01C9005B3207
:1011B00007EB010C7958ACF1080C8C4500F08880E5
:1011C0004A6822F00302934273D289688C45F7D1B2
:1011D000DCF80C207B68E260C4F808C09460CCF8AE
:1011E0000C408FE6A11946F0010C42F00106C4F84C
:1011F00004C0284679613961C1F80CE0C1F808E003
:101200004E60E25000F09EFA0834DDE67B6879E635
:1012100008F1010818F0030F0CF1080C7FF485AEFB
:101220002DE0DC68A34208BF02303FF43EAEBBE6CF
:1012300019441C464A68DB6854F8086F42F0010202
:101240004A602846F3609E6000F07CFABCE603F139
:101250005C0003F15B0EC30012E69A0902F139014A
:10126000C9003832A4E7BC4254D0BC68626822F09E
:1012700003025DE759F80839994540F0868010F07F
:10128000030F00F1FF30F5D17B6823EA04037B6094
:1012900064009C423FF6C7AE002C3FF4C4AE1C4233
:1012A00040467FF43EAE64001C4200F10400FAD0D8
:1012B00037E68C468CE7B3F5AA7F15D8F30B03F11C
:1012C000780003F1770EC300DAE54FF48051EDE6C4
:1012D0007B689210012101FA02F213437B6062469F
:1012E00079E70123536029E740F25452934222D810
:1012F000B30C03F17D0003F17C0EC300C0E503F1E4
:10130000100BAEE6542A29D81A0B02F16F01C9005E
:101310006E324DE7204B196859441960B2E6CAF3A2
:101320000B0000287FF4AEAE08EB0B03BA6843F065
:1013300001035360EEE67F204FF47E734FF07E0E84
:101340009EE504F108012846009301F0E1FC009BB2
:101350001968DFE601204FF00009BCE6B2F5AA7F6C
:1013600005D8DA0B02F17801C900773220E740F2A4
:1013700054518A4205D89A0C02F17D01C9007C3291
:1013800016E74FF47E717E2212E77B6880E7F00853
:1013900006F1080300E600BF38100020000000003E
:1013A00001F0FF01102A2BDB10F0070F08D010F816
:1013B000013B013A8B422DD010F0070F42B3F6D11A
:1013C000F0B441EA012141EA014122F007047FF033
:1013D00000070023F0E80256083C85EA010586EA8A
:1013E000010685FA47F5A3FA87F586FA47F6A5FAC6
:1013F00087F68EB9EED1F0BC01F0FF0102F00702D2
:1014000032B110F8013B013A83EA010313B1F8D17C
:101410000020704701387047002D06BF354603385D
:10142000073815F0010F07D1013015F4807F02BF96
:10143000013015F4C03F0130F0BC0138704700BFE7
:10144000032A70B422D940EA01039B0711D0037824
:101450000C78A3421DD10A44013105E010F8013F88
:1014600011F8014BA34214D19142F7D1002070BC76
:1014700070470D680668AE420C46034601F1040150
:1014800000F1040008D1043A032AF2D8002ADED180
:10149000ECE7181B70BC704721461846D7E700BF21
:1014A000844641EA000313F003036DD1403A41D36F
:1014B00051F8043B40F8043B51F8043B40F8043B2E
:1014C00051F8043B40F8043B51F8043B40F8043B1E
:1014D00051F8043B40F8043B51F8043B40F8043B0E
:1014E00051F8043B40F8043B51F8043B40F8043BFE
:1014F00051F8043B40F8043B51F8043B40F8043BEE
:1015000051F8043B40F8043B51F8043B40F8043BDD
:1015100051F8043B40F8043B51F8043B40F8043BCD
:1015200051F8043B40F8043B51F8043B40F8043BBD
:10153000403ABDD2303211D351F8043B40F8043B5D
:1015400051F8043B40F8043B51F8043B40F8043B9D
:1015500051F8043B40F8043B103AEDD20C3205D36D
:1015600051F8043B40F8043B043AF9D2043208D065
:10157000D2071CBF11F8013B00F8013B01D30B88D7
:1015800003806046704700BF082A13D38B078DD0B5
:1015900010F003038AD0C3F10403D21ADB071CBF87
:1015A00011F8013B00F8013B80D331F8023B20F8F1
:1015B000023B7BE7043AD9D3013A11F8013B00F82A
:1015C000013BF9D20B7803704B7843708B788370B2
:1015D000604670478842F0B50DD98B1898420AD200
:1015E0008418002A51D0224613F8014D02F8014D0B
:1015F0009942F9D1F0BD0F2A48D941EA00039B076F
:1016000046D100F1100401F11003154653F8106C97
:1016100044F8106C53F80C6C44F80C6C53F8086CDC
:1016200044F8086C103D53F8046C44F8046C0F2D1A
:1016300003F1100304F11004E8D8A2F1100323F021
:101640000F0302F00F0E1033BEF1030F19440344D1
:1016500021D91E1F0D467446043C55F8047B46F8FC
:10166000047F032CF8D8AEF1040424F003040434FE
:101670002144234402F0030262B1013B0A4411F801
:10168000014B03F8014F8A42F9D1F0BD0346F3E75D
:101690000346F2E7F0BD7246EEE700BF70B486077E
:1016A00046D0541E002A41D0CAB2034602E014F1CB
:1016B000FF343BD303F8012B9D07F8D1032C2ED91F
:1016C000CDB245EA05250F2C45EA054519D903F1A8
:1016D00010022646103E0F2E42F8105C42F80C5CB9
:1016E00042F8085C42F8045C02F11002F2D8A4F15E
:1016F000100222F00F0204F00F041032032C1344E6
:101700000DD91E462246043A032A46F8045BFAD84D
:10171000221F22F003020432134404F003042CB10C
:10172000C9B21C4403F8011B9C42FBD170BC70473A
:1017300014460346C2E700BF014801F083BD00BF65
:1017400064230020014801F07FBD00BF6423002016
:1017500038B5074C0023054608462360FCF76CFAB1
:10176000431C00D038BD2368002BFBD02B6038BD54
:101770007823002000290CBF022200224FF480634E
:1017800000F000B82DE9F043614C256883B00446B1
:101790000F4690461E4615B1AB6B002B64D0B8F1D6
:1017A000020F06D0B8F1010F00F29F80002EC0F2A8
:1017B0009C80636ED80734D52146284601F02AF96B
:1017C000216B41B104F14003994202D0284601F057
:1017D0009FFA00232363B4F90C300022A2616260F7
:1017E0001A063AD423F44A6323F00303B8F1020F34
:1017F000A3811DD001AB6A462146284601F026FD93
:10180000A3891843A081002E32D1009E3046FFF7F5
:1018100005FB074600286BD0A38943F08003A38112
:1018200028E0A3899905C7D4A06D01F00BFDC3E79B
:101830000025616E002604F1430243F002030120FB
:10184000A660CE07A38122602261606101D4980561
:101850003ED5284603B0BDE8F0832169284601F053
:1018600057FAB4F90C30BDE7284601F02BF996E79A
:10187000002FCBD0AB6B002B33D0009BB4F90C20E6
:1018800027609E421CBF42F40062A281B8F1010FA2
:1018900004BF42F00102A28192B212F00803276154
:1018A00066610ED0D1071AD5656E7642002315F019
:1018B0000105A661A36009D00025284603B0BDE854
:1018C000F083A360656E15F00105F5D19305C0D4D2
:1018D000A06D01F0B9FC284603B0BDE8F083A66016
:1018E000F0E7284601F0EEF8C7E74FF0FF35B0E724
:1018F000DDF80090B14504D04846FFF78FFA07465F
:1019000020B9B4F90C304FF0FF3592E74E4683E72B
:101910003C03002000000000000000000000000068
:1019200000000000000000000000000000000000B7
:1019300000000000000000000000000000000000A7
:1019400090F800F06DE9024520F007016FF0000CFF
:1019500010F0070491F820F040F049804FF00004A7
:101960006FF00700D1E9002391F840F000F1080082
:1019700082FA4CF2A4FA8CF283FA4CF3A2FA8CF3BA
:101980004BBBD1E9022382FA4CF200F10800A4FA21
:101990008CF283FA4CF3A2FA8CF3E3B9D1E9042375
:1019A00082FA4CF200F10800A4FA8CF283FA4CF3AC
:1019B000A2FA8CF37BB9D1E9062301F1200182FA66
:1019C0004CF200F10800A4FA8CF283FA4CF3A2FA6C
:1019D0008CF3002BC6D0002A04BF04301A4612BA7A
:1019E000B2FA82F2FDE8024500EBD2007047D1E97D
:1019F000002304F00305C4F100004FEAC50514F00C
:101A0000040F91F840F00CFA05F562EA05021CBFDC
:101A100063EA050362464FF00004A9E7B1B1037819
:101A2000B3B10144431C994214D010B41A785C1C21
:101A300032B1A142234606D01A785C1C002AF8D1A4
:101A4000181A10BC7047081A10BC70470846704737
:101A500018467047081A70472DE9F84F4B6E9C04E2
:101A600093462FD59368126853B30E46074602F18A
:101A7000080919E920045FEA9A0817D0043D0024F8
:101A800001E0A04510D0324655F8041F384601F059
:101A9000BBF8431C04F10104F3D10023CBF8083058
:101AA000CBF80430BDE8F88FDBF808302AF0030AE1
:101AB000A3EB0A03CBF8083009F10809002BD8D1B1
:101AC0000020EAE701F00AFA0023CBF80830CBF84F
:101AD0000430BDE8F88F00BF2DE9F04FADB01D46D2
:101AE0008B4690460793069018B1836B002B00F04D
:101AF000F380DBF86430BBF90C00DF0781B202D45D
:101B00008E0540F1FC808C040AD4DBF8643040F48C
:101B1000005123F40053ABF80C10CBF8643089B2B9
:101B2000080740F1B380DBF81030002B00F0AE80E6
:101B300001F01A030A2B00F0B58000230DF17009A3
:101B40000B93119310930393CDF83C90CA46CDF8B4
:101B500010B098F800304446FBB1252B02D11CE0B0
:101B6000252B03D014F8013F002BF9D1A4EB080575
:101B70009DB1109B119ACAF8008001332A44072BAB
:101B8000CAF80450119210937ADD002A40F0B08414
:101B9000039B10922B44CA4603932378002B00F03A
:101BA000E08300204FF000038DF8373004F1010886
:101BB00062780546064603464FF0FF3408F10108F7
:101BC000A2F12001582900F2DE82DFE811F02102A3
:101BD000DC02DC022902DC02DC02DC02DC02DC02C8
:101BE000DC0289029502DC02A200BD02DC029F0138
:101BF000A401A401A401A401A401A401A401A401BD
:101C0000A401DC02DC02DC02DC02DC02DC02DC021D
:101C1000DC02DC02DC02B201DC02DC02DC02DC02FF
:101C2000DC02DC02DC02DC02DC02DC029701DC020A
:101C3000DC02DC02DC02DC029B01DC02DC0253027F
:101C4000DC02DC02DC02DC02DC02DC02DC02DC02A4
:101C5000DC02DC025A021B02DC02DC02DC026E0245
:101C60001B02DC02DC027302DC02F50182010902C4
:101C7000D702DC029A02DC02A700DC02DC022E02A0
:101C80000AF1080A039B2B44039386E759460698FA
:101C900000F0ACFD18BBBBF80C1001F01A030A2BC6
:101CA0007FF44BAFBBF90E30002BFFF646AFDBF8ED
:101CB0006430DB0705D48F0503D4DBF8580001F04E
:101CC000C3FA2B4642465946069800F04DFD039054
:101CD00003982DB0BDE8F08F00F0F4FE09E7DBF8C3
:101CE0006430D90704D4BBF80C309A0540F1AA84BB
:101CF0004FF0FF33039303982DB0BDE8F08FDBF86E
:101D0000580001F09FFABBF90C0081B2FBE6764265
:101D1000079243F0040398F800204FE708969E06C8
:101D200000F150840799DD060A4600F1EF8358065A
:101D300040F1EC830E8804310027012207914FF017
:101D400000018DF837100025611C00F0168123F08A
:101D50008001029156EA070140F01481002C40F006
:101D60005C83002A40F0B78313F00103059300F071
:101D700057840DF1B00B30230BF8413D059BA34276
:101D8000B8BF234601930DB101330193029B13F0B9
:101D90000203099302D0019B02330193029B13F0CB
:101DA00084030A9340F01782089B019A9D1A002D24
:101DB00040F31182102D40F39084109B119AC44E71
:101DC000D6461027A2461946069C07E001F1020CF0
:101DD0000EF1080E0146103D102D11DD481C103289
:101DE000072811928EE8C0001090EFDD002A40F025
:101DF000E481103D102D11464FF0010CCE46EDDC74
:101E000054466146F2462A4407291192CAF80060F6
:101E1000CAF80450109100F3EC829DF837500AF193
:101E2000080A481C002D40F0DE81099B002B00F0C1
:101E3000F88102320EA902230728119210908AE835
:101E40000A0040F3EA81002A40F08C830A9B802B31
:101E50004FF001001146CA4640F0E781089B019D02
:101E60005E1B002E40F3E181102E9A4D40F350840A
:101E7000D4461027A246069C07E001F1020E0CF1A1
:101E8000080C0146103E102E11DD481C10320728A8
:101E900011928CE8A0001090EFDD002A40F09D82A6
:101EA000103E102E4FF0010E1146CC46EDDC54468C
:101EB000E2463244BEF1070F11928AE86000CDF885
:101EC00040E000F369830AF1080A0EF1010071464F
:101ED000ABE1089613F0200240F08C8313F0100160
:101EE00040F01A8313F0400200F0168307980A4668
:101EF0000146043106880791002720E7089643F041
:101F00001003E7E7089643F0100308E743F0800367
:101F100098F8002052E6A2F13001002618F8012BB3
:101F200006EB860601EB4606A2F130010929F5D938
:101F300046E60896002840F0088443F010039E0609
:101F400000F14C83DD0600F1F382580640F1F08287
:101F5000079DB5F900602A46F71704323046394626
:101F60000792002871F10002C0F25D83611C9DF8A8
:101F700037504FF001027FF4EAAE56EA070100F055
:101F80004D820293012A00F08C82022A40F05C828A
:101F90000B98CB46330906F00F0143EA07733A0961
:101FA0001E461746435C0BF8013D56EA0703F1D184
:101FB000A9EB0B030593E1E6002840F0C0839906E6
:101FC00000F16783DA0600F1F1805B0640F1EE80F4
:101FD000079A136804320792BDF80C201A80B8E5FE
:101FE00007983D4A08960B92066878223021043003
:101FF0008DF8392043F00203079000278DF8381040
:1020000002229CE60896002899D08DF8375096E772
:1020100098F80020002D7FF4D1AD01202025CDE5DA
:1020200043F0010398F80020C8E50896002840F026
:10203000938329490B919F0600F1E8820798DE06F9
:10204000014600F170825D0640F16D820431068820
:1020500007910027D80740F1228256EA070100F0D5
:102060001E8230218DF8392043F002038DF838109C
:10207000022264E60896002840F06B8317490B9112
:10208000D9E7079908960A688DF848204FF00000B4
:102090000A468DF83700043201200190079205901E
:1020A0000DF1480B0293002470E643F0400398F8CA
:1020B000002083E598F800206C2A03BF98F80120DF
:1020C00043F0200308F1010843F0100376E500BF58
:1020D00098494100A84941007C49410068494100B4
:1020E00007990E680A46002E02F10402FFF60FAEB1
:1020F000079298F8002061E598F8002001202B2530
:102100005CE507990896D1F800B04FF000028DF811
:1021100037200E1DBBF1000F00F0E582671C00F0B8
:10212000C4822246002158460193FFF739F9019BEA
:10213000002800F0E582A0EB0B02059207960293BF
:102140009DF83750002419E698F800202A2A08F153
:10215000010700F0E982A2F130010929B8464FF0E9
:1021600000043FF62DAD18F8012B04EB840401EBBD
:102170004404A2F130010929F5D921E543F02003F7
:1021800098F800201AE50896002840F0DB82002A23
:1021900000F0E78001218DF848204FF00002019106
:1021A0008DF8372005910DF1480B7BE7079A1368EE
:1021B00004320792039A1A60CBE40FAA04992046CE
:1021C000FFF74AFC002840F039811099119A01F17B
:1021D000010CCE46FFE51099119A481C9DF8375026
:1021E000002D3FF422AE01320DF137050121072801
:1021F00011921090CAF80050CAF8041040F30881F8
:10220000002A40F0BC81099B002B3FF41FAE0EABAF
:10221000022208461C931D92CA4601460AF1080A8A
:1022200001300A9B802B3FF419AE059BE41A002C69
:102230002EDD102CB34D1EDDD6461026069FDDF890
:1022400010A006E0881C0EF1080E1946103C102C58
:1022500010DD4B1C1032072B11928EE8600010939A
:10226000F0DD002A65D1103C102C4FF00100114622
:10227000CE46EEDCF246224407281192CAF80050FE
:10228000CAF80440109000F385800AF1080A013072
:102290000599CAF800B00A4407281192CAF8041038
:1022A000109040F38280002A40F01881029B109227
:1022B000580735D5089B01995C1A002C40F3E7803C
:1022C000CA46102C40F3188210998F4E069FDDF8F5
:1022D00010B0102506E0881C0AF1080A1946103CC7
:1022E000102C11DD4B1C1032072B1192CAF8006024
:1022F000CAF804501093EEDD42BB103C102C4FF096
:1023000001001146CA46EDDC224407281192CAF8A2
:102310000060CAF80440109051DD002A40F09B8113
:10232000039B089A01998A42ACBF9B185B180393E0
:102330004EE00FAA51463846FFF78EFB002840F0CA
:102340003F811099119A481CCE467FE70FAA594643
:102350003846FFF781FB60B91099119A481CCA46AC
:10236000BDE7119BDDF810B0002B40F0D4810023B5
:102370001093DBF8643013F0010FBBF80C3002D17E
:102380009A0540F1DE805B063FF5B2AC03982DB0B4
:10239000BDE8F08F002A40F00681059A1D920123C6
:1023A0001192CDF870B01093CA460AF1080A029B48
:1023B000590704D5089B01995C1A002C81DC039B0A
:1023C000089901988142ACBF5B181B18039372BB3C
:1023D00000231093CA46FFF7BCBB0FAA04992046FE
:1023E000FFF73AFB50BB1099119A01F1010ECC4650
:1023F00048E5002A40F040819DF83710002900F0A0
:102400001B8101220DF1370110461D921C91CA4615
:1024100001460AF1080A013007E5029B012A00F093
:102420009880022A0DD1029300260027B0E50FAA5A
:1024300004990698FFF710FB0028C9D0DDF810B00A
:1024400097E7029300260027494600E05946F20824
:1024500042EA4772F80806F007030746164630338B
:1024600056EA070201F8013C01F1FF3BEED1029A66
:10247000D6077FF59DAD302B3FF49AAD023930235E
:102480000BF8013CA9EB010305938B4676E4039B13
:10249000089A8A42ACBF9B185B18039398E7022204
:1024A0004DE4002F08BF0A2E52D3CB4630463946A2
:1024B0000A22002301F010FB30320BF8012D3046C8
:1024C000394600230A2201F007FB06460F4656EA6A
:1024D0000703EBD16CE50594CB464FE40FAA0499B2
:1024E0000698FFF7B9FA0028A8D1119ACA465EE704
:1024F0000FAA04990698FFF7AFFA00289ED1CA46A2
:10250000FFF7C0BBA8494100984941000431166853
:1025100007910122002712E407980146043106685A
:10252000079100270BE40E6804310791002791E51D
:1025300007990E680A46F717043207923046394663
:102540000FE5DBF8580000F07FFEBBF80C301AE70F
:10255000029B02930DF1B00B303601230BF8416D55
:1025600005930BE40FAA04990698FFF775FA002863
:102570007FF464AF1099119A481CCA4651E60FAA1D
:1025800004990698FFF768FA00287FF457AF10996E
:10259000119A481CCA4648E4002A40F09180012064
:1025A0001146CA4641E60FAA04990698FFF754FA65
:1025B00000287FF443AF1098119A0130CA4667E6AD
:1025C000D346D6E6079E073626F0070202F1080139
:1025D000D2E9006707910122FFF7B1BB079E0736DA
:1025E00026F00706D6E9000106F108020792064622
:1025F0000F46B6E4079E073626F0070202F10801EF
:10260000D2E9006707910022FFF799BB079E0736C2
:1026100026F0070101F108000790D1E9006719E5EC
:10262000CB46FFF7ABBB2D25764267EB47078DF80E
:1026300037500122FFF788BB099BB3B9114601202F
:10264000CA46F2E5DBF8580000F0FEFD4FF0FF331C
:102650000393FFF750BB0FAA04990698FFF7FCF904
:1026600000287FF4EBAE119AA9E60EAB02221C9370
:102670001D920120CA46D0E50FAA04990698FFF7DB
:10268000EBF900287FF4DAAE1099119A481CCA467B
:10269000A4E5079A03991368CD1708460432294622
:1026A0000792C3E90001FFF754BA58460796029310
:1026B000FFF746F9002405909DF83750FFF75EBB01
:1026C0000FAA04990698FFF7C7F900287FF4B6AE61
:1026D0001099119A481CCA46A7E51099119A204EE4
:1026E0000131FFF790BB062C28BF062405940796FE
:1026F0000194DFF870B0D5E41098194E013003E66C
:1027000005949DF83750079602930446FFF736BBB1
:102710008646FFF7CEBB06980FAA5946FFF79CF9ED
:1027200000283FF424AE24E6079998F801200C68AD
:10273000043144EAE474B8460791FFF73FBA8DF8D4
:1027400037503CE48DF8375021E58DF83750FFF7CE
:10275000F4BB8DF8375091E48DF8375069E400BF31
:1027600098494100904941002DE9F0410C46ADF5F2
:102770008D6D8989666EE589199621F002010646FC
:10278000E069ADF80C1017464FF48061626AADF84D
:102790000E5098461AAD0023079016A8099206938A
:1027A000009504950291059100F048FD43463A4694
:1027B00069463046FFF790F9051E07DB304669464B
:1027C00000F028F9002818BF4FF0FF35BDF80C3095
:1027D0005B0603D5A38943F04003A381169800F05C
:1027E0002FFD28460DF58D6DBDE8F08138B5304BD5
:1027F0001B6805460C4613B19A6B002A38D0B4F911
:102800000C2093B218070CD52069A8B113F001026F
:102810001ED0636900225B42A361A260F0B1002078
:1028200038BDD9063CD5580726D4206942F00803A4
:10283000A3819BB20028E9D103F42072B2F5007F96
:10284000E4D02846214600F02FFDA3892069DDE76A
:10285000990758BF6269A2600028E0D1B4F90C3032
:102860001A06DDD543F04003A3814FF0FF3038BD99
:10287000184600F027F9C2E7216B51B104F140037B
:10288000994204D0284600F043FAB4F90C20002302
:10289000236300232069636022F024022060C5E7DF
:1028A00042F0400209232B604FF0FF30A28138BD77
:1028B0003C030020024B13B1024800F005B87047FA
:1028C00000000000352B4100002301461A4618463F
:1028D00000F0DABFB1F90C309AB22DE9F0410D46A3
:1028E000110780463AD46A6843F40063002AAB813A
:1028F0006FDDAC6A002C49D000229BB2D8F8006092
:10290000C8F8002013F4805267D02A6D5F0705D500
:1029100069682B6B521A0BB1EB6BD21A0023E96971
:102920004046A047441C3CD0B5F90C302A692A60C7
:1029300023F400630022AB81DB046A6047D4296B77
:10294000C8F8006011B305F14003994202D0404637
:1029500000F0DEF900202863BDE8F0812E69AEB1F9
:102960002C682E6091070CBF6B690023A41BAB6021
:102970000AE0234632466F6AE9694046B8470028B4
:10298000A4EB0004064404DD002CF2DC0020BDE8CA
:10299000F081AB8943F04003AB814FF0FF30BDE8DD
:1029A000F081D8F800401D2CF3D8194BE340DB43ED
:1029B00013F00103EDD1B5F90C206B6022F4006334
:1029C0002969AB81DA042960B9D5002CB7D1286513
:1029D000B5E7EA6B002A8CDCD8E70123E9694046B9
:1029E000A047431C024602D0AB89AC6A8EE7D8F8F8
:1029F0000030002BF8D01D2B01D0162B02D1C8F8C7
:102A00000060C3E7AB8943F04003AB81BDE8F081D0
:102A10000100402038B50D46044608B1836BBBB1B8
:102A2000B5F90C0088B16B6EDB0701D4810517D5B1
:102A300020462946FFF74EFF6B6EDA07044602D4A4
:102A4000AB899B0507D5204638BD0446204638BDD6
:102A500000F038F8E4E7A86D00F0F6FB204638BD3A
:102A6000A86D00F0EFFBE3E7014900F0AFBB00BF4A
:102A70007139410010B5002304468181C281036091
:102A800043608360436603614361836119460822A2
:102A90005C30FEF703FE07480749084A084B2062EE
:102AA000E4616162A262E36204F15800BDE8104093
:102AB00000F0C4BBB5364100D9364100153741009E
:102AC0003537410010B50446124800F0BBFBA26B3D
:102AD000D2B904F53B731048C4F8E8320321C4F8B6
:102AE000E022E063C4F8E41260680421FFF7C2FF4B
:102AF00001220921A068FFF7BDFF02221221E06830
:102B0000FFF7B8FF0123A3630248BDE8104000F0BF
:102B10009BBB00BF60230020692A4100014800F0F0
:102B200091BB00BF74230020014800F08DBB00BFA3
:102B30007423002038B50A4C0A4D641BA4100AD037
:102B400004F18043013B05EB8305013C55F8043952
:102B50009847002CF9D1BDE8384001F0C1BF00BF53
:102B6000F04A4100EC4A41002DE9F04782B080462E
:102B70008946144600F054FB012836D04A4604F139
:102B80005C0301A9404600F031FE421C064625D0F8
:102B9000A8B39DF804E000250DF1040A09E02368BC
:102BA0005A1C226083F800E00135B54227D215F89F
:102BB0000AE0A368013B002BA360F0DAA769BB42DF
:102BC00071462246404602DBBEF10A0FE7D100F013
:102BD000B5FD431CE8D102B0BDE8F087A38943F0FE
:102BE0004003A38102B0BDE8F08709F1FF33FE2B5B
:102BF000C4D85FFA89FE06468DF804E0CBE7484664
:102C000002B0BDE8F08700BF30B5536E13F0010F7E
:102C1000B2F90C30144683B005469AB201D1900542
:102C20001CD5900406D4626E43F4005342F4005263
:102C3000A381626628462246FFF796FF636EDA0795
:102C4000054602D4A3899B0502D5284603B030BDB2
:102C5000A06D00F0F9FA284603B030BDA06D0191D7
:102C600000F0F0FAB4F90C3001999AB2D9E700BF3C
:102C7000F8B5244F0C460646FEF75EFDBB685D685E
:102C8000C4F57E610F3125F00305294421F47F61ED
:102C900021F00F01A1F58054B4F5805F07DB00211E
:102CA0003046FEF755FDBB682B44984204D03046B1
:102CB000FEF748FD0020F8BD61423046FEF748FDB2
:102CC00001300DD0104BBA6819682D1B45F0010575
:102CD0003046091B55601960FEF734FD0120F8BD30
:102CE00000213046FEF734FDBA68831A0F2BDEDD73
:102CF000064C0549246843F00103001B536008603B
:102D0000D5E700BF6807002038100020700B0020B6
:102D1000002944D02DE9F0410D468046FEF70CFD18
:102D200055F8047C694927F00103A5F10804E2186D
:102D30008E685068B24220F003005ED0FE075060FB
:102D40000BD455F8087CE41B01F1080EA568754505
:102D50003B446DD0E768EF60BD6015186D68ED0706
:102D60003ED543F001026260E350B3F5007F17D215
:102D7000DB08581C9A104D6851F83070A760012389
:102D8000934001EBC0022B43083AE2604B6041F8EC
:102D90003040FC604046BDE8F041FEF7D3BC7047D0
:102DA0005A0A042A52D89A0902F13907FF0002F19F
:102DB0003805C819CA59083890424FD0516821F0D7
:102DC00003018B4232D292689042F7D1C368A0606F
:102DD000E3609C60C4604046BDE8F041FEF7B2BCD1
:102DE00095683B4FBD42034440D0D068E86043F053
:102DF000010285606260E350B7E7FF07034407D430
:102E000055F8082CA41A1344A068E268C2609060C8
:102E1000304A126843F00100934260608C60B9D37D
:102E20002D4B40461968FFF723FFB3E71046CDE767
:102E300011184968C90744D49168D268CA6003442C
:102E400043F0010091606060E350A3E7142A16D8B4
:102E500002F15C07FF0002F15B05AAE7AA1001235B
:102E60004D6893402B434B600346B0E743F00102AB
:102E70004C610C61E560A5606260E3508AE7542A0A
:102E800006D81A0B02F16F07FF0002F16E0590E7FA
:102E9000B2F5AA7F06D8DA0B02F17807FF0002F13B
:102EA000770586E740F25450824206D89A0C02F128
:102EB0007D07FF0002F17C057BE74FF47E777E25DE
:102EC00077E743F001016160136063E76807002062
:102ED00070070020740B0020681000209368002BFE
:102EE00073D02DE9F04F8B8983B00C461907009001
:102EF000164626D5226922B313F0020035682CD07D
:102F00004FF00009B04FC846B246B84543464A465E
:102F100028BF3B460098B8F1000F50D0E169666ABF
:102F2000B047002858DDDAF808301B1A8144A8EBB6
:102F30000008CAF80830002BE7D1002003B0BDE834
:102F4000F08F21460098FFF751FC002840F03381B4
:102F5000A389356813F00200D2D113F0010945D1DD
:102F60004F46019637B39A05D4F8088040F1838024
:102F70004745C346C0F0AB8013F4906F40F0AC807F
:102F80002068BA465A464946FEF724FBA2682368E1
:102F9000A2EB08025B44A2602360019A9368A3EB52
:102FA0000A03D144A7EB0A079360002BC5D0A3897D
:102FB000002FD8D1D5F800906F680835D2E7D5F842
:102FC0000090D5F8048008359FE70020704721461F
:102FD0000098FFF71FFD70B3B4F90C3043F04003C5
:102FE0004FF0FF30A38103B0BDE8F08F8146334638
:102FF0004E46A8469A464D464EB380B32068236994
:103000006269B145CB4628BFB34698425F4604D9B2
:10301000A36813449B4500F3A68093454BDB1346FE
:10302000676AE16900982A46B847071ED4DDB9EB04
:103030000709CCD00120DAF80830DB1B3D44F61B31
:10304000CAF80830002B3FF478AF002ED5D108F134
:10305000080313E9600098460833002EF9D0324681
:103060000A212846FEF79CF9002800F0A1800130D3
:10307000A0EB0509C2E720682369984202D863697A
:103080009F425DD2B84528BFB84642464946FEF742
:10309000A1FAA3682268A3EB08034244A36022605C
:1030A0000BB1C24679E721460098FFF7B3FC002830
:1030B00092D1C24671E75A462946FEF78BFAA268BA
:1030C0002368A2EB0B025B44A2602360AFE7206899
:1030D000B846BA46BB4655E762692068216902EBEB
:1030E0004208A0EB010A08EBD8780AF101004FEA88
:1030F000680838444045424684BF804642465B05E6
:1031000044D511460098FDF799FE8346002855D016
:1031100052462169FEF7C4F9A38923F4906343F072
:103120008003A3810BEB0A00A8EB0A03C4F810B0DC
:10313000C4F814802060A360B846BA46BB4621E7B5
:103140006FF00041B94228BF39464A4691FBF3F17E
:103150000098666A03FB01F3E169B047B0F1000A29
:103160003FF71BAF38E71A4629460193FEF732FABC
:103170002268019B00981A4422602146FFF74AFC0E
:10318000019B00287FF428AF1F4650E7009800F00D
:10319000EBF883460028C5D1009D21692846FFF73A
:1031A000B7FDB4F90C300C2223F080032A6015E738
:1031B00006F1010922E74FF0FF30BFE6009A0C2329
:1031C0001360B4F90C3009E700FCFF7F2DE9F843E8
:1031D00010F538771FD0884606464FF000097D6805
:1031E000BC68013D11D4A389012B05F1FF3508D935
:1031F000B4F90E3001332146304602D0C04749EAC7
:1032000000096B1C04F16804EDD13F68002FE6D182
:103210004846BDE8F883B9464846BDE8F88300BF94
:10322000044B054A1B685B6B002B08BF134693F8E1
:10323000280170473C0300207C0B0020704700BF32
:10324000704700BF704700BF704700BF70B50C46A5
:10325000B1F90E10002990B015461E4614DB01AAE4
:1032600000F0E8FB00280FDB029A02F47042A2F59E
:103270000052B2FA82F252094FF480634FF40060B8
:1032800032602B6010B070BDA289002312F0800064
:10329000336004D0402218462A6010B070BD4FF44D
:1032A00080632B6010B070BD8A8992070B4606D5EB
:1032B00001F1430201211A601A6159617047F0B5AA
:1032C00083B001AB6A460C460646FFF7BFFF009984
:1032D00005463046FDF7B2FDB4F90C30D8B1019A7D
:1032E000154F0099F76343F08003A38120602061AC
:1032F00061611AB92B43A38103B0F0BD3046B4F924
:103300000E1000F0ABFBA0B1A38923F0030343F040
:1033100001031BB2EEE79A05EED423F0030304F198
:10332000430243F002030121A38122602261616113
:10333000E2E7B4F90C30DDE7692A410082B049B117
:103340005AB16BB113780B601278101C18BF0120B2
:1033500002B0704701A9002AF3D1104602B07047AD
:103360006FF00100F4E700BF002900F095802DE91F
:10337000F04F0D46164683B0804606F10B07FEF768
:10338000DBF955F804EC162F2EF00304A5F108091B
:103390003CD810221746BE423DD8944243DAC44B73
:1033A000996809EB0400884200F0B480436823F078
:1033B000010101444968C9074CD51EF0010F00F016
:1033C0009B8031464046FDF739FD064600283AD03D
:1033D00055F8043C23F001034B44A0F108029A4243
:1033E00000F02181221F242A00F20781132A00F213
:1033F000DB8003462A46116819605168596092685B
:103400009A6029464046FFF783FC1CE027F0070737
:10341000002F3A46BFDA00260C233046C8F80030A9
:1034200003B0BDE8F08F2E46E31B0F2B1ED8D9F852
:10343000043003F0010323434C44C9F804306368AB
:1034400043F0010363604046FEF77CF9304603B069
:10345000BDE8F08F23F00303E11891421FDBC3683E
:1034600082682E46D3600C469A60DDE7D9F80420C6
:1034700009EB070102F001024C4443F0010317433A
:10348000C9F804704B60636843F00103083163605E
:103490004046FFF73DFCD6E71146FDF7CFBC1EF0D6
:1034A000010F8ED155F8081CA9EB010ADAF80410B7
:1034B00021F003010B442344934225DBC268816859
:1034C0005646CA609160DAF80C1056F8080F221FB1
:1034D000242AC160886000F29480132A6FD9296879
:1034E000CAF808106968CAF80C101B2A00F2A280FA
:1034F00008350AF1100263E055F8083CA9EB030A0D
:10350000DAF8041021F0030163189342FFF659AF73
:103510005646D8E7416821F0030BA34407F1100099
:10352000834556DA1EF0010F7FF44BAF55F8081CA7
:10353000A9EB010ADAF8041021F003018B44584585
:10354000E2DC5646DAF80C1056F8080F221F242A3F
:10355000C160886000F28F80132A40F28A80296857
:10356000CAF808106968CAF80C101B2A00F28A8091
:1035700008350AF110022968116069685160A9686C
:1035800091600AEB0701ABEB070242F00102996080
:103590004A60DAF8043003F001031F434046CAF8DA
:1035A0000470FEF7CFF851E72B6803606B68436047
:1035B0001B2A2DD800F1080305F108021BE732464B
:1035C0002968116069685160A96891601C46D146FC
:1035D0002AE709EB0701ABEB070B4BF001029960FF
:1035E0004A6055F8043C03F001031F43404645F888
:1035F000047CFEF7A7F82E4628E72946FDF7EAFFE8
:10360000FFE6294630461C46D146FDF7E3FF0BE7AF
:10361000AB688360EB68C360242A17D000F1100305
:1036200005F11002E7E650F8043C23F003031C44C4
:103630002E46F9E6A968CAF81010E968CAF814100D
:10364000242A0CD010350AF11802B9E72B6903615E
:103650006B69436105F1180200F11803CBE62A6992
:10366000CAF818206A69CAF81C2018350AF1200225
:10367000A6E732467FE7294630460193FDF7AAFFC9
:10368000019B7EE7A968CAF81010E968CAF814100F
:10369000242A03D010350AF118026CE72A69CAF807
:1036A00018206A69CAF81C2018350AF1200262E75E
:1036B0006807002010B50C46B1F90E1000F0F6F9BD
:1036C000002803DB236D0344236510BDA38923F485
:1036D0008053A38110BD00BF2DE9F0411646B1F91A
:1036E0000C201F46D3050C46054607D500220223B1
:1036F000B1F90E1000F0C4F9B4F90C20B4F90E10B1
:1037000022F48052A2813B4632462846BDE8F04171
:1037100000F0A4B810B50C46B1F90E1000F0B0F9E5
:10372000A389421C0EBF23F4805343F480532065C9
:10373000A38110BDB1F90E1000F008B9F8B50D461F
:103740001446064610B1836B002B4BD0B4F90C2005
:10375000A369A36091B2080739D52369002B36D03D
:10376000EDB289042F4615D522686169D31A8B42C0
:103770001CDA0133A168501C0139A160206015706A
:1037800062699A421AD0A389DB0701D50A2D15D0A8
:103790003846F8BD616E42F4005221F40051A28116
:1037A000226861666169D31A8B42E2DB21463046AA
:1037B000FFF730F940B922680123DBE721463046A4
:1037C000FFF728F90028E3D04FF0FF37E0E7214664
:1037D0003046FFF70BF80028F6D1B4F90C20236926
:1037E00091B2BDE7FFF76EF9B0E700BFF0B506464E
:1037F00085B01F4689B1104C104D2468646B002CB5
:1038000008BF2C46D4F8E040A047431C03D1002257
:103810008A233A60336005B0F0BD0C460649074A7A
:103820000968496B002908BF11462246D1F8E040DB
:1038300001A9A047E9E700BF3C0300207C0B002062
:1038400021B1FF2A04D80A7001207047084670474A
:103850008A2303604FF0FF30704700BF70B50D46FC
:10386000084C114606461A46284600232360F9F7FD
:10387000F1FD431C00D070BD2368002BFBD03360EA
:1038800070BD00BF782300202DE9F8432C4D06467B
:10389000286898460F469146FFF7D4FC294B1C68D0
:1038A000D4F84831002B3ED05A681F2A1CDC02F1A4
:1038B000010E76B103EB82010124C1F88890D3F8A0
:1038C000880194402043022EC3F88801C1F8088182
:1038D00023D00232C3F804E0286843F82270FFF7CF
:1038E000B3FC0020BDE8F883174B0BB34FF4C8704E
:1038F000FDF794FA0346D8B1D4F8482102600021BC
:1039000041600A46C4F848014FF0010EC0F8881122
:10391000C0F88C11002EDCD0CCE7D3F88C110C430E
:10392000C3F88C41D5E704F5A673C4F84831BBE76A
:103930002868FFF789FC4FF0FF30BDE8F88300BF2F
:10394000780B0020644941001D0E410038B5074C3A
:103950000023054608462360FAF78AF9431C00D085
:1039600038BD2368002BFBD02B6038BD78230020A6
:1039700070B559B105460C4610B1836B002B3CD095
:10398000636ED80705D5B4F90C302BB90026304644
:1039900070BDA38999053CD521462846FEF79AFFBC
:1039A000E36A064633B1E169284698470028B8BF64
:1039B0004FF0FF36A3891A0622D4216B41B104F1DE
:1039C0004003994202D02846FFF7A2F9002323635F
:1039D000616C21B12846FFF79BF900236364FFF770
:1039E0009DF8636E0022DB07A2810ED5A06DFFF764
:1039F00027FCFFF799F8304670BDFFF763F8BFE783
:103A000021692846FFF784F9D7E7A06DFFF71CFC72
:103A1000ECE7A06DFFF716FCB4F90C30002BBBD11E
:103A2000666E16F00106B1D1A06DFFF70DFC3046B1
:103A300070BD00BF38B50B46074C05461146184609
:103A400000232360FAF717F9431C00D038BD236820
:103A5000002BFBD02B6038BD7823002038B5074CF5
:103A60000023054608462360FAF70AF9431C00D0F4
:103A700038BD2368002BFBD02B6038BD7823002095
:103A800070B50D46084C114606461A4628460023D6
:103A90002360FAF7F7F8431C00D070BD2368002BB1
:103AA000FBD0336070BD00BF7823002070B50D4699
:103AB000084C114606461A46284600232360F9F7AB
:103AC000AFFC431C00D070BD2368002BFBD03360DB
:103AD00070BD00BF7823002053B94AB9002908BF40
:103AE00000281CBF4FF0FF314FF0FF3000F07AB9D3
:103AF000ADF1080C6DE904CE00F006F8DDF804E045
:103B0000DDE9022304B070472DE9F0478C460D46ED
:103B10000446089E002B51D18A4217466DD9B2FA4D
:103B200082FEBEF1000F0BD0CEF1200C01FA0EF593
:103B300020FA0CFC02FA0EF74CEA050C00FA0EF41F
:103B40004FEA174A250CBCFBFAF81FFA87F90AFB63
:103B500018CC45EA0C4508FB09F3AB420AD9ED192C
:103B600008F1FF3280F02381AB4240F22081A8F1BE
:103B700002083D44ED1AA4B2B5FBFAF00AFB105559
:103B800044EA054400FB09F9A14509D9E41900F10B
:103B9000FF3380F00A81A14540F2078102383C449E
:103BA000A4EB090440EA08400021002E61D024FA69
:103BB0000EF4002334607360BDE8F0878B4207D9B0
:103BC000002E54D0002186E821000846BDE8F08789
:103BD000B3FA83F1002940F08E80AB4202D38242D7
:103BE00000F2FA80841A65EB03050120AC46002E32
:103BF0003FD086E81010BDE8F08712B90127B7FB67
:103C0000F2F7B7FA87FEBEF1000F34D1EB1B3A0C86
:103C10001FFA87FC0121B3FBF2F8250C02FB1833D5
:103C200045EA03450CFB08F3AB4207D9ED1908F14F
:103C3000FF3002D2AB4200F2D1808046ED1AA3B22F
:103C4000B5FBF2F002FB105543EA05440CFB00FC07
:103C5000A44507D9E41900F1FF3302D2A44500F2CC
:103C6000B8801846A4EB0C0440EA08409DE73146B2
:103C70003046BDE8F087CEF1200405FA0EF307FACE
:103C80000EF720FA04F83A0C25FA04F448EA03087F
:103C9000B4FBF2F14FEA184502FB11441FFA87FC0E
:103CA00045EA044501FB0CF3AB4200FA0EF409D9D6
:103CB000ED1901F1FF3080F08A80AB4240F287803D
:103CC00002393D44EB1A1FFA88F5B3FBF2F002FB10
:103CD000103345EA034500FB0CF3AB4207D9ED195D
:103CE00000F1FF386FD2AB426DD902383D44EB1A78
:103CF00040EA01418FE7C1F1200722FA07F88B4023
:103D000005FA01F448EA030320FA07FE4FEA134CD0
:103D1000FD404EEA040EB5FBFCF94FEA1E440CFBD5
:103D200019551FFA83F844EA054509FB08F4AC422B
:103D300002FA01F200FA01FA08D9ED1809F1FF3090
:103D400043D2AC4241D9A9F102091D442D1B1FFAEF
:103D50008EFEB5FBFCF00CFB10554EEA054400FB53
:103D600008F8A04507D9E41800F1FF3529D2A0458D
:103D700027D902381C4440EA0940A4EB0804A0FB00
:103D800002894C45C6464D4615D312D056B1BAEB02
:103D90000E0364EB050404FA07F7CB401F43CC4045
:103DA000376074600021BDE8F0871846F8E6904659
:103DB000E0E6C245EAD2B8EB020E69EB0305013832
:103DC000E4E72846D7E7404691E78146BEE701464B
:103DD00078E702383C4445E7084608E7A8F10208BE
:103DE0003D442BE7704700BF0100000002000000C7
:103DF0000400000008000000100000002000000087
:103E00004000000080000000000080000000000171
:103E10000000000200000004000000080000001084
:103E20000000000000000000000000000000000092
:103E30000000000000000000000000000000000082
:103E400000000000000000000128011002038002B1
:103E500053290351FF01026902026B1005800040E3
:103E60004011088102560009000F00088202560026
:103E700009000F0002350002250103F0AA1104C059
:103E80000040000AC2010A010A010A00900203FF71
:103E90005A8102650B0EF9585F666D747B828990BA
:103EA000979EA5AC03F0AA1202D32003BF37BE022F
:103EB000360003F0AA1104C50001400001280110DA
:103EC0000253290351FF01026902026B10058001B0
:103ED00040401103F0AA1104C00040000AC2010AC8
:103EE000010A010A0090022D70110000891080075C
:103EF0008003C0078003C003C0020003580020C62F
:103F000037000D000F00110008180010F0030C20FE
:103F100000060B0B3308810256000B0011000882CB
:103F20000256000B00110002350002250103F0AA21
:103F30001002D10203F0AA110AC2010A010A010A01
:103F400000900203FF5A8102650B0EF9585F666DFF
:103F5000747B828990979EA5AC03F0AA1202D320AD
:103F600003BF37BE02038102360003F0AA1104C565
:103F7000000140000128011002038002532903516F
:103F8000FF01026900026B100580004040110881AA
:103F900004AC0010001000088204AC0010001000F7
:103FA00002350002250103F0AA1002D10203F0AA93
:103FB000110AC2010A010A010A00908203F0AA1242
:103FC00002D32003BF07BE03FF5A8102650B0EF91F
:103FD000585F666D747B828990979EA5AC0236000F
:103FE0000000000001010203800253290351FF0178
:103FF000026900026B1005800040401108810256E2
:10400000000A00100008820256000A001000023563
:104010000002250103F0AA110AC2010A010A010ADD
:1040200000900203F0AA1202D32003BF07BE03FFD1
:104030005A8102650B0EF9585F666D747B82899018
:10404000979EA5AC03F0AA1105C4AA55018004C52A
:10405000001FFF00012801100203810253290351B0
:10406000FF01026900026B102D70110000891080A1
:1040700009F004F804F804F804F80200041B002016
:1040800091BF0011000F00190009180010F0030C77
:104090002000060B0B330580013E3E11088101E133
:1040A0000006001000088201E10006001000022551
:1040B0000103F0AA1002D10203F0AA110AC2010AF8
:1040C000010A010A00900203F0AA1202D32003BFE2
:1040D00007BE03FF5A8102650B0EF9585F666D74C7
:1040E0007B828990979EA5AC0000000001280110FA
:1040F0000203810253290351FF01026900026B1080
:104100002D7011000089108009F004F804F804F8FB
:1041100004F80200041B002091BF0011000F0019D9
:104120000009180010F0030C2000060B0B3305806B
:10413000013E3E11088101E10010001000088201DB
:10414000E1001000100002250103F0AA1002D102C4
:1041500003F0AA110AC2010A010A010A009002032F
:10416000F0AA1202D32003BF07BE03FF5A810265E3
:104170000B0EF9585F666D747B828990979EA5AC93
:10418000000000005658523030000000302E322E11
:104190003136000055534152540000004661696CAD
:1041A000656420746F206372656174652075736146
:1041B0007274207461736B0D0A000000484944203A
:1041C000436F6D6D616E6473000000004661696C41
:1041D000656420746F20637265617465204849448A
:1041E00020636F6D6D616E642070726F63657373B1
:1041F0006F72207461736B0D0A00000048494420FF
:104200005265706F727400004661696C6564207459
:104210006F2063726561746520484944207065723F
:10422000696F646963207265706F72742074617362
:104230006B0D0A00302E322E313600005658524493
:10424000454C45544500000043524153484E4F579A
:104250000000000000FFFFFFFFFFFF00092795504F
:10426000D2040000021E0104A5000078E70000004F
:104270000000000000000000000001010101010138
:1042800001010101010101010101CAB40080F080B6
:10429000187040209200FFFF0000001EA551008012
:1042A000A00020A040200204FFFF0000001E00002C
:1042B00000000000000000000000000000000000FE
:1042C00000000010000000000000000000000000DE
:1042D000000001757012790000030014689F0080CF
:1042E000FF137F003F801F00FF091F000F800100A8
:1042F00000000000000000000000000000000000BE
:1043000000000000000000000000000000000000AD
:10431000000000000000000000000000000000009D
:10432000000000000000000000000000000000008D
:10433000000000000000000000000000000000007D
:10434000000000000000000000000000000000006D
:104350000000B19000FFFFFFFFFFFF0009273412AC
:10436000D2040000FF200104A5000078007875AA9F
:10437000553BB22910505400000001010101010118
:104380000101010101010101010100000010000013
:10439000000000000000000000000000000000100D
:1043A000000000000000000000000000000000000D
:1043B00000100000000000000000000000000000ED
:1043C000000000FC004265796F6E640A2020202006
:1043D0002020015B702079070022091441B70E8864
:1043E000DF137F003F801F00EF0917000E800100E0
:1043F0007E00073A029281000800000000000000E1
:1044000000000000000000000000000000000000AC
:10441000000000000000000000000000000000009C
:10442000000000000000000000000000000000008C
:10443000000000000000000000000000000000007C
:10444000000000000000000000000000000000006C
:104450000000CA9000FFFFFFFFFFFF000927341292
:10446000D2040000FF200104A5000078007875AA9E
:10447000553BB22910505400000001010101010117
:104480000101010101010101010100000010000012
:10449000000000000000000000000000000000100C
:1044A000000000000000000000000000000000000C
:1044B00000100000000000000000000000000000EC
:1044C000000000FC004265796F6E640A2020202005
:1044D0002020015B702079070022091439540F88CD
:1044E000DF137F003F801F00EF0917000E800100DF
:1044F0007E00073A029281000800000000000000E0
:1045000000000000000000000000000000000000AB
:10451000000000000000000000000000000000009B
:10452000000000000000000000000000000000008B
:10453000000000000000000000000000000000007B
:10454000000000000000000000000000000000006B
:104550000000349000FFFFFFFFFFFF000927341227
:10456000D2040000FF200104A5000078007875AA9D
:10457000553BB22910505400000001010101010116
:104580000101010101010101010100000010000011
:10459000000000000000000000000000000000100B
:1045A000000000000000000000000000000000000B
:1045B00000100000000000000000000000000000EB
:1045C000000000FC004265796F6E640A2020202004
:1045D0002020015B70207907002209141EF50A884B
:1045E000FF0EFF003F801F007F071B000E800100B1
:1045F0007E00073A029281000800000000000000DF
:1046000000000000000000000000000000000000AA
:10461000000000000000000000000000000000009A
:10462000000000000000000000000000000000008A
:10463000000000000000000000000000000000007A
:10464000000000000000000000000000000000006A
:104650000000869000FFFFFFFFFFFF0009273412D4
:10466000D2040000FF200104A5000078007875AA9C
:10467000553BB22910505400000001010101010115
:104680000101010101010101010100000010000010
:10469000000000000000000000000000000000100A
:1046A000000000000000000000000000000000000A
:1046B00000100000000000000000000000000000EA
:1046C000000000FC004265796F6E640A2020202003
:1046D0002020015B702079070022092839540F88B7
:1046E000DF137F003F801F00EF0917000E800100DD
:1046F0001EF50A08FF0EFF003F801F007F071B000A
:104700000E8001007E00073A02928100080000003E
:104710000000000000000000000000000000000099
:104720000000000000000000000000000000000089
:104730000000000000000000000000000000000079
:104740000000000000000000000000000000000069
:104750000000E190766964656F5F70726F630000BE
:104760004661696C656420746F206372656174656D
:1047700020766964656F2070726F636573736F7202
:10478000207461736B0D0A0070726F785F74696DCD
:10479000656F75745F74696D65720000FF00FF00DE
:1047A000493243004661696C656420746F2063720E
:1047B0006561746520493243207461736B0D0A0092
:1047C00054494D45445F5354415254004661696C0D
:1047D000656420746F206372656174652074696D0F
:1047E00065642073746172747570207461736B0DED
:1047F0000A000000414443004661696C656420740E
:104800006F20637265617465204144432074617355
:104810006B0D0A004C4544004661696C6564207468
:104820006F20637265617465204C45442074617328
:104830006B0D0A0046414E004661696C6564207448
:104840006F206372656174652046616E20746173C8
:104850006B0D0A003132333420202020202020200C
:10486000202020200000000049444C4500000000AA
:10487000546D725100000000546D72205376630035
:1048800000C20100C000000000080000000000009D
:104890002D2D2042696773637265656E20426579CC
:1048A0006F6E64202D2D0A00444953504C415942EB
:1048B0004F4152442056302E342E32002D2D2025CB
:1048C00073202D2D0A0000002D2D2056657273696E
:1048D0006F6E202573202D2D0A00000031363A30EE
:1048E000373A3436000000004F63742031302032F4
:1048F000303233002D2D20436F6D70696C65643A42
:10490000202573202573202D2D0A00005553424C7D
:104910006F6164004661696C656420746F20637226
:104920006561746520555342204C6F616465722047
:104930007461736B0D0A000048494420436F6D6D2C
:10494000616E6400737461636B206F766572666C70
:104950006F772025782025730D0A00006C6F67663D
:104960000000000040030020303132333435363748
:10497000383941424344454600000000303132336B
:10498000343536373839616263646566000000008B
:10499000286E756C6C29000020202020202020200B
:1049A0002020202020202020303030303030303087
:1049B000303030303030303043000000504F5349F9
:1049C000580000002E000000002020202020202081
:1049D00020202828282828202020202020202020AF
:1049E00020202020202020202088101010101010BF
:1049F000101010101010101010040404040404040B
:104A000004040410101010101010414141414141A4
:104A10000101010101010101010101010101010186
:104A20000101010110101010101042424242424296
:104A30000202020202020202020202020202020256
:104A400002020202101010102000000000000000FE
:104A50000000000000000000000000000000000056
:104A60000000000000000000000000000000000046
:104A70000000000000000000000000000000000036
:104A80000000000000000000000000000000000026
:104A90000000000000000000000000000000000016
:104AA0000000000000000000000000000000000006
:104AB00000000000000000000000000000000000F6
:104AC000000000000000000000000000F8B500BF7A
:104AD000F8BC08BC9E467047B528410029444000F8
:104AE000F8B500BFF8BC08BC9E46704705444000BE
:104AF00018F0FF7F0100000030B482B0049C5BB36B
:104B00001D46036843F480330360C9B241F0B441E9
:104B1000416083680193019B13F0010FF9D10023D9
:104B200006E0990001F58001096845F8231001337A
:104B3000A342F6D3D2B242F0B442426083680193FA
:104B4000019B13F0010FF9D0036823F48033036055
:104B5000002002B030BC70470220FAE701607047C5
:104B600082B0416083680193019B13F0010FF9D07B
:104B7000019800F00E0002B0704700007144400040
:104B800075444000774440007B4440007F4440002F
:104B9000B94440000945400081444000854440003C
:104BA0009144400009022200010100C032090400C2
:104BB0000001030000000921110100012226000765
:104BC00005810340000400001201000200000040C3
:104BD000BD3501100001010203010000B8020020F0
:104BE000BC000020F40000200180FFFFFFFF000058
:104BF0000110FFFF0210FFFF0310FFFF0410FFFF73
:104C00000120FFFF0220FFFF05000000010000005F
:104C1000544641000A010100807C797673706D6A08
:104C20006764615F5C595754524F4D4B484644424C
:104C3000403E3B3A38363432302F2D2B2A28272558
:104C4000242221201E1D1C1B1A18171615141312BE
:104C50001111100F0E0D0D0C0B0B0A090908080796
:104C60000706060505040404030303030202020207
:104C7000010101010101000000000000000000012D
:104C800001020202020203030303030303040404F8
:104C900004040505050505060606070707080808B4
:104CA0000909090A0A0B0B0C0C0D0D0E0F0F101140
:104CB000111213141515161718191B1C1D1E20216F
:104CC00022242527292A2C2E30323437393C3E41E4
:104CD00044474A4D5054575B5F63676C70757A80E8
:104CE0004747000098020020080200200000000052
:104CF00010020020AC02002009028500030100C060
:104D000032080B0002010100020904000000010149
:104D1000000209240100011E0001010C240201010E
:104D20000200020300000009240302010100010047
:104D3000090401000001020002090401010101024D
:104D40000002072401020101000B240201020210EB
:104D50000180BB0009058405000101000007250151
:104D600000000000090402000103000000092111F5
:104D70000100012226000705810340000400000015
:104D80001201000200000040BD35010100010102D6
:104D90000301000094000020A8000020B8020020B9
:104DA00049AA400069AA4000C1AA40006BAA40007D
:104DB0000000000006FFFF0901A101090209031517
:104DC0000026FF00750895408102090609071500B5
:104DD00026FF0075089540B102C0000000030000E6
:104DE00000000000000000000000000000000000C3
:104DF00000000000000000000000000000000000B3
:104E00000403090442696773637265656E000000FC
:104E10004265796F6E64000100127A00AAAAAAAAFC
:104E20000100000040030020000000002C060020CC
:104E300094060020FC060020000000000000000096
:104E40000000000000000000000000000000000062
:104E50000000000000000000000000000000000052
:104E60000000000000000000000000000000000042
:104E70000000000000000000000000000000000032
:104E80000000000000000000000000000000000022
:104E90000000000000000000000000000000000012
:104EA0000000000000000000000000000000000002
:104EB00000000000000000000000000000000000F2
:104EC00000000000000000000000000000000000E2
:104ED00001000000000000000E33CDAB34126DE67F
:104EE000ECDE05000B0000000000000000000000E8
:104EF00000000000000000000000000000000000B2
:104F000000000000000000000000000000000000A1
:104F10000000000000000000000000000000000091
:104F20000000000000000000000000000000000081
:105250000000000000000000680700206807002030
:1052600070070020700700207807002078070020D2
:105270008007002080070020880700208807002082
:105280009007002090070020980700209807002032
:10529000A0070020A0070020A8070020A8070020E2
:1052A000B0070020B0070020B8070020B807002092
:1052B000C0070020C0070020C8070020C807002042
:1052C000D0070020D0070020D8070020D8070020F2
:1052D000E0070020E0070020E8070020E8070020A2
:1052E000F0070020F0070020F8070020F807002052
:1052F00000080020000800200808002008080020FE
:1053000010080020100800201808002018080020AD
:10531000200800202008002028080020280800205D
:10532000300800203008002038080020380800200D
:1053300040080020400800204808002048080020BD
:10534000500800205008002058080020580800206D
:10535000600800206008002068080020680800201D
:1053600070080020700800207808002078080020CD
:10537000800800208008002088080020880800207D
:10538000900800209008002098080020980800202D
:10539000A0080020A0080020A8080020A8080020DD
:1053A000B0080020B0080020B8080020B80800208D
:1053B000C0080020C0080020C8080020C80800203D
:1053C000D0080020D0080020D8080020D8080020ED
:1053D000E0080020E0080020E8080020E80800209D
:1053E000F0080020F0080020F8080020F80800204D
:1053F00000090020000900200809002008090020F9
:1054000010090020100900201809002018090020A8
:105410002009002020090020280900202809002058
:105420003009002030090020380900203809002008
:1054300040090020400900204809002048090020B8
:105440005009002050090020580900205809002068
:105450006009002060090020680900206809002018
:1054600070090020700900207809002078090020C8
:105470008009002080090020880900208809002078
:105480009009002090090020980900209809002028
:10549000A0090020A0090020A8090020A8090020D8
:1054A000B0090020B0090020B8090020B809002088
:1054B000C0090020C0090020C8090020C809002038
:1054C000D0090020D0090020D8090020D8090020E8
:1054D000E0090020E0090020E8090020E809002098
:1054E000F0090020F0090020F8090020F809002048
:1054F000000A0020000A0020080A0020080A0020F4
:10550000100A0020100A0020180A0020180A0020A3
:10551000200A0020200A0020280A0020280A002053
:10552000300A0020300A0020380A0020380A002003
:10553000400A0020400A0020480A0020480A0020B3
:10554000500A0020500A0020580A0020580A002063
:10555000600A0020600A0020680A0020680A002013
:10556000700A0020700A0020780A0020780A0020C3
:10557000800A0020800A0020880A0020880A002073
:10558000900A0020900A0020980A0020980A002023
:10559000A00A0020A00A0020A80A0020A80A0020D3
:1055A000B00A0020B00A0020B80A0020B80A002083
:1055B000C00A0020C00A0020C80A0020C80A002033
:1055C000D00A0020D00A0020D80A0020D80A0020E3
:1055D000E00A0020E00A0020E80A0020E80A002093
:1055E000F00A0020F00A0020F80A0020F80A002043
:1055F000000B0020000B0020080B0020080B0020EF
:10560000100B0020100B0020180B0020180B00209E
:10561000200B0020200B0020280B0020280B00204E
:10562000300B0020300B0020380B0020380B0020FE
:10563000400B0020400B0020480B0020480B0020AE
:10564000500B0020500B0020580B0020580B00205E
:10565000600B0020600B0020FFFFFFFF0000020036
:105660005423002043000000000000000000000060
:10567000000000000000000000000000000000002A
:1056800000000000430000000000000000000000D7
:10569000000000000000000000000000000000000A
:1056A00000000000430000000000000000000000B7
:1056B00000000000000000000000000000000000EA
:1056C0000000000043000000000000000000000097
:1056D00000000000000000000000000000000000CA
:1056E0000000000043000000000000000000000077
:1056F00000000000000000000000000000000000AA
:105700000000000043000000000000000000000056
:105710000000000000000000000000000000000089
:105720000000000043000000000000000000000036
:105730000000000000000000000000000000000069
:1057400000000000413841003D33410000000000EE
:10575000C8494100C44941006448410064484100CF
:105760006448410064484100644841006448410085
:10577000644841006448410064484100FFFFFFFF66
:10578000FFFFFFFFFFFFFFFFFFFF0000010041538E
:105790004349490000000000000000000000000034
:1057A0000000000000000000000000000000415365
:1057B0004349490000000000000000000000000014
:1057C00000000000000000000000000000000000D9
:1057D000FFFFFFFFFFFFFFFFFFFFFFFF885626A130
:00000001FF
